:020000040800F2
:10000000F0FF012061DE0408C9DE0408F59801084C
:10001000C9DE0408C9DE0408C9DE040800000000C7
:10002000000000000000000000000000C9DE04081D
:10003000C9DE040800000000C9DE040881AA000827
:10004000C9DE0408C9DE0408C9DE0408C9DE0408E4
:10005000C9DE0408C9DE04083D7D0008457D0008AE
:100060004D7D0008557D00085D7D0008097B000876
:100070001D7B0008317B0008457B0008597B000888
:100080006D7B0008817B0008C9DE0408C9DE040816
:10009000CD950408C9DE0408C9DE0408657D0008A2
:1000A000799400088D930008899400087D930008D6
:1000B000B5930008C5930008D59300084979000856
:1000C0003D7900087D79000871790008C9DE0408CF
:1000D000C9DE0408594C0408654C0408714C040836
:1000E0006D7D0008C9DE0408C9DE0408C9DE040805
:1000F00069940008C9DE040859940008C9DE0408A0
:10010000C9DE0408C9DE0408E5930008C9DE040856
:100110007D4C0408894C0408F59300080D8C0408F4
:10012000A97B0008BD7B0008D17B0008E57B0008A7
:10013000F97B0008C9DE0408C9DE0408C9DE04082A
:10014000C9DE0408C9DE0408C9DE0408C9DE0408E3
:10015000C9DE0408C9DE0408C9DE0408C9DE0408D3
:10016000C9DE0408C9DE0408C9DE0408C9DE0408C3
:10017000C9DE0408C9DE0408C9DE0408C9DE0408B3
:1001800099940008C9DE0408E5790008D9790008C7
:10019000C9DE040800000000C9DE0408C9DE040846
:1001A000C9DE0408C9DE0408C9DE0408954C040849
:1001B000B1790008A5790008C9DE0408C9DE040881
:1001C000957B00080D7C0008217C0008357C000828
:0801D000C9DE0408C9DE0408C1
:0801D800A4DB0400010000009B
:10600000074BD0F8C4105B68D0F8D0205B1A9A42D6
:10601000B8BFC0F8D030012380F8FC3000207047B2
:10602000001000E0027A0B4B0168134410B413F81F
:10603000013CCC5824F00104CC50CA181368DB078B
:10604000FCD4027D5DF8044B0223934043F00C0323
:106050004B607047C07905084368C26C10B49A6100
:10606000EFF31182502383F312884168046C0B68AC
:1060700023EA0403846C2343D2B20B6082F31188B9
:10608000436981681A68096822F001021A60D0E940
:1060900008421C605A60D0E90A429C60DA60B0F89D
:1060A0006420CA6200235DF8044B0377704700BF89
:1060B000002A4FEA014C30B503460ABFE6468E4639
:1060C0008C4600F1C005002419689A6841EA0C0169
:1060D00042EA0E029A60C3E900140C33AB42F3D1DA
:1060E000D0F8C030C0F8C44043EA0E03C0F8C03056
:1060F000C0F8C84030BD00BF83695969B3F810C00B
:106100000A6830B49C6822F0010224680A60E268E0
:1061100022EA0C02E260046890F814C020680822A9
:1061200002FA0CF202403AD123480578022000FA24
:106130000CF06060002D30D0187F012830D0D3F8EB
:10614000D8200132C3F8D820EFF31181502282F316
:10615000128858681C6C026822EA04025C6C2243B4
:10616000C9B2026081F31188D3E90C405A69996879
:10617000096814605060D3E90E409460D060B3F8B1
:106180009C00C86210680124204310601C7783F8CB
:10619000D540CA681B8A1343CB6030BC7047FEE70A
:1061A00083F8D520D3F8DC000A68013022F0010220
:1061B000C3F8DC000A60F0E7C818002010B40C4CEB
:1061C0006368002B11DD002004F1080C0146DCF8A7
:1061D000943003F1C00259600C339342FBD16368E1
:1061E000013083420CF1E40CF1DC5DF8044B7047A4
:1061F000C8180020704700BF024B03EB401393F810
:10620000B5037047C8180020F8B58469D4F8DC706D
:10621000D4F8E0303D68D4F89C1003F01F0304224A
:106220009A4015420E6804F19C0017D016F0040F36
:1062300014D00B689B0603D40B6823F004030B6097
:10624000D4F8CC307A6013B19847D4F89C104B68DE
:106250001BB90B6823F001030B60F8BD02229A40C2
:10626000154218D016F0020F15D00B689D0606D403
:106270000B6823F00A030B60012384F8C130D4F8C3
:10628000C8307A60002284F8C020002BDFD0984705
:10629000D4F89C10DBE708229A402A42D7D0320774
:1062A000D5D50A6822F00E020A60012202FA03F331
:1062B0007B60002384F8C030D4F8D030C4F8D820F4
:1062C00084F8C120002BBFD1C1E7D0E90920131AFF
:1062D00058425841704790F8573830B53BB990F85C
:1062E000551890F856380124DAB2914200D830BDE2
:1062F000B0F85E5804FA03F22A43A0F85E2801338E
:10630000F2E70379024613F0010006D0D2E9073123
:10631000D2685B1A013A03EA0200704710B50379AC
:1063200013F0010304460ED0FFF7EBFF034650B114
:10633000226A6369E1689B5C0132B2FBF1F001FB08
:106340001022DBB22262184610BD03799B070AD5E2
:10635000436A8269D154436A02690133B3FBF2F1A3
:1063600002FB113343627047704701717047037934
:10637000014613F0020007D00B69D1E90921013B66
:10638000521A1A40D2B2981A704700BF3D4BD3F848
:1063900004358BB93C4A4FF4A87002232A214010DF
:1063A000C2F8A804C2F89834C2F89C34C2F8A034E9
:1063B000C2F8A414012070473449334AA1FB0313E7
:1063C0009B0C10B4A3F108010324C2F898441329CC
:1063D00027D8DFE801F0462626262626262646264A
:1063E0002626262626264626310A294B294903EB4E
:1063F00040031B8A5B00A3F5AB7381FB0301DB1732
:10640000C3EBA1035B00263303EBC300032102248B
:10641000B0F50C7FC2F89C44C2F8A014C2F8A434B2
:1064200003DB00205DF8044B70474010C2F8A8045D
:106430005DF8044B01207047154B174903EB4003EF
:106440001B895B00A3F5A97381FB0301DB17C3EB79
:10645000E1035B001A3303EB430003EB80000221EE
:10646000D5E70B4C34F810004000C3F3C401B0F57D
:10647000A87344BF6FF4A073C3181B115B002A33C9
:10648000D800C4E700200040C818002083DE1B436A
:10649000E8FC0408398EE3384FECC44E10B584464E
:1064A0004FEA810E102312F4004F14BF0E2407246C
:1064B0005200013BCCF8004092B2F444F3D100EB1F
:1064C00081128C01035142F82130122010BD00BF0F
:1064D00010B584464FEA810E0424130B03EB4303EB
:1064E00018331201013CCCF8003092B2F444F4D1DC
:1064F00000EB01130A01845043F82140062010BD2F
:10650000704700BF704700BF034B00EB400003EB38
:10651000C00393F8BD047047C8180020064B93F8D9
:106520006C25824283BF00EB400003EBC003D3F82D
:10653000C0040020704700BFC81800200B4890F826
:106540006D1589B101EB4101002310B4490000F23F
:10655000AC401C4650F82320063302B114608B4235
:10656000F8D15DF8044B7047704700BFC818002091
:106570000B4890F86D1589B101EB4101002310B46F
:10658000490000F2AC401C4650F82320063302B10B
:1065900014608B42F8D15DF8044B7047704700BF20
:1065A000C8180020204B1B78002B3CD12DE9F0416E
:1065B0001E4C94F86D25A2B31D4E04F2AC42502738
:1065C0004FF02C0E1D4607E094F86D1552F8180B8D
:1065D00001338B42056024DA117C0029F4D0516824
:1065E000880AA0F5801006EB000854284FF0FE0C36
:1065F00098BF98F818C0EFF3118087F31288D1F88C
:1066000024800EFB0C4C08F10108CCF89885D1F8D9
:1066100014C04CF0010CC0B2C1F814C080F3118852
:10662000D2E7BDE8F081704700000020C8180020C4
:10663000E8FC040800EE100AB8EE400A704700BFFC
:10664000BCEEC00A10EE103A98B2704707280AD87C
:10665000064B4FF49A7202FB0033B3F8AC07B0FA62
:1066600080F0400970470020704700BFC818002024
:10667000072807D8044B4FF49A7202FB003301221B
:1066800083F8AE27704700BFC8180020072808D835
:10669000044B03EB401393F8B42312B1012283F8A7
:1066A0009A237047C8180020072808D8054B03EB29
:1066B0004013B3F89803B0FA80F040097047002007
:1066C000704700BFC8180020054B93F86C25824224
:1066D00086BF03EB4013D3F8A4030020704700BF2C
:1066E000C8180020012343770020704708B50346EF
:1066F0008269006BD96A02449A6101B1884700201F
:1067000008BD00BF436A1B681B6A5B685B78024672
:1067100013F0010008BF5077704700BFC26281616B
:10672000704700BF704700BF043070470B4B93F8B1
:106730005820596D0244D2B283F8582093F858205B
:1067400001441206596505D593F8582082F080025D
:1067500083F85820024B01225A707047C02900204C
:10676000000000202DE9F047144FFD6DED0A1FD009
:106770000026B14607F1940874193B6E1048D3F80F
:1067800028A0C7F88C9004EBD47464101023424600
:10679000E102D0470F280BDD0A4B03F1100153F83B
:1067A000042B013207D18B42F9D12546B542E3DCF7
:1067B000E802BDE8F087661CF8E700BFC0290020AA
:1067C000202A0020542A0020194BD3F8A410D3F813
:1067D000A8208A1A322A05DCD3F8BC208A1A002A9B
:1067E00011DC7047D3F8AC1049B193F8B820888811
:1067F000096802F00102120100FA02F28A61002225
:10680000C3F8BC207047D3F8AC206AB110689288F6
:1068100010B44469224218BF120432315DF8044BAF
:106820008261C3F8BC1070473231C3F8BC107047A6
:10683000C0290020074AD2F8AC304BB192F8B820FA
:106840009988186802F00102130101FA03F38361C9
:1068500000207047C0290020044B4FF40070D3F88B
:10686000C830108000200B60704700BFC029002096
:1068700000207047012070470120704700207047BA
:10688000164AD0F8C0305268D0F8B81010B5044697
:1068900073B1501A83420BDC94F8B030C4F8B820BE
:1068A000012B10D0D4F8B4300133C4F8B43010BD8B
:1068B000D4F8C430C4F8B8200B44C4F8BC3094F801
:1068C000B030012BEED104F1C801201D3DF022F9BA
:1068D000D4F8B4300133C4F8B43010BD001000E077
:1068E000CB070DD470B590F82830C468012B8CB05C
:1068F00007D0B4F1807F01D9012303770CB070BDBC
:1069000070471B4A1B4BD2F8F8505B68466AB5EBE0
:10691000530F4FEA530228D20721022352085B008B
:1069200095429BB201D20139F8D1B4F1807FB38096
:10693000E4D9012201A9002302770291B72402A918
:106940003046CDE903328DF814208DF82820CDE9AA
:106950000633CDE908338DF804400B933DF0DAF8A7
:106960003268136A002BFCD1C8E70223DDE700BFC1
:10697000C02900200000002030B590F82830012BFD
:106980008BB0044608D0407F10B901200BB030BD59
:10699000002363770BB030BD456A2B681A7B2ABB96
:1069A000637F002BF1D01449009114490191022119
:1069B000002301220291284669468DF80C208DF8AB
:1069C0002020CDE90433CDE9063309933DF0A2F848
:1069D0002A68136A002BFCD1094B93F8FD30D84389
:1069E00003F0010300F001006377D3E71B6A002B7B
:1069F000D6D00020CAE700BF08000020BC2A002033
:106A0000C029002030B504468BB094F82830012B03
:106A100008D0637F0BB10023637701200BB030BD3A
:106A20001B6A23B1656A2B681A7B002AF8D1637F41
:106A3000002BF2D01049009110490191022100234E
:106A400001220291284669468DF80C208DF82020FD
:106A5000CDE90433CDE9063309933DF05BF82A68AC
:106A6000136A002BFCD1064B93F8FD3003F00102B2
:106A7000DB076277D1D5C8E708000020BC2A0020D8
:106A8000C029002030B5204A204B95B0044620484C
:106A90000493CDE900200023151D083ACDE90A230F
:106AA000CDE90E331B480990626A207F0595069355
:106AB000109313931193012312688DF80C30022563
:106AC00007938DF820308DF834308DF84830031D51
:106AD00002950C93136A002BFCD198B10E4B0A0E51
:106AE0005A730E330A0A080C5A7099701870606A4B
:106AF00069463DF00FF8636A1A68136A002BFCD1EF
:106B000015B030BD054BEDE7140000200567000807
:106B1000C02A0020E5660008000000200D000020CB
:106B200010B5044694B050220749684648F08EFEDE
:106B3000606A69463CF0EEFF636A1A68136A002BCC
:106B4000FCD114B010BD00BF58FD0408F8B50546CF
:106B5000406A0068046A002CFCD12C7FA869002CD4
:106B600036D0244C060E6677052704F11E06B07059
:106B70004FEA104C000A86F800C07070086867651C
:106B800016682066012B4FF00000A6662E63A067F2
:106B900023D0022B1BD1536820674A6862671E44CA
:106BA000154A84F86C000121E3672E6384F8801095
:106BB000C4F88420114B6A7F686AA3F11401002A8B
:106BC00008BF19463CF0A6FFEB6A6BB1286BF8BD15
:106BD0000B4E0427A6F11D04C9E7074A84F86C3060
:106BE000C4E91C20E067E5E76B6A1A68136A002BAA
:106BF000FCD1EBE700000020ED6600083800002023
:106C00001D00002000B583B081610192049A0093B9
:106C1000C26201236A4601A9FFF798FF03B05DF83D
:106C200004FB00BFF0B50746406A066895B01D46F4
:106C3000346A002CFCD1CDE90944CDE90E44CDE9FC
:106C4000104406948DF820401394304C0B9204F1BC
:106C5000A40300932E4B01930223029301232D4A98
:106C60008DF80C308DF834308DF848303B7F04922D
:106C700004F19C0205921A1D0C950792002B3ED040
:106C80000B0E84F89D3004F19E03234E6268D6F803
:106C9000F8C09970080C090A59701870BCEB520FB3
:106CA000786A4FEA52012DD2072302224908520086
:106CB0008C4592B201D2013BF8D17B7F8280E3B157
:106CC00069463CF027FF786A03681A6A002AFCD1FB
:106CD0006268D6F80831B3EB520F4FEA520113D273
:106CE00007240222490852008B4292B201D2013C91
:106CF000F8D18280284615B0F0BD05A9E1E704F17E
:106D00009D03C2E70222D8E70222F2E7000000203A
:106D1000C42A002005670008C0290020F0B5826958
:106D200092F8BC30012B8BB0054625D0023B012BDD
:106D30002DD892F82C31D26F164C63F07F0313706C
:106D40008669D6F880305F1C0FCCEC46ACE80F00AB
:106D5000F36FCDE900370FCCACE80F0094E80300E7
:106D60008CE80300694606F110003CF0D3FEAA69E6
:106D700011690B6A002BFCD1D2F880305A8852BAC4
:106D8000EA819A8852BA2A82DB885BBA6B82012038
:106D90000BB0F0BDA8FD0408F0B590F8BC30D0F8F9
:106DA0008060012B8BB0044648D032D9023B012BC6
:106DB0002CD890F82D31C26F434D63F07F031370D0
:106DC000D0F880305F1C0FCDEC46ACE80F00E36FCD
:106DD000CDE900370FCDACE80F0095E803008CE853
:106DE0000300694604F110003CF094FE2269136A26
:106DF000002BFCD173885BBAA4F8B030B3885BBABF
:106E0000A4F8B230F3885BBAA4F8B43001200BB018
:106E1000F0BDC36F4FF0FF321A605A609A60DA60BB
:106E2000D0F8C0300522B3F57A7FC0F8D0201FD843
:106E3000032380F8BC3001200BB0F0BD90F82C216A
:106E400090F82D319B1A5B100133DBB206EB430245
:106E500036F813305BBAA0F8B03053885BBAA0F8AC
:106E6000B23093885BBAA0F8B43001200BB0F0BD0B
:106E700003691A7B1AB35B690BB390F87830F3B1EE
:106E800090F82C31C26FC4F8840063F07F03137054
:106E900090F82C1190F82D31D0F880200B48C4F8D0
:106EA000E4005B1A07330121C4F8DC30E36F84F897
:106EB000E0100A44C4E9353284F8BC10A6E7022386
:106EC00084F8BC30A2E700BFA8FD040801600008F8
:106ED000F8B50C4B1D685A69154005405D617DB1E0
:106EE000094F0126B5FA85F4C4F11F0407EB8403AA
:106EF00006FA04F4D3F80C0103689847A543F1D1CE
:106F0000F8BD00BF00040140C02900202DE9F8436E
:106F10000269C36812EA030828D005460E464FF0FE
:106F20000047B8FA88F327FA03F2D2431B3B2A61E1
:106F300008EA0208042B16D8DFE803F03B30251AD4
:106F40000300B36A002B3FD003F1FF3900231FFA7F
:106F500089F9B362746A34B1236820464946984778
:106F60006468002CF8D1B8F1000FDAD1BDE8F883DD
:106F700070680028F7D0696B036889B29847B8F148
:106F8000000FCED1F2E7B0680028ECD0A96B0368FF
:106F900089B29847B8F1000FC3D1E7E7F06800283D
:106FA000E1D0E96B036889B29847B8F1000FB8D116
:106FB000DCE730690028D6D0296C036889B298478D
:106FC000B8F1000FADD1D1E7EB6A1FFA83F9C1E741
:106FD0002DE9F8430768D7E90415A8610A7D0E6812
:106FE0002C68022303FA02F242F00C0272602A7D3E
:106FF000934043F00C036360097A184BBA69581840
:1070000010F8018C56F808C02CF0010C46F808C0A6
:1070100095F808904B44304613F8015C635923F00F
:1070200001036351635943F00203635143F0A8FC29
:10703000FA694946204643F0A3FC56F808307A68BE
:1070400043F0010346F80830635943F001036351EC
:10705000536843F003035360BDE8F883C079050823
:10706000F8B5314D05EB401393F8B43303B9F8BDCF
:107070002E4B93F84CE193F84D2196454FEA40147E
:107080000CD002EB420C03EBCC0C9CF85061771E49
:10709000012F4FEA420C3AD9032E33D0244B2C4413
:1070A00003EB4010A4F898130FF036FF2B78D4F8B8
:1070B000B023D4F89C138BB1D2F8943001248C40C7
:1070C00003F1C001420010F4004F90B202D15A689F
:1070D00022435A600C338B42F4D1F8BDD2F894307D
:1070E000012401F11002944003F1C001420010F4A8
:1070F000004F90B202D15A6822435A600C338B423F
:10710000F4D1F8BD561C06F003067645C6D094446B
:1071100003EBCC03034493F85D110029BED02B1977
:10712000012283F89A23B9E7C8180020C02900205B
:10713000601C002070B5384C4FF49A7303FB004379
:1071400093F8BB3703B970BD344D95F84CC195F831
:107150004D319C450ED003EB430205EBC20292F881
:1071600050E10EF1FF36012E4FEA430231D9BEF154
:10717000030F29D04FF49A7303FB00F0284B04440B
:107180001844A4F8AC170FF0C7FE95F8B411D5F861
:10719000B031024669BB0121D4F8DC089847D4F825
:1071A000D858B4F8B837D4F8D428B5F8B41019437F
:1071B0005368A5F8B4106FF30F03034353601368CB
:1071C00043F00103136070BD5E1C06F003066645C4
:1071D000D0D01A4405EBC202024492F85D11002996
:1071E000C8D04FF49A7303FB0043012283F8AE2703
:1071F000C0E7D4F8B417D4F8D8084979D0F8B0006B
:1072000001F0FC01084404219847D4F8D8388000E4
:10721000A3F8AC0070BD00BFC8180020C029002032
:107220007420002086E700BF10B5044647F008FD33
:1072300081B22046BDE8104012E700BF10B50446F9
:1072400047F0FEFC81B22046BDE8104072E700BF67
:1072500038B50B4D00EB400005F2AC4303EBC00327
:1072600093ED027AD3ED037AE7EE007AC400254469
:10727000B0EE670A47F0E4FCD5F8AC34186038BDCE
:10728000C818002070B5274C94F84C2194F84D3163
:107290009A4242D194F878275AB302EB4201224B2A
:1072A00094F8B401C2EBC10C03EBCC0CD4F8B821B8
:1072B00008B31E4D1E4C40F20D3E00E01A68D3F894
:1072C000A810B3F8AC004E682E4030434860086800
:1072D00040F001000860D2F8DC13214041EA0E01C1
:1072E000C2F8DC13D168B83341F480716345D160D2
:1072F000E4D170BD1A6811689C8821F0800111608A
:10730000D4625062B3F8B410D468B83321436345F3
:10731000D16023F8040CEDD170BD45F021FF0028A9
:10732000B8D170BDC0290020782B00200000FFFFDD
:10733000E0E0FFFFF8B5A0F507642379DB0725D56A
:10734000657994F8543805F001073D46FBB1D4F84F
:1073500048341A68D36A5B08536294F8583823B1EA
:10736000B4F862380133A4F86238606C85F001012A
:1073700043F0F6FC012384F85738002384F855388D
:1073800084F85638A4F85E3884F85438F8BD94F878
:107390005768012E04BF94F8553884F856382046B3
:1073A000FEF799FF4EB9012384F8573887EA0301A5
:1073B000606CBDE8F84043F0D3BC002384F8573834
:1073C0003946F5E770B5094C05460726013E00D160
:1073D00070BD94F9000012F069FE031E04DBEA1888
:1073E00061789171A278EA540434EFE7D0FD040883
:1073F0002DE9F843DDF820800F46154600212022B4
:1074000004461E4648F044F9B8F1000F0CD0D8F8F5
:107410000030E3811B0C2382D8F80430B8F80A202E
:10742000E3821B0C62822383384646F0A7FCEB06FE
:1074300019D4431EB8B107EB000C01E0013B12D395
:107440001CF801EDBEF12E0FF8D1C01A421E032A1E
:10745000A8BF0322082B03F10109A8BF0823904607
:10746000B9441A4606E008280246B946A8BF0822D1
:107470004FF000084FF02033394623606360204608
:1074800048F0E4F904F10800154B238142464946CF
:10749000837048F0DBF9611EE21D11F801CFACF1F9
:1074A0006103192B9CBFACF1200C81F800C0914204
:1074B000F3D104F10A0011F8013FA3F16102192A86
:1074C0009CBF203B0B708142F5D118232373330CF2
:1074D000A382E572099B6683E361BDE8F88300BF80
:1074E000202020002DE9F04FDFF844B4DBF8A400A1
:1074F00085B0CBF8A800002B5ED013440C4617468D
:1075000001F5FE7A99461DE0002F62D0DBF8D430F9
:10751000BB4200F0C480DBF8D030BB4200F0F68004
:10752000DBE93631BB424BD8B94200F26E81791AA1
:10753000204640F0B9FB01374F4504F500740AF5C9
:10754000007A39D0DBF8E030BB42DDD8DBF8F05010
:10755000FB1A296BDA0802328A4203F0070602D3CB
:10756000AB6B9A420BD929461046029240F06CFB55
:10757000029A0546002800F06881CBF8F0002B79CC
:10758000002B40F01C81D5F82880B8F1000F00F0E6
:1075900055812B6BD21AEB6806EBC20203EB422239
:1075A00020462B464FF400710137C0474F4504F584
:1075B00000740AF5007AC5D1002005B0BDE8F08F4F
:1075C000B942B4D94FF400720021204648F060F867
:1075D000B1E74FF400723946204648F059F880234D
:1075E00084F8BE310C2384F8C231DBF8D010C44AD1
:1075F000DBF8C830C4F8C6119142C4F8CA3100F3B0
:107600000981C04AC04D82FB010285FB01050A4485
:10761000C817C0EB6212C0EB2530BC4D84F8C10125
:1076200085FB0265C2EB82168010891B013120F0B8
:107630003F0015440843D117C1EBE5110A4484F813
:10764000BF21AF4A84F8C001013B934200F3EE80B2
:10765000AC4AAD4882FB031280FB03101A44D917D1
:10766000C1EB6212C1EB2031A84884F8C51180FB40
:107670000250C2EB821589105B1B013321F03F01E0
:1076800010441943D317C3EBE0131A4484F8C41110
:1076900084F8C3214AF65523A4F8FE314BE74FF096
:1076A000FF3384F8EC3184F8ED3184F8EE3184F85E
:1076B000EF315223237063706123A37084F8E731A4
:1076C0004123E37084F8E6317223002584F8E43125
:1076D00084F8E531DBF8E830C4F8E8314FF4F072B3
:1076E0002946201D47F0D4FF552384F8FE316FF062
:1076F0005503C4F8F051C4F8F451C4F8F85184F8B3
:10770000FC5184F8FD5184F8FF3114E74FF4007206
:107710000021204647F0BCFF7D4B03CB45F6EB0331
:10772000238090230222C4F80710A3700821F823B5
:10773000C4F80300617322746375DBF8C8302273E8
:10774000A27384F82C20DBF8D0209B1A2362DBE99B
:1077500036239B1A63620023E372E3736377A37794
:10776000E37784F82D3084F82E3084F82F3084F8B5
:107770003130684BA361684BC4F842303E23237715
:10778000012384F83030654A802384F8403084F83F
:1077900046104AF65521A4F8FE1103CA604BC4F8FE
:1077A0004700C4F84B1003CB1388A4F84F309378EC
:1077B000C4F85200C4F8561084F85130BBE64FF4B8
:1077C00000720021204647F063FF002E44D12B6C4D
:1077D00004F12008002B7BD02B6B52491122CDE9FC
:1077E00000662046FFF704FE2B6C1A6C002A7ED040
:1077F0001B6B4D49CDE9006640461122FFF7F8FDAD
:1078000004F140084FF4E0736DE0F91A204640F0AF
:107810004BFA90E6FF2284F8C1214FF6FF72A4F8DC
:10782000BF21374A013B93427FF712AFFF2384F811
:10783000C5314FF6FF73A4F8C3312BE741464FF42F
:107840000072204647F024FF75E6384A231F43F8AC
:10785000042F9A45FBD16EE6D5E910253301002AA5
:1078600043D0023B002D3FF466AE013BAD6CF9D135
:10787000A0464FF40073002D3FF45DAECDE9027ACF
:1078800008EB0306A24608E00024CDE900C4FFF798
:10789000AFFDAD6CBDB1B04515D02C7929682B6B0F
:1078A000404605F11C0C112208F12008002CEBD1F8
:1078B0006A792C6942F02102CDE900C4FFF798FDF6
:1078C000AD6C002DE7D15446029FDDF80CA032E6E6
:1078D000CDE900663346DBF8CC1008222046FFF7DE
:1078E00087FD4FF4F0736D6CC5E7013BBAE7CDE956
:1078F00000660D49334640461122FFF779FD7FE7C8
:10790000FF03FB00832008829755454181808080DA
:107910000C7905083F00FF0029940E0D1879050821
:10792000247905080479050808790508DEADBEEF5D
:10793000C029002000207047704700BF01483DF07B
:107940005DBE00BF54310020084810B4D0F8943711
:10795000D0F8C84799691A682CB1234600F2947090
:107960005DF8044B18475DF8044B7047C0290020B0
:1079700001483DF043BE00BFB8310020084810B4B4
:10798000D0F8F837D0F82C4899691A682CB12346FA
:1079900000F5FF605DF8044B18475DF8044B704735
:1079A000C029002001483DF029BE00BF1C32002044
:1079B000084810B4D0F85C38D0F8904899691A6833
:1079C0002CB1234600F65C005DF8044B18475DF8C7
:1079D000044B7047C029002001483DF00FBE00BF96
:1079E00080320020084810B4D0F8C038D0F8F448ED
:1079F00099691A682CB1234600F50C605DF8044BB8
:107A000018475DF8044B7047C029002010B1036887
:107A100082889A61704700BF10B1036882889A62B9
:107A2000704700BFD3B20F2B21D8124B00B503F122
:107A30006F0E02E00333734516D093F800C08445FF
:107A4000F8D193F801C08C45F4D10B489B7802EB38
:107A5000420200EB8201A83000EB8200C1F8B03096
:107A600081F8A8305DF804FB00205DF804FB0020DD
:107A7000704700BFE8FD04080000002010B40C4C63
:107A8000002304F60C1C01E0152B0CD003EB430281
:107A900001331CF802108142F6D1144494F90E0906
:107AA0005DF8044B70474FF0FF305DF8044B7047B2
:107AB000C029002030B5124C002304F5B87C02E048
:107AC00001331F2B1AD05CF833508542F8D10CEBF0
:107AD000C30EDD009EF804E08E45F1D1094802EBAB
:107AE00042022C4400EB820394F87511C3F8B010E5
:107AF000A83000EB820083F8A81030BD002030BD14
:107B0000E8FC0408000000200348D0F8783113B1E5
:107B100000F5B47018477047000000200348D0F803
:107B20009C3113B100F5C670184770470000002063
:107B30000348D0F8C03113B100F5D870184770472A
:107B4000000000200348D0F8E43113B100F5EA70DA
:107B500018477047000000200348D0F8083213B1DE
:107B600000F5FC7018477047000000200348D0F86B
:107B70002C3213B100F50770184770470000002041
:107B80000348D0F8503213B100F510701847704711
:107B9000000000200348D0F8743213B100F51970CA
:107BA00018477047000000200348D0F8983213B1FE
:107BB00000F5227018477047000000200348D0F8F5
:107BC000BC3213B100F52B7018477047000000203D
:107BD0000348D0F8E03213B100F53470184770470D
:107BE000000000200348D0F8043313B100F53D70C5
:107BF00018477047000000200348D0F8283313B11D
:107C000000F5467018477047000000200348D0F880
:107C10004C3313B100F54F70184770470000002037
:107C20000348D0F8703313B100F558701847704707
:107C3000000000200348D0F8943313B100F56170C0
:107C40001847704700000020104A114B013800EB24
:107C5000C00002EB80020F48D2F86821996C824282
:107C600014BF02220122114382B09964996C0A4028
:107C70000192019A9A6C42F004029A649B6C03F0A0
:107C800004030093009B02B0704700BF0000002077
:107C90000010024000000240F0B50138194C00EB22
:107CA000C00004EB80041D461748D4F8683183B047
:107CB000834214BFA120A0200E46174640F0CAFB05
:107CC000124B9A6C42F004029A649B6C94F97D0109
:107CD000C4F8786103F004030193B909019BC4F867
:107CE000805140F05BFA94F97D31002B08DB580994
:107CF000074903F01F03012202FA03F341F8203081
:107D000003B0F0BD0000002000000240001002405F
:107D100000E100E0800AA0F58010542807D8054B48
:107D200003441B7E0B2B02D8034AD0567047002019
:107D3000704700BFE8FC0408B07905080120FFF790
:107D4000C7B800BF0220FFF7C3B800BF0420FFF789
:107D5000BFB800BF0820FFF7BBB800BF1020FFF777
:107D6000B7B800BF4FF47870FFF7B2B84FF47C405B
:107D7000FFF7AEB830B1036882881B691A4214BF9E
:107D800001200020704700BF70B50D4682B0164636
:107D90000446B8B1036803F138439B0A0B4A134405
:107DA00093F8680240F056FBC5F38103CDE9003635
:107DB00005F01302A1882068C5F3411343F014FBBA
:107DC00002B070BD4FF0FF33E8E700BFE8FC0408E5
:107DD00000B1D9E770472DE9F84FBD4F642303FB8D
:107DE00000730646D3F87C47D3F88487D3F88857C6
:107DF000002C00F06281B8F1000F04D098F9063031
:107E0000002B40F05A8125B195F90630002B40F047
:107E10005481731CDBB2B8F1000F04D0152288F82E
:107E2000062088F8073015B11622AA71EB714FF0C1
:107E3000640A0AFB06FA07EB0A0994F8280040F0E6
:107E400009FB2946404645F091F899F88E3799F894
:107E50008C27002B0CBF4FF01E0B4FF03E0B404603
:107E60005946FFF7B5FF28469A4D99F88D27594690
:107E70005544FFF7ADFF4C220021284647F008FC8F
:107E8000D9F87C379FED947A5B68C9F89437934BA7
:107E9000B9F890A79A68924B9FED925AC2F30222CA
:107EA0001344B0EE084A93F870228F4B5B6802F0DF
:107EB0001F02D34007EE903AF8EE677A4FF0000CBD
:107EC000C7EE275A40F2145807EE90AA9FED877A22
:107ED000F8EEE77A25EE844AC7EE274ADFED847A8A
:107EE000B0EE007AE5EE877AA5EE875A74EEE72ABF
:107EF00037EE856AF7EE003ABAF5C87F0CF1010E4D
:107F000007EE90EAD5BF4FF49672782264233223AD
:107F10001344F8EEE76A07EE903A66EEA56AB8EE0B
:107F2000E77AA2F13202C7EE267AD5BF4FF416796E
:107F30004FF4827941464FF4FA7107EE102A77EE3A
:107F4000E37AB8EEC77AFCEEE77A37EE447A17EEBA
:107F5000903AC7EE267A01EB0902FCEEE77A17EEBB
:107F6000900A07EE909AB8EEE73A07EE902A23EED1
:107F7000243AF8EEE77A83EE277A37EE453A32EE86
:107F8000C77AC3EE267A77EEE37AFCEEE77A17EE4D
:107F9000901AC7EE267A77EEE37AFCEEE77A17EED0
:107FA000902A02F1020909EB010B07EE90BAF8EEF4
:107FB000677AB0EE467AA6EEA77AF4EEC74AF1EEFB
:107FC00010FA7EDC43EA00095FFA89F9B9F10F0F74
:107FD00079D841EA02091FFA89F9B9F1FF0F72D87D
:107FE0001B05000400F47F0003F07F630343414856
:107FF00043EA0C7300EA01210B4392B2134364225B
:1080000002FB067628460027C6F898370123C6F8F3
:10801000A037C6F89C77C6F8A477C6F8A877C6F844
:10802000B077C6F8B47743F091F996F8D537202B9E
:10803000D9B21AD196F8D437012B16D0242386F85A
:10804000D537D6F894371A6822F001021A601A68F8
:1080500022F480521A601A681A601A6842F001020B
:108060001A6086F8D51786F8D47794F92A0000218B
:1080700040F094F894F92A2094F82A30002A08DB7A
:108080005909012203F01F0302FA03F31A4A42F8C6
:10809000213094F92900002140F080F894F929203A
:1080A00094F82930002A08DB5909012203F01F0344
:1080B00002FA03F3104A42F82130BDE8F88FF44683
:1080C0001AE701316FE7BEF10F0FF8D1002396E7F1
:1080D000C029002054310020286B6E4E0010024051
:1080E000E8FC040800001643000000200024744946
:1080F0000000704200FFFF0000E100E008B1002234
:1081000042E6704770B50F4C94F86C65BEB104F54B
:108110006674002504E00135B54204F120040ED058
:10812000237F002BF7D0E06800220028F3D0217DC8
:108130000135FFF729FEB54204F12004F0D10120FA
:1081400070BD00BFC818002070B590F8BE311C0982
:10815000013C052C0FD81A4E06EB44020546B2F836
:10816000780203F00F0340FA03F2D20703D595F823
:10817000C121012A01D0012070BD9A40013A10406E
:10818000264447F031FC96F884320E4A034402EB51
:10819000C30452F83320A38810691840ECD00023A0
:1081A00095F8BF2185F8C13102212046FFF7ECFD8B
:1081B000D5F82021136843F008031360DBE700BF04
:1081C000E8FC04080C330020800000F1804000F53A
:1081D00014500068704700BF800000F1804000F537
:1081E00014500160704700BF10B4254B2548996DAD
:1081F000254A41F0805183B09965996D01F0805115
:1082000001910199016841F480710160996D41F417
:1082100080619965996D01F4806100910099D3F8AE
:10822000901041F40041C3F89010FF24CA2053215C
:10823000546250625162D3F89430DB0014D4134B73
:1082400013490022C3F80425C3F80825C3F80C25F8
:10825000C3F81025C3F81425C3F81825C3F8001572
:1082600003B05DF8044B7047A2F50062084BD2F8EA
:1082700000259A42E3D103B05DF8044B704700BF7C
:108280000010024000700040002800400020004024
:10829000316665422DE9F84FD0F828618368F5B260
:1082A0001F68534B083DA3FB05352D09044626F0F6
:1082B000FF08013500F1F80A00F1BC0929464046E3
:1082C00042F0A0FBD4F8E8200023B2F5807F84F8C8
:1082D000EC301CD00ED9B2F5804F18D070D8B2F562
:1082E000806F14D0B2F5805F6FF4006114BF382343
:1082F00004230FE0102A78D06BD8012A4ED0042A2C
:1083000016BF6FF400616FF00801382302E06FF0D0
:1083100008010423524607F1180A38465AF803C0E8
:1083200001EA0C014AF80310D4F8E8B0594642F0CB
:108330001FF9BBF5807F2DD01DD8BBF1100F51D098
:108340002FD8BBF1010F02D0BBF1040F2CD10827AD
:10835000DAF800303B43CAF800301023C4F8C430C8
:108360004A462946404642F00BFB336843F002037D
:108370003360BDE8F88FBBF5804F0BD019D8BBF543
:10838000806F07D0BBF5805F0ED107F11C0A4FF458
:108390000067DDE707F11C0A0827D9E76FF008013D
:1083A000B8E7BBF1400FD2D00AF1380A4FF40067AA
:1083B000CEE7BBF5803FF7D107F1500A0827C7E7A2
:1083C000B2F5803F14BF6FF400616FF008013823ED
:1083D000A0E7402A15BF6FF400616FF00801382351
:1083E000002397E74FF40067B2E76FF4006191E76D
:1083F000CDCCCCCC2DE9F0472423D0F82051C0F8C7
:10840000A0312A688168002322F001022A602B60D3
:108410006B60AB604279C0F8A83180F89C31C0F83D
:10842000A031C0F83831C0F8A431C0F8403193020F
:1084300003F48053C0F828311303C0F8241103F467
:108440000053AC49C0F82C31130203F480638D4211
:10845000C0F8303104BF0423C0F844310379044626
:1084600003F001084FEA880113F0020600F5907747
:10847000C4F8341102F0010000F0CC8041F0080192
:10848000C4F83411002840F0D78094F8C0314BB1C3
:10849000D4F8483143F00803C4F848314FF400439E
:1084A000C4F85831D4F8A0312423C4F8A0312B6883
:1084B00023F001032B601307384640F1E4803DF0C0
:1084C000FFF9012817D0D4F84831002B40F0F28092
:1084D0006B6823F490436B60AB6823F02203AB60BE
:1084E000AB6843F00803AB602B6843F001032B60DB
:1084F000384642F047FBB8F1000F5FD0D4F8FC805B
:10850000B8F1000F00F0AC80D4F80431C4F8A0300A
:108510008023202104F13C0A4FF00009E3644FF46A
:108520008053C4E916135046C4E91199C4E914995B
:10853000C4F83C8043F058F950463CF0BFFED4F8F4
:10854000A431C4F898A1202B676633D162698AB33D
:10855000E36899B271B394F89C0101282AD0A4F879
:108560007C116549A166654994F86000E16664493B
:10857000216701214FF0220C8842C4F8A891C4F869
:108580007821C4F8749084F89C11C4F8A4C108D070
:1085900084F8601094F86110012900F0938084F849
:1085A00060901023C4F8A831002384F89C31202364
:1085B000C4F8A031D8F80430C4F8143146B3D4F864
:1085C0000051DDB1D4F80821C4E92752102200235C
:1085D000C4F8A4208022C4E92A3204F19C064FF496
:1085E00080523046C4E92C33C4E92E3243F0FCF803
:1085F00030463CF063FE002855D0FEE7D4F8AC319D
:108600001A6842F080021A601A6842F040021A604A
:10861000BDE8F08700283FF438AFB8F1000F3FF411
:1086200034AFD4F8483143F00203C4F848314FF472
:108630008033C4F8503128E7D4F84831B8F1000F3E
:1086400005D04FF4803143F00203C4F8501143F0D9
:108650000103C4F848314FF40033C4F84C3114E737
:10866000D4F8AC311A6842F480721A609A6842F009
:1086700001029A601A6842F020021A601A6842F0F9
:1086800010021A609AE73DF01BF901283FF433AF5E
:10869000D4F8483193B96B6823F490436B60AB68AE
:1086A00023F02A031FE7C4F89461C4F8C47068601B
:1086B000BDE8F08738463DF0DBFB09E738463DF082
:1086C000D7FBE8E79BB2504605F124013CF084FE5D
:1086D00000287FF466AF84F89C012B6843F4807314
:1086E0002B60AB6843F00103AB60AB6843F0400321
:1086F000AB605FE700800040410F0408750F04087D
:10870000790F040838B50409013C052C1AD80F4D1F
:1087100005EB440200F00F03B2F8780240FA03F2CE
:1087200012F0010210D0012202FA03F3013B1840BB
:10873000254447F059F995F88432054A034402EB81
:10874000C30038BD002038BD104638BDE8FC040821
:108750000C33002070B5002486B0CDE90144CDE98A
:1087600003440DF1040CC0E93544C0E93744C0F8B6
:10877000E440054600F1E80EBCE80F00AEE80F004B
:10878000CEF8004095F80101059444F23B36A5F877
:108790002C6108B906B070BDFFF7B4FF0E4B04465C
:1087A000294688B12622C28041F80C3F42F014FFCE
:1087B0000A49A2880868B2FA82F24FF00043D34017
:1087C00003430B6006B070BD41F80C3F06B0BDE836
:1087D000704042F001BF00BF816800080004014002
:1087E0002DE9F84F6F4EC0EB001306EBC303D3F82F
:1087F0004C4C002C00F0908093F8BC8C054607018F
:1088000040463FF027FE4FEA5813012208F01F08A8
:10881000013B02FA08F2052B09D8DFE803F0ABB1FF
:1088200003B7BDA560498B6B23EA02038B637B1BF7
:1088300006EBC30305F1010B93F8500CFFF762FF41
:108840005FFA8BFB804618B1122380F807B0837162
:108850007B1B06EBC30393F8510CFFF753FF8246D3
:1088600018B1132380F807B083717B1B06EBC30399
:1088700093F8520CFFF746FF814618B1142380F895
:1088800007B083717F1B06EBC706504696F8542C41
:108890002E21FFF79DFA96F8552C48460E21FFF73A
:1088A00097FA96F8532C2E214046FFF791FA236849
:1088B0003E4A23F04003944223602FD03C4B9C421D
:1088C00036D103F5EC339A6B42F480429A639A6B8B
:1088D00022F480429A63636843F4805363602368A0
:1088E0005B0611D4236823F47F4323F0BF0343F4D2
:1088F000457343F003032360636823F4706323F03C
:10890000040343F4E0636360E36923F40063E36119
:10891000236843F040032360BDE8F88F224B1A6CB4
:1089200042F480521A641A6C22F480521A64D2E71C
:10893000204B9C420DD0204B9C42CCD103F554439C
:108940001A6C42F400421A641A6C22F400421A644F
:10895000C1E703F5EA339A6B42F400429A639A6BDB
:1089600022F400429A63B6E70F490B6B23EA020335
:108970000B635CE70C49CB6A23EA0203CB6256E740
:1089800009490B6C23EA02030B6450E70649CB6BE1
:1089900023EA0203CB634AE703498B6A23EA020313
:1089A0008B6244E7C02900200010024000300140E3
:1089B00000380040003C0040003C01402DE9F04FF1
:1089C000DFF890929E4E9F4F83B082464FF0010891
:1089D000DAF800506C684C4500F049819A4B9C4293
:1089E00000F0488103F580639C4200F04681974A7D
:1089F00094420CBF4FF0030C4FF0FF3C2368BAF8D1
:108A0000041028899AF86820009223F040038842D5
:108A100085F82480236014D0B1F5807F0B46A8BF71
:108A20004FF48073022BB8BF0223206893FAA3F39C
:108A3000B3FA83F320F03800013B40EAC30323601C
:108A400029819AF80CB0A97A59451ED08049CCEBFF
:108A50000C1201EBC202019292F8500CFFF752FE89
:108A6000019A92F8532CBBF1000F40F0D98010B15D
:108A70002E21FFF789F9226842F001022260226864
:108A800042F00202226085F80AB0236895F80CE0F3
:108A900043F0400323602B6A9A68002A00F0F280BA
:108AA00000201433844653F8101C944401EA060253
:108AB00039B16969002937D0B2F1805F34D0BA4248
:108AC00032D053F8142C143302EA060122B1B1F16A
:108AD000805F29D0B94227D053F80C2C0130002AEE
:108AE000E1D1BEF1000F1FD0009BEBB1012802D8ED
:108AF000BCF1070F10D9296ADAF8000044F0D0FD64
:108B0000DAF8083013B11A689B889362504603B0B4
:108B1000BDE8F04FFEF75CBA00EB800082002B6AE4
:108B200013441B7B002BE6D02B6A9B684FF0000B95
:108B3000002B00F09180BBF1000F02D09BF80C30AD
:108B40002BB1DAF8083013B11A689B8893622B6A4C
:108B500018682B6A59682B6AD3F808C06368BCF19F
:108B6000010F23F48053636014DD6246A3689B0702
:108B7000FCD5002851D030F8023BA381A368DB0765
:108B8000FCD5E36809B121F8023B023A012AEDDC89
:108B90000CF0010C636843F480536360BCF1000F78
:108BA00014D12B6A1B7B1BBB2B6A1B69002B2AD0A1
:108BB0002B6ADAF874001B699847012828D002282C
:108BC00021D100232B6203B0BDE8F08FA3689A0780
:108BD000FCD5002831D003782373A368DB07FCD5CC
:108BE000E3680029DDD00B702B6A1B7B002BDBD0E8
:108BF000DAF80830002BD7D01A689B8893612B6A6B
:108C00001B69002BD4D1D5F820B02B6A14332B620A
:108C10002B6A9B6803B36C688DE74FF6FF73ACE774
:108C200010B14E21FFF7B0F8226822F00102226055
:108C3000226822F00202226025E7FF23CCE700BF72
:108C40000080FFFF0080012000380040003C014010
:108C5000C0290020003001402B6A1B6883B12B6AB9
:108C6000D3E900A100222962C3E90022B0E64FF057
:108C7000000CC3E64FF0010CC0E64FF0020CBDE65D
:108C80002B62A0E7BEF1000F3FF44EAF009B002B1C
:108C90007FF445AF48E700BFF8B58569002D56D091
:108CA0002C68236A1B7B002B5DD1D4E904160F6866
:108CB0000B7A4249626830680B4413F801CC57F8CC
:108CC0000C3023F0010347F80C30377A3944022383
:108CD00011F801CC50F80C1021F0010140F80C10F3
:108CE000317D8B4043F00C034360536823F0020353
:108CF0005360536823F001035360236A1B693BB13F
:108D0000236A686F1B69984701284AD0022820D03F
:108D1000236ADA694AB9586900282BD09969216217
:108D2000C3E90522BDE8F84048E6216A94F824200A
:108D30000E7B1433F6B223621ABB002E2AD12846CA
:108D4000FEF746F92868016ACB69002B14DCF8BDF0
:108D50002362236ADA691433002AF9D1236ADA69B3
:108D6000002AE2D1D7E7AB68002B9ED01A689B8817
:108D700093619AE72062F8BDBDE8F840143144F0F1
:108D80008FBC216A286844F08BFC002384F82430CF
:108D9000002ED4D0AB68002BD1D01A689B88936288
:108DA000CDE7236A2868143B2362016ACB69002B54
:108DB000AEDD143144F074FCAAE700BFC0790508A9
:108DC00008B51D20FFF79EFC10B190F9063053B195
:108DD0001E20FFF797FC10B190F9063003B108BDD3
:108DE0005523C38008BD5523C380F1E7F8B50E4C69
:108DF00094F86C75A7B104F2AC74C7F109070925A2
:108E0000013D0FD0A6683079FFF77CFC94F8B810CC
:108E1000F27908B1FEF7B8FFAF4204F59A74EFD1CA
:108E20000120F8BDAB68FFDEC8180020F8B5EFF3ED
:108E30001185502383F31288D0F800311B6813F09A
:108E4000010303D0EDB285F31188F8BDD0F8A0215D
:108E5000D0F8A4110A4302F02102212A0446F1D0DD
:108E6000D0E9091291424FD090B24AD819462369ED
:108E70001B1A9BB2A162D4F8A0110026202984F805
:108E8000B061DFD1A1698918DCD0002BDAD094F869
:108E90009C21012AD6D0D4F89401A4F87631212758
:108EA0000122C4F8A861C4F87011C4F8A071A4F834
:108EB0007431D4F8207184F89C2178B3DFF870E025
:108EC00090F824C0C0F82CE0DFF868E0C0F830E08B
:108ED0009445DFF864E08663C0F834E007D080F89A
:108EE000242090F82520012A12D080F82460102137
:108EF00000222023C4F8A81184F89C21C4F8A031D2
:108F0000A0E7081A83B2B5E7012380F8B03199E7EA
:108F100007F128023CF060FA0028E8D10023402243
:108F20003A6284F89C31BB6843F08003BB6089E7F8
:108F3000190F04083D0F0408790F040870B5D0F824
:108F40002041E3699906054614D5606AEB6AC0B210
:108F5000002B73D0296B9847D5F82041236823F460
:108F600080732360A36823F00103A360A36943F027
:108F70000803A361E369DA0744BF01232362E369BD
:108F80009B0744BF02232362E3695E0744BF0423B7
:108F90002362E369180744BF08232362E369590683
:108FA00015D54023236295F8C161002E30D0D5F845
:108FB0000031D3B12846FFF739FF95F8B031002BC7
:108FC00048D095F8C161D5F82041002E4AD0D5F897
:108FD000003153B1E369DB0606D56B6B13B19847DB
:108FE000D5F820411023236270BDE3691A06F1D53C
:108FF000D5E90923934230D0A969CA5CD2B2A262F2
:109000002A690133B3FBF2F102FB1133AB62E1E7F2
:1090100095F8BE01FFF776FB2368012223F00803D1
:10902000236085F8C1210028C1D032462021FEF7F7
:10903000ABFED5F80031002BBCD1D6E7EB696A69ED
:10904000D054EB69EA680133B3FBF2F102FB113350
:10905000EB6181E7D5F82041B9E7236823F080036D
:109060002360B7E795F8BE01FFF74CFB23680122A8
:1090700023F00803236085F8C1210028A7D03246D9
:109080002021FEF781FEA2E7BFF34F8F0549064B73
:10909000CA6802F4E0621343CB60BFF34F8F00BF96
:1090A000FDE700BF00ED00E00400FA052DE9F843FC
:1090B000BFF35F8F464A00210B46C2F89410084662
:1090C000C2F898300133112BC2F89C10C2F8A010DE
:1090D000F6D10523C2F89430BFF34F8FBFF36F8FE3
:1090E000BFF35F8F3B4C3A4FC2F894000026012536
:1090F00020E0002A3AD0D4F80080637AA17AE07A9E
:109100001B0643EA017343EA4203217B627BC7F8F3
:10911000986043EA804343EA414343EA024301360D
:1091200043F00103032EC7F89C8004F11004C7F834
:10913000A0301CD06368227A002BDAD0D4F80080EB
:10914000002ADAD128F01F02A3EB0209B9F1200F9F
:1091500038BF4FF02009484646F07AFA431E05FA18
:1091600003F2914508BF1846C2B2C6E7FEE70523E1
:10917000C7F89430BFF34F8FBFF36F8FFB68164C67
:109180004FF6FF02134043F00523144A43F47A03D9
:10919000FB60D2F89430C4F82C3E3CF0E5FAD7F8E6
:1091A000FC100F4B0F4AB0FBF2F241F08071C7F890
:1091B000FC100021596019680B4841F00101196049
:1091C0008368C4F8302E43F480438360BDE8F8839D
:1091D00000ED00E0A8030020C0290020001002409C
:1091E000001000E040420F000070004008B572B669
:1091F000FFF74AFF03689B0AA3F58013542B57D847
:10920000F0B5374C23441B7E0B2B50D8354D40799D
:1092100005EB83148708D4F8346E334C03EB8300DA
:109220004FF0020E03EB40000EFA07FE38444FEAFF
:10923000831CF768002941D047EA0E0704EB800E33
:10924000CEF87415CEF88425F760EFF3118E502216
:1092500082F312882C2101FB0340D0F8702542B321
:10926000C0F89425111D214A214E03EB830003EB26
:109270004000800006441030024452F8040F08B148
:109280000860011DB242F8D100225FFA8EFE0A602A
:109290008EF311882C2202FB0344D4F89435BBB121
:1092A000AC44DCF8342ED36843F00103D360F0BD46
:1092B00070470E4A01FB03212431D5E727EA0E0748
:1092C000F76004EB8006C6F87415C6F88425BCE781
:1092D0006544D5F8342ED36823F00103D360F0BD84
:1092E000E8FC0408C0290020C8180020381E00200F
:1092F000581E002003689B0AA3F58013542B00D945
:1093000070470E4A13441B7E0B2BF9D810B40C4C3B
:10931000427904EB83109208D0F8340E0223934074
:10932000C26829B922EA03035DF8044BC3607047A1
:1093300013435DF8044BC360704700BFE8FC0408AA
:10934000C029002003689B0AA3F58013542B0FD873
:10935000084A13441B7E0B2B0AD80749427901EBBC
:10936000831192080223D1F8341E9340DB430B6132
:10937000704700BFE8FC0408C029002001490248EA
:10938000FDF7C4BD381E0020002C014010B5064C6E
:10939000064804F5AE61FDF7B9FD04F2FC6104482E
:1093A000BDE81040FDF7B2BDC8180020002C0140F8
:1093B0000044014002494FF08040FDF7A7BD00BFC7
:1093C000641E002001490248FDF7A0BD901E002048
:1093D0000004004001490248FDF798BDBC1E002072
:1093E0000008004001490248FDF790BDE81E00203A
:1093F000000C0040F8B5164D164E2A69EB681A406D
:109400004FF00040B2FA82F320FA03F3DB4302EAA2
:109410000301C2B1012A2B6101D00A46F2E7D6F856
:1094200074768FB1013F0023BFB2C6F87436D6F808
:10943000704634B123682046394698476468002C4A
:10944000F8D10022DCE7F8BDEF6ABFB2EFE700BF5A
:1094500000100040C818002001490248FDF756BD21
:109460006C1F00200034014001490248FDF74EBD49
:109470006C1F00200034014001490248FDF746BD41
:10948000981F00200040014001490248FDF73EBD01
:10949000F01F00200048014001490248FDF736BD99
:1094A0001C200020005001402DE9F0414FF40F72C4
:1094B0008CB05648564D002146F0EAF8554B1A6ECE
:1094C00042F400621A661A6E02F400620092009A78
:1094D0009A6D42F001029A659A6D02F001020192C2
:1094E000019A9A6D42F002029A659A6D02F00202A8
:1094F0000292029A9A6D42F004029A659A6D02F005
:1095000004020392039A9A6D42F008029A659A6DDA
:1095100002F008020492049A9A6D42F010029A65D1
:109520009A6D02F010020592059A9A6D42F020029F
:109530009A659A6D02F020020692069A1A6E42F41B
:1095400000521A661A6E02F400520792079A1A6EB7
:1095500042F480321A661A6E02F480320892089A37
:109560001A6E42F400321A661A6E02F40032099240
:10957000099A1A6E42F480221A661A6E02F4802248
:109580000A920A9A1A6E42F480121A661B6E03F44B
:1095900080130B930B9B4FF00008A5F5237605F67F
:1095A0002C2440F28B2755F82810002354F8332040
:1095B000914226D001330C2BF8D1002008F1070886
:1095C0003EF048FFB845EED14FF0000840F28B273F
:1095D00055F82810002354F8332091420CD0013361
:1095E0000C2BF8D1002008F107083EF033FFB845F6
:1095F000EED10CB0BDE8F08106EBC30393F8BC0CD0
:10960000F1E706EBC30393F8BC0CD7E7381E002044
:1096100074FF040800100240800AA0F5801054284E
:109620000DD8074B03441A7E0B2A08D8054B03EBD1
:109630008213D3F8342E136843F00103136070478C
:10964000E8FC0408C02900201F4A204B904210B4B7
:109650005B6827D002F50062904223D002F5406299
:1096600090421FD002F5806290421BD002F58062CA
:10967000904217D002F50062904213D01448154A68
:1096800081688468C1F302210A4414F4E06F92F8FF
:10969000702202F01F0223FA02F000D040005DF8B1
:1096A000044B70470A480B4A81688468C1F3C221A1
:1096B0000A4414F4605F92F8702202F01F0223FA49
:1096C00002F0ECD04000EAE7002C0140000000204E
:1096D00000100240E8FC04082DE9F04F93B000238D
:1096E0000093A74BA74CA84FA3F61856A44D4FF0D4
:1096F0000009A64BD5F800B093F88E204FEA9B23C3
:10970000A3F58013542B00F2CC8033441B7E0B2B2B
:1097100000F2C780012A17F903A000F00381022A92
:1097200002D1BAF1080F34D14FF00008414650463B
:109730000FF0B8F90FF042FA90F9003013B1542B42
:1097400040F0DB8108F104081FFA88F8B8F1100F27
:10975000ECD1009B0021002B00F0AD80894A0AE08B
:1097600033441B7E0B2B0DD8FB5653450DD0E432F2
:10977000944200F09D80906803689B0AA3F58013D3
:10978000542BEDD900235345F1D1437968799842A0
:10979000EDD109F10109B9F1080F05F11C05A8D1B6
:1097A000009B0133042B009304F1E4049ED1784A1A
:1097B00092F86C35013302F5667A03934FF0010B92
:1097C000039B5B456AD0714BDAF80C609AF8102065
:1097D00093F8A2300092002E60D06D4AD6F8009027
:1097E0005568B288019209F13840002D4FEA902067
:1097F00040F3A880634A002405E00134AC4202F142
:10980000E40200F09C8011688142F6D15D4B019D1D
:10981000E42202FB0434009B8AF81030019BCAF852
:109820000C60B3FA83F7C7F11F034FF00302CAF8C5
:109830000430CAF81840B27186F807B0A16C206CE9
:109840005E0001224FF0030C0CFA06FC02FA06F649
:109850003143A1644E490E7840EA0C0002FA03F34A
:109860002064D4F84CC0D4F8940099B2002E00F0D3
:109870004A8143EA0C03E364C9F81850FCF718FC6A
:1098800020460BF1010BFCF7E7FB40F20113BBF1A3
:10989000090FAAF81C300AF1200A91D113B0BDE8D3
:1098A000F08F013A012A7FF674AF4FF0000A3BE7D0
:1098B00000297FF46EAFA8683649002205E0013226
:1098C000102A01F10C0100F064834B689842F6D134
:1098D000697952B25846FEF7EDF82F4A4068516850
:1098E0000023884203F1010309D0102B02F1240266
:1098F0003FF44FAF5168884203F10103F5D1DBB269
:10990000264A013B03EBC30302EB830393F9843143
:10991000002B7FF43EAF1A4BC9EBC90903EB890357
:10992000A3603DE7BAF1010F3FF4FEAE09F1010972
:10993000B9F1080F05F11C057FF4DBAE30E7042C0C
:1099400000F03E82124AE42101FB052211690591D3
:10995000002900F0EA8290604FF05401013082F853
:10996000E810C4B20A4982F8E9406A1C4A60059AC4
:10997000116802915179976804910022054915E018
:10998000000A0508D0180020B0790508B83A002070
:10999000C8180020A8000020680100200000002056
:1099A0000132102A01F10C0100F0F382486887426D
:1099B000F6D104990298069352B2FEF77BF8994BC0
:1099C000DFF89082D0E90171E42202FB0532C2E99E
:1099D0000771414600224868069B874202F1010256
:1099E00009D0102A01F124013FF458AF486887429A
:1099F00002F10102F5D1D2B28B49013A02EBC20267
:109A000001EB820292F9841100297FF447AFE4212F
:109A1000079301FB05F3590001EBA301C1EB4121C1
:109A200001EB8141494282F885418048069301EB70
:109A300041044FF08C0C04EB041400EB84040CFB89
:109A400001F100F54C7000EB410176481844C0E983
:109A5000351C542182F884113322C0F8A020744AA6
:109A6000C0F89C40C0F80C900298D418FFF7ECFDA9
:109A7000079B062B00F0AB81072B6E496E4B6F4A9C
:109A800018BF1A466E4B18BF0B46B0FBF3F3B0FB82
:109A9000F2F26448DDF80890E42101FB0501013B86
:109AA0009BB2013AA1F8A420A1F86C30A365069BF3
:109AB00003F1500100F1080319440023A4F85030C9
:109AC000E3656365484640F005FFD9F80030049A25
:109AD00043F08003C9F800300C2A22D8DFE812F0E6
:109AE000E101210021002100BD0121002100210010
:109AF0009E012100210021007A01009B0121002B01
:109B00007FF42CAE45E6C7F12F0702FA07F343EACC
:109B10000C032D04E3643246C9F81850FCF7C8FA68
:109B2000AEE6404A0298E42303FB0523022259696A
:109B30000368079123F00103036060230A934FF445
:109B40008073109301230B930A234FF00009CDE992
:109B50000D320AAACDF83090CDF83C90CDF8449063
:109B600040F006FD0799B1F5807F0AD040F2D1811F
:109B7000B1F5804F05D000F2DF81B1F5806F40F084
:109B8000EA8108234FF00409029A02F1180151F802
:109B90000920134341F80930059B1879002840F04B
:109BA000A681029A136843F0010313600023D8F8DA
:109BB0000420974203F1010300F09481102B08F177
:109BC0002408F4D14FF0FF334FF00008164A03EB9E
:109BD000C30302EB83034746D3F86801194B98424D
:109BE00014BFA120A0203EF035FC174B0D499A6C04
:109BF0001648DDF808C042F004029A649B6C049A8F
:109C000003F004030C2A0993099B9BBF104B03EB41
:109C100042030022B3F8F82DE42303FB05131A8353
:109C2000002320E0C8180020000000205C3B00203A
:109C3000D0180020D0DD0600449508001055220001
:109C400040771B000000024000100240EC42002060
:109C5000E8FC0408680100208C4500F0798101339C
:109C6000042B00F0998150F833100029F4D1C04939
:109C7000B8460F46D1F854180131C7F8541807EB0D
:109C8000C301029FC1F83478DB0003444046998841
:109C90000A439A80B74923469022FDF7FDFFB64B51
:109CA000E42707FB05374FF00008FD692A6842F0FA
:109CB00002022A602A6842F00A022A60C4E91D886A
:109CC0003A6AC4F88C204FF44052C4F890208023A4
:109CD0001022E3672267D7F8A020C4F88820E9B2F1
:109CE000A64AD7F80C90069B0839A2FB01214FF435
:109CF0000072C4F8802009F11802A26603F168021C
:109D00009F4B4FF4006C1A440909D7F89C30E36666
:109D100025F0FF000131C4F884C00491029040F0A6
:109D20002FFED5F800E0C4F820E0D5F804E0C4F830
:109D300024E0069BD5F808E0C4F828E0D5F80CE04C
:109D4000C4F82CE0C4E92A8803F1A0028C4BC4F8C3
:109D5000B0801A443B6AC4F8C4308023C4F8B430DD
:109D60004FF40053C4F8C830D7F8D830C4F8C03026
:109D700009F110094FF48073C4F8A090C4F8B8300A
:109D8000D7F8D430C4F8A4304FF48063C4F8BC30A2
:109D90000499029840F0F4FD2B6823636B686363B9
:109DA000AB68A363EB68E3632B68D6F8009043F0DD
:109DB00002032B602B6843F00A032B60B5882AE569
:109DC0006B4A032382F8A33013B0BDE8F08F6D4ACD
:109DD0006D4B5AE6029868490368E42202FB0512BB
:109DE00023F001034FF480515161036000230C9371
:109DF0000F93119360230A934FF480731093012300
:109E00000B934FF0020C0A230AAACDE90D3C4FF048
:109E1000040940F0ADFB4FF40063B5E602985649E3
:109E20000368E42202FB051223F001034FF4807162
:109E30005161036000230C930F9311934FF0600E58
:109E40000123CDE90AE34FF002090A230AAACDE96A
:109E50000D39109140F08CFB93E602984649036857
:109E6000E42202FB051223F001031021516103607B
:109E700060230A934FF48073109301230B93022203
:109E80000A23CDE90D324FF000090AAACDF830902F
:109E9000CDF83C90CDF8449040F06AFB4FF400635D
:109EA00072E6029834490368E42202FB051223F0AB
:109EB000010301215161036000230C930F9311935F
:109EC00060230A934FF4807310934FF002090A2322
:109ED0000AAACDE90D390B9140F04AFB08234FF057
:109EE000000951E65FFA83F808F1FF336EE6FEF7EA
:109EF00009FC814638B1059B0221DA79FDF744FF60
:109F00005423A9F80630029A536C43F40043536477
:109F100047E610293AD018D8012926D00429DDD0E7
:109F20004FF400634FF038092EE6114A022382F8FD
:109F3000A33013B0BDE8F08FB1F5803F14BF4FF4EC
:109F4000006308234FF038091EE64029C6D0E7E732
:109F5000B846DB0099E6B1F5805F4FF4006314BFAB
:109F60004FF038094FF004090EE608230CE600BF55
:109F7000B83A0020F9600008C8180020CDCCCCCC3D
:109F8000D0180020882A1100A0BB0D004FF40063F8
:109F9000FAE500235B68FFDE00239B88FFDE00BF3D
:109FA000F8B5830AA3F58013542B1BD80E4C234419
:109FB0001E7E0B2E16D80D4C013904EB861789B284
:109FC0001546C7F8401EFFF73FFBB0FBF5F2013A1C
:109FD000D7F8340EC7F8382E07F63861BDE8F840D8
:109FE0003BF0F8BBF8BD00BFE8FC0408C029002026
:109FF0002DE9F843830AA3F58013542B50D8154656
:10A00000444A13441F7E0B2F4AD8DFF8149109EB02
:10A0100087160446D6F8343E83424FEA87183FD06D
:10A02000013989B2C6F8401EC6F8340EFFF70CFBA2
:10A0300009F6346108F1080300220B44B0FBF5F087
:10A040000138C6F83C2EC6F8380EC3E9022296F84D
:10A05000713E03F0FF022BB309EB080501EB8711FA
:10A0600004312046022685F8716E3BF0B3FB2A4A84
:10A070000123944285F8713E38D0B4F1804F14D05A
:10A08000A2F59432944210D002F5806294420CD032
:10A0900002F58062944208D002F59432944225D0B1
:10A0A000BDE8F88386F8702ED6E795F8702E012A61
:10A0B000F6D085F8716EA168184A0A40A26085F84A
:10A0C000713E85F8716E6368A26823F00073C14425
:10A0D00023F07003636022F0800201210023A2605C
:10A0E00089F8711E89F8703EBDE8F88395F8702EE6
:10A0F000012AD5D085F8716EA168084A0A40A2608D
:10A1000085F8713E85F8716E6368A26823F4700368
:10A11000DBE700BFE8FC0408002C01408800CEFF0C
:10A12000C029002070B50468A30AA3F58013542B3E
:10A1300004D82D4E33441D7E0B2D00D970BD204612
:10A14000FFF756FF294BA80103EB85150222D5F82E
:10A15000341E85F8712E8D68254A2A40062A06D0BD
:10A16000B2F5803F03D00A6842F001020A6003445E
:10A170000122204983F8712E002351F833209442A4
:10A180000AD001330C2BF8D1012100203EF006F853
:10A19000194B01221A6070BD06EBC306012196F926
:10A1A000BD4C96F8BD5C20463DF0F8FF002CC5DBA9
:10A1B000114C6B0905F01F02012101FA02F21B2D5F
:10A1C00044F8232006D119203DF0E8FF4FF000733A
:10A1D000236070BD2E2DB1D12C203DF0DFFF4FF458
:10A1E0008053636070BD00BFE8FC0408C0290020F4
:10A1F00007000100A009050800E100E037B590F86C
:10A200006738032B04462FD10023204D8DF80730EB
:10A210009DF8073094F868289A4201D803B030BD01
:10A220009DF8073005EBC30393F85C388BB181F0E0
:10A23000010383B19DF8073005EBC303D3F8580839
:10A24000FDF7E4FB9DF807300133DBB28DF80730F2
:10A25000DEE70B46EDE79DF8073005EBC303D3F8C7
:10A260005808FDF7D9FBEDE7D0E910039B7903F01F
:10A270000103994204D003B0BDE83040FDF7C6BBEE
:10A2800003B0BDE83040FDF7C7BB00BFB83A0020BF
:10A2900038B5044600790D4650B1FEF733FA08B1DF
:10A2A0000323C380E2792946BDE83840FDF790BD1D
:10A2B00038BD10B522210446FFF7EAFF2046FFF71C
:10A2C00041F8BDE810400121FFF714B810B5012195
:10A2D0000446FFF7DDFF20460021BDE81040FFF7F0
:10A2E00009B838B510F8133CA0F66C041BBB94F801
:10A2F00058388BBBD4E909239A421CD05A1CA16957
:10A30000A262CB5C21695B0043F40073A4F85C3863
:10A310000A2384F85A38012384F8583894F86738A7
:10A320008A4228BF0022012BA26201D0042B02D155
:10A33000606CFFF7CBFF94F85438002B6DD194F884
:10A3400055380133DBB2092B84F8553825D1204626
:10A35000BDE83840FBF7BFBF94F95A586DB1B4F867
:10A360005C184B08A4F85C3801F001012046013D5F
:10A37000FFF744FF84F85A58DDE7D4E909239A42ED
:10A3800084F85858D7D194F86738012B01D0042BA2
:10A39000D1D1606CFFF78DFFCDE70A2B3DD194F84A
:10A3A00057382BB9B4F85E3843F00103A4F85E388F
:10A3B0002379D9070AD5B4F85E08820501D4C3070A
:10A3C00018D4B4F864380133A4F86438012284F84E
:10A3D000542894F857280023012A84F855381CD1B2
:10A3E000617984F85738606C01F00101BDE83840AC
:10A3F00040F0B6BCE36AC0F3470013B1216B984745
:10A40000E4E7E3696269D054E369E2680133B3FBCE
:10A41000F2F102FB1133E361D8E738BD904BD3F87A
:10A420000C25012A2DE9F04100F081828D4A8E4CE5
:10A43000D2F888308D4943F470038C42C2F88830DA
:10A4400004D08B4A2046121B45F000FA854B8949FF
:10A450009C600A68884D42F480720A60D968874A15
:10A460004FF6FF0001400A43DA603DF037FF7C4BB6
:10A47000D3F80805FBF78AFF814A136803F4C06329
:10A48000B3F5806FD2F8803023F48073C2F8803047
:10A4900060D0734A7B4BD2F80415D3F8A474D3F878
:10A4A000A064D3F8988451B177498B68C96803F0E8
:10A4B0000C030C2B6BD0082B6DD1734B1B68734CAA
:10A4C00071498B68C96803F00C030C2B74D0042B02
:10A4D00076D16D490B684B6823F0FE4343F080430F
:10A4E0004B603DF0FBFE002840F0B9806649D1F892
:10A4F000943043F00103C1F89430D4F8980804E094
:10A50000D4F898381B1A022B55D8D1F894309B07F1
:10A51000F6D5D1F8983043F00103C1F89830D4F85B
:10A520009808594904E0D4F898381B1A022B42D8ED
:10A53000D1F898309A07F6D58B6803F00C030C2BF2
:10A5400000F0B8810B6823F080730B60D4F8980892
:10A550004D4951E013684E4923F4C06343F400733E
:10A5600013606B68322000FB03F3A1FB03135169F6
:10A570009B0C480503F1010306D500E023B15169A6
:10A58000490503F1FF33F9D43D4B5B6981E701F0E5
:10A590000301032991D03C493C4C0B6843F48033C0
:10A5A0000B60D4F898080B689B0389D4D4F89838CA
:10A5B0001B1A642BF7D9FEE701F00301022988D0AA
:10A5C00031490B6843F480730B60D4F8980804E0B9
:10A5D000D4F898381B1A022BEDD80B685A05F7D51A
:10A5E0004B6823F0FE4343F080434B607EE7D4F892
:10A5F00098381B1A022BDED80B689B01F7D4C86869
:10A60000244A731E024048EA0313134343EA072314
:10A6100043F08053CB600B681B4A43F080730B60A0
:10A62000CB6843F08073CB60D4F8981804E0D4F87A
:10A6300098385B1A022BBED813689801F7D50D4BDA
:10A640001A68120728D41A6822F00F0242F0080292
:10A650001A601B6803F00F03082B1DD0FEE7AAE762
:10A660000020004000ED00E000F0012000000008A4
:10A67000D8F1012000200240000000200003FA056C
:10A6800000700040C818002000100240B83A0020B6
:10A6900083DE1B430C809F01B5490B689B0140F191
:10A6A000F280CB68C86803F00303032B00F03C8101
:10A6B000CE68CA68AF4FB04BC2F34162C0F303101B
:10A6C000C6F30626013201305200B3FBF0F306FB5D
:10A6D00003F3B3FBF2F3BB4206D98B688B6823F01C
:10A6E000F00343F080038B60A14B9A6842F00302B1
:10A6F0009A60D4F8981841F2883004E0D4F8982889
:10A70000521A8242AAD89A6802F00C020C2AF5D199
:10A7100099689A4A41F4E0619960996821F47C5102
:10A7200041F4E0619960996821F0F0019960136843
:10A7300003F00F03082B00F2A7808D4C904EA36806
:10A7400023F4E063A360A36823F46053A3603BF0A9
:10A750000BF8A368C3F30313334493F8143E03F0D8
:10A760001F0320FA03F76F603DF0B8FD002840F0AA
:10A77000DA80D4F88830834A834923F00303C4F88D
:10A780008830D4F8883023F00C03C4F88830D4F82B
:10A79000883023F03003C4F88830D4F8883023F0B0
:10A7A000C003C4F88830D4F8883023F44073C4F868
:10A7B0008830D4F8883023F44063C4F88830D4F863
:10A7C000883023F44053C4F88830D4F8883023F418
:10A7D0004043C4F88830D4F8883023F44033C4F8B8
:10A7E0008830D4F89C3023F00303C4F89C30D4F8AC
:10A7F000883023F0407343F00073C4F88830D4F8F5
:10A80000883023F04063C4F88830D4F8883023F0CF
:10A81000405343F00053C4F88830D4F8883023F014
:10A82000404343F00043C4F88830A36B43F4807383
:10A83000A363A36B23F48073A363544B5A601A6819
:10A8400022F4FE4242F400521A601A6842F060029A
:10A850001A604A4A1160D3F80435A26802F00C026B
:10A86000082A05D00C2A43D0434B042A18BF3B4684
:10A870003F4A9268C2F30312164496F8142ED3404E
:10A880006B60BDE8F081E9E6136823F00F0343F045
:10A8900008031360D4F8981841F28830136803F065
:10A8A0000F03082B3FF449AFD4F898385B1A834262
:10A8B000F4D9D3E6CB6803F0030188457FF47BAE7F
:10A8C000013E03F0F002B2EB061F7FF474AE03F416
:10A8D000FE42B2EB072F7FF46EAE03F07842B2F186
:10A8E000805F7FF468AE13F0CC6F3FF4A8AE62E6F1
:10A8F000E168E26801F003010229C2F3031202F1E8
:10A90000010208BF1C4BB3FBF2F3194AD168D268AD
:10A91000C2F34162C1F30621013201FB03F352008D
:10A92000B3FBF2F3A4E799E6CB68CB68DCE6104A08
:10A93000174C0021C3F80C15D4F89818136843F489
:10A940008073136004E0D4F898385B1A022B4FD858
:10A9500013685D05F7D55368054D43F08043536098
:10A960000121D4F89808916041F2883217E000BFC5
:10A970000010024000B4C4040024F400002002408F
:10A98000E8FC04087FBB22200407040000200040EC
:10A99000B83A0020D4F898381B1A934228D8AB68EC
:10A9A00003F00C03042BF5D11C4B1D4A5A603DF0FB
:10A9B00095FCE8B94FF480732B602B60D4F898189D
:10A9C000184B04E0D4F89828521A022A10D81A68B2
:10A9D00012F00072F6D14FF480504FF0FF31D86082
:10A9E0009A611962D3F8942042F40002C3F89420CB
:10A9F0004FF0E02300221A615A619A6172B60A4947
:10AA00000A4A0B68106823F0070343F001030B6048
:10AA100080F3088853689847FEE700BF00000020D5
:10AA20000024F40000100240000001400000FF1F5D
:10AA300010B504460220FDF7C7FB042C034628BFCF
:10AA400000240120FDF7C0FB9C420AD128B10B4A2B
:10AA5000936803F00303032B00D010BDD368DB071A
:10AA6000FBD42046FBF792FC0028F6D021460220BA
:10AA7000FDF7B2FB72B6FEF707FB00BF0010024005
:10AA800010B4EFF31182102383F312880D4C0E4B98
:10AA9000D4F8A4104FF0E0200131C4F8A41081696B
:10AAA000C3F89C180021C3F8A0180169D2B282F340
:10AAB0001188D3F898285DF8044B0132C3F8982820
:10AAC000704700BFC0290020B83A002030B4EFF32F
:10AAD0001183102282F312884FF0E0220F4894690C
:10AAE0001169C90344BF0121C0F8A0180C4948BF2F
:10AAF0009469D1F8A450D0F8A028DBB283F3118870
:10AB0000D1F8301E4FF47A702A4400FB01F31B1B6E
:10AB100030BCB3FBF1F300FB02307047B83A0020C1
:10AB2000C0290020134B5B68C3F308030BBBEFF392
:10AB30001183F3B910B4104B104C4FF0E02CD3F844
:10AB4000A420DCF81800D3F8A4108A42F7D1D4F876
:10AB50009C188842F3D8D3F8304E4FF47A7101FB39
:10AB600004F31B1AB3FBF4F35DF8044B01FB023052
:10AB70007047ABE700ED00E0C0290020B83A0020A4
:10AB80002DE9F04FBD4F87B03B7805931BB90120ED
:10AB900007B0BDE8F08F97F86C350393B84BDFF83A
:10ABA000F0B2D3F8A430049307F566770BF5387A42
:10ABB0004FF00009ABF6A406039B994500F0F68020
:10ABC000BB69D7F80480D3E93354FFF7ABFF01909A
:10ABD00096F88D0C96F88CCC04F10041393901229D
:10ABE000542805EB410102FA08F205EB4C0301D1B0
:10ABF000A6F896CC994240F22D81B3F800E01EEA07
:10AC0000020F00F01F81B3F802E01EEA020F00F00D
:10AC10003081B3F804E01EEA020F00F02C81B3F893
:10AC200006E01EEA020F03F10803E3D1A3EB050ED1
:10AC300099424FEA6E0E40F20D81A4EB0E04452CB2
:10AC400028BF452403EB4404A34280F00A81002579
:10AC50009C46A8462946CDF80890B3F8009009EA2A
:10AC60000209894518BF02331AD1B3F8029009EAE4
:10AC70000209494518BF043312D1B3F8049009EA18
:10AC80000209494518BF06330AD1B3F8069009EA0C
:10AC90000209494503F1080302D19C42DDD802E0D4
:10ACA0009C4200F2A480B8F1110FDDF8089040F248
:10ACB000D880D8F1150200F1D4807249019CD1F8F6
:10ACC000D8339E45D6F8A03C38BFC1F8D8E3E11A86
:10ACD000002918DB03F5F42303F590739C4284BF2D
:10ACE00023460533C6F8A03C664B6649D3F8D833F3
:10ACF000052B86BF053BDBB2002386F88C3C4FF06A
:10AD0000FF33C1F8D8333AB105FA02F2C8F114089A
:10AD1000012505FA08F515435B4AC5F3C43302EB78
:10AD20008303D3F8241E05F01F0302EB8303D3F83B
:10AD3000243E43EA0133C5F3441102EB8101C5F31C
:10AD4000842502EB8502D1F8241ED2F8242E43EA92
:10AD5000011343EA022383EA132282EA1212D6F88D
:10AD60008C1B02F00F020F2A01F101015AD1B3F539
:10AD7000803F57D254284FEA13131ED0B3F5606FAB
:10AD8000C6F88C1B23D0AAF80C300599049A5846B3
:10AD90000CF04CF909F10109B9F1080F0BF15C0B4A
:10ADA00007F120070AF1140A7FF406AF01230120FE
:10ADB00086F8883C07B0BDE8F08FB6F8902CC6F84E
:10ADC0008C1B0132B3F5606FA6F8902CDBD12C49B7
:10ADD00091F84D2102EB420201EBC2024A4492F883
:10ADE0005D210D2ACFD180238AF81E30CDE7A3EB59
:10ADF0000C0C26494FEA6C0C0CF1010C81FB0C91F8
:10AE0000A1EBEC710129B8BF01218D404FF0010C7D
:10AE1000884401390CFA01F10D4333F8021C9C46B9
:10AE200011401AE7542804D1B6F8903C0133A6F833
:10AE3000903CD6F8883BC6F88C1B0133C6F8883B9B
:10AE40000021A3E70233A3EB050E99424FEA6E0EF1
:10AE50003FF6F3AEBCF1000F03D00CF1FF3C86F8D7
:10AE60008CCC542896D1B6F8923C0133A6F8923C8B
:10AE700090E70433DAE60633D8E600BFC8180020AE
:10AE8000C029002000000020E8FC04085655555554
:10AE90005C43002070B51F4B93F84C2193F84D3163
:10AEA0009A4231D11C484568002D10DD10F8086B1E
:10AEB000002406B3037F012B20D0426913680134BC
:10AEC00043F00103A54200F1E4001360F1D1FFF764
:10AED00029FE124BD3F85448002C0BDD03F6340343
:10AEE00003EBC40419689A88C86808330243A34274
:10AEF000CA60F7D170BDFBF7AFF8DEE7002380F83A
:10AF0000D430FBF7A9F8D8E742F02AF90028C9D1D4
:10AF100070BD00BFC0290020C8180020B83A00202A
:10AF20002DE9F04704460068217D026802238B402A
:10AF30001A4209D0A669A04D4FF49A7202FB06523C
:10AF400092F8981811B14360BDE8F0879B4F9C4977
:10AF5000D7F804C091F8B4119A4FC7F8A4CC0029CF
:10AF600000F0A480D2F8B427D2F810C01168DCF841
:10AF7000002022F00102CCF80020CA6822F480727E
:10AF8000CA602A78002ADED04FF49A7306FB03F3D6
:10AF900005EB030A8C49DAF8D4088C4A03EB010963
:10AFA000C1B20839A2FB0121DAF8B437090901312D
:10AFB00020F0FF00D3F800803FF024FD01238AF841
:10AFC0009838D7F8AC3C002B00F08280D8F80020ED
:10AFD0004FF49A7303FB065342F08002C8F8002036
:10AFE000D3F894284FF0FF31B2F5807FC8F82C10C9
:10AFF00073D000F29680012A00F0BA80102A22D184
:10B00000D8F82020D3F8D01822F01002C8F8202059
:10B01000D3F8C82842EA0100D8F81820D3F8CC1891
:10B0200022F47F42014342EA1122C8F81820D3F8E3
:10B03000C428D8F8203023F0A00343EA021343F0D9
:10B040001003C8F820304FF49A7303FB0655002311
:10B05000D5F8D408C5F87038C1B2A3F13333083934
:10B06000A3FB013109094A46013120F0FF003FF0FE
:10B0700087FCD5F8D428206853686FF30F0343F09A
:10B0800016035360136843F001031360D5F8B42727
:10B09000B5F8B8371268D1680B43D360474B227DAF
:10B0A0005968C7F8A81C022393404CE7D2F8D4C8CB
:10B0B000DCF8001021F00101CCF80010D2F8B41730
:10B0C000B2F8B8C70968CA6822EA0C02CA6058E731
:10B0D000FFF728FDC7F8AC0C78E7D8F82020D3F8A4
:10B0E000D01822F48072C8F82020D3F8C82842EA89
:10B0F0000100D8F81C20D3F8CC1822F0FF0201433D
:10B1000042EA1142C8F81C20D3F8C428D8F82030ED
:10B1100023F4206343EA022343F48073C8F8203009
:10B1200091E7B2F5805F8ED1D8F82020D3F8D018FF
:10B1300022F48052C8F82020D3F8C82842EA01003F
:10B14000D8F81C20D3F8CC1822F47F42014342EAFD
:10B150001122C8F81C20D3F8C428D8F8203023F4D2
:10B16000204343EA023343F48053C8F820306AE7AF
:10B17000D8F82020D3F8D01822F00102C8F82020F7
:10B18000D3F8C82842EA0100D8F81820D3F8CC1820
:10B1900022F0FF02014342EA1142C8F81820D3F816
:10B1A000C428D8F8203023F00A03134343F00103E6
:10B1B000C8F8203047E700BFC8180020001000E0A2
:10B1C000C0290020B83A002030210020CDCCCCCCC2
:10B1D0002DE9F04F864C237887B01BB9012007B0CA
:10B1E000BDE8F08F834BD3F8A4300493FFF79AFCAB
:10B1F00094F86C350193002B00F0F2807E4AD2F86F
:10B20000AC3C04F2AC74A0EB030902F6A40B02F60A
:10B21000843A2546002601270594B9F1000F04DB86
:10B22000D5F8F0304B4500F3C180714A4FF49A7362
:10B2300003FB062393F8983803F0FF08002B7DD01A
:10B24000AB68A9891A68D5F828315C68D368A4B2BC
:10B25000C4F1160423EA0103072CD3606ED9664AB1
:10B26000D2F88C3B0133C2F88C3BD5F83031002248
:10B27000CDE9028618689E469446012116E0BCF18D
:10B28000140F1FDC16F1080848BF06F117084FEA33
:10B2900028160CEB281C06F1FF38013102FA06F6DD
:10B2A00007FA08F88C4248EA06020BD306465EF815
:10B2B000040F8C42A0EB0606E1D8CCF115064FF046
:10B2C000150CE8E7BCF1150FDDE9028664D14B4CA3
:10B2D000C2F38421C2F3441004EB810104EB80002B
:10B2E000D1F8A41ED0F8A40E090241EA001102F020
:10B2F0001F0004EB8000C2F3C43204EB8202D0F8DA
:10B30000A40ED2F8A42E014341EA023181EA1122AF
:10B3100082EA121202F00F020F2A3DD1C1F30F117F
:10B320004FF6FF72914237D0B1F5606F42D0AAF864
:10B330000C10049A414658460BF078FE2846FCF75C
:10B34000A9FF019B0136B34205F59A750BF15C0B21
:10B350000AF1140A7FF461AF2749059C01220023FA
:10B3600081F8882C019AC1F8AC3C4FF49A7303FB26
:10B370000243A26894F8B4101268D4F8E80011F0FF
:10B38000020F116A04F59A7414BF41EA8001014367
:10B39000A3421162EDD121E71749D1F8882B013280
:10B3A000C1F8882BB6B14FF00008C2E7002007B003
:10B3B000BDE8F08F0F4A92F84D3103EB430302EBE7
:10B3C000C303334493F85D310D2BB0D180238AF849
:10B3D0001E30AEE719465822094844F037FAE2E732
:10B3E000054B012283F8882C019AC3F8AC2CF5E6B2
:10B3F000C8180020C0290020B83A0020E8FC040842
:10B40000E84600202DE9F84FFFF78CFB2E4FDFF8C0
:10B41000C4B07D682D4C2E4E82464FF00008002DA2
:10B4200046DD00231A46E42000FB0371013391F846
:10B43000DD109D4242EA0102F6D142EA08095FFAB4
:10B4400089F99046DBF80430C3F308036BBBEFF3D4
:10B45000118353BB4FF0E020D4F8A4308169D4F8B5
:10B46000A4209342F8D1D6F89C289142F4D8D4F87D
:10B4700030CE4FF47A7202FB0CF0401AB0FBFCF0B5
:10B4800002FB0300A0EB0A03B3F5FA6F02DCB8F18C
:10B49000000FC4D1B9F1000F04D00D4B93F88D2CDF
:10B4A000542A09D04846BDE8F88FFFF70FFBE9E7BB
:10B4B000C1464FF00008C5E7B3F8942C0132A3F859
:10B4C000942C4846BDE8F88FC8180020C0290020F9
:10B4D000B83A002000ED00E02DE9F0410746FFF703
:10B4E00021FBDFF86480164C164D0646D8F8043070
:10B4F000C3F3080303BBEFF31183EBB94FF0E02C68
:10B50000D4F8A430DCF81810D4F8A4209342F7D172
:10B51000D5F89C289142F3D8D4F830CE4FF47A7203
:10B5200002FB0CF0401AB0FBFCF002FB0300831B93
:10B53000BB42DBD3BDE8F081FFF7C8FAF7E700BFF5
:10B54000C0290020B83A002000ED00E02DE9F843C2
:10B55000DFF8B080294C2A4F461E4FF0E025D8F87E
:10B560000430C3F30803002B44D1EFF31183002B05
:10B5700040D1D4F8A430A969D4F8A4209342F8D1DA
:10B58000D7F89C289142F4D8D4F8300E4FF47A7250
:10B5900002FB00F9A9EB0109B9FBF0F902FB0399E1
:10B5A000D8F80430C3F308030BBBEFF31183F3B9EE
:10B5B000D4F8A430A969D4F8A4209342F8D1D7F8DC
:10B5C0009C289142F4D8D4F830CE4FF47A7202FB22
:10B5D0000CF0401AB0FBFCF002FB0300A0EB0903E7
:10B5E000B3F57A7FDCD3013EB9D2BDE8F883FFF72B
:10B5F0006DFAF3E7FFF76AFA8146D1E7C029002028
:10B60000B83A002000ED00E038B5094C04F540756B
:10B6100002E00834AC420AD094F90620002AF8D19E
:10B62000204620210834FCF7AFFBAC42F4D138BDF2
:10B630000C3300202DE9F04F874C83B0D4F8B0B024
:10B6400094F8B83000910646BBF1000F0BD083F0A0
:10B650000202BBF80410C2F34002120101FA02F226
:10B66000DBF800108A61D4F8AC703FB1BA8803F0FF
:10B6700001031B0102FA03F33A689361013E774D1F
:10B68000DFF8DCA1F6B2BBF1000F08D0DBF8002038
:10B69000BBF8043051690B4218BF1B04936137B1EA
:10B6A0003A68BB8851690B4218BF1B0493610120A3
:10B6B0000DF04AF9DDF80080019646466B68C3F349
:10B6C0000803002B40F0BF80EFF31183002B40F004
:10B6D000BA804FF0E02CD4F8A430DCF81800D4F88D
:10B6E000A4209342F7D1DAF89C289042F3D8D4F8FA
:10B6F000302E4FF47A7101FB02F8A8EB0008B8FB7A
:10B70000F2F801FB03884FF0E0296B68C3F30803EC
:10B71000002B40F09580EFF31183002B40F09080D8
:10B72000D4F8A430D9F81810D4F8A4209342F7D153
:10B73000DAF89C289142F3D8D4F830CE4FF47A72DC
:10B7400002FB0CF0401AB0FBFCF002FB0300A0EB84
:10B750000803B3F57A7FD8D3013EAFD1019EBBF188
:10B76000000F08D0DBF80020BBF8043051690B4211
:10B7700018BF1B04936137B13A68BB8851690B420B
:10B7800018BF1B04936100200DF0DEF8DDF8008087
:10B79000019646466B68C3F30803002B57D1EFF3BD
:10B7A0001183002B53D14FF0E02CD4F8A430DCF8F7
:10B7B0001800D4F8A4209342F7D1DAF89C289042DC
:10B7C000F3D8D4F8302E4FF47A7101FB02F8A8EBCD
:10B7D0000008B8FBF2F801FB03884FF0E0296B6822
:10B7E000C3F308034BBBEFF3118333BBD4F8A4308E
:10B7F000D9F81810D4F8A4209342F7D1DAF89C288D
:10B800009142F3D8D4F830CE4FF47A7202FB0CF0A8
:10B81000401AB0FBFCF002FB0300A0EB0803B3F5F9
:10B820007A7FDCD3013EB5D1019E013EF6B2FF2EF8
:10B830007FF429AF03B0BDE8F08FFFF747F9ECE7DD
:10B84000FFF744F983E7FFF741F980465BE7FFF72D
:10B850003DF98046C1E700BFC029002000ED00E0AF
:10B86000B83A00202DE9F84F01305D4F5D4C5E4D38
:10B870004E1E5FFA80FB32210520FFF7DBFE4FF4FE
:10B88000FA784FF0E0297B68C3F30803002B40F0FF
:10B890009F80EFF31183002B40F09A80D4F8A430FE
:10B8A000D9F81810D4F8A4209342F7D1D5F89C28E1
:10B8B0009142F3D8D4F8300E4FF47A7202FB00FABA
:10B8C000AAEB010ABAFBF0FA02FB03AA7B68C3F3F6
:10B8D0000803002B79D1EFF31183002B75D1D4F835
:10B8E000A430D9F81810D4F8A4209342F7D1D5F891
:10B8F0009C289142F3D8D4F830CE4FF47A7202FBF0
:10B900000CF0401AB0FBFCF002FB0300A0EB0A03B2
:10B91000B3F57A7FDAD3B8F10108B4D1FA215846E9
:10B92000FFF788FE4FF47A784FF0E0297B68C3F385
:10B930000803002B50D1EFF31183002B4CD1D4F826
:10B94000A430D9F81810D4F8A4209342F7D1D5F830
:10B950009C289142F3D8D4F8300E4FF47A7202FB4F
:10B9600000FAAAEB010ABAFBF0FA02FB03AA7B6811
:10B97000C3F3080333BBEFF311831BBBD4F8A4302C
:10B98000D9F81810D4F8A4209342F7D1D5F89C2800
:10B990009142F3D8D4F830CE4FF47A7202FB0CF017
:10B9A000401AB0FBFCF002FB0300A0EB0A03B3F566
:10B9B0007A7FDCD3B8F10108B8D1013EBFF45BAFA8
:10B9C000BDE8F88FFFF782F8EFE7FFF77FF89DE714
:10B9D000FFF77CF8824679E7FFF778F88246C6E7FA
:10B9E00000ED00E0C0290020B83A0020094B5A6859
:10B9F000B0EB520F01464FEA520309D20722022050
:10BA00005B084000994280B203D2013AF8D17047F6
:10BA100002207047000000202DE9F04F774E83B0E0
:10BA200006F1A008012707E00137052F06F12806D7
:10BA300008F1050800F083803378022BF4D198F9DF
:10BA400003A05FFA87F9BAF1FF3F18BF5FFA8AFADD
:10BA500009F1FF3512BFD3464FF00F0B4FF0000A2C
:10BA6000EDB24FFA8AF229460020FBF7DBFF58B10E
:10BA70004468634A002351688C4202F1240203F1B6
:10BA8000010309D0102BF6D10AF1010A5FFA8AFAF4
:10BA9000DA45E6D9002420E0DCB25A49631E03EB04
:10BAA000C30201EB8201920091F984C1BCF1000F45
:10BAB000EAD103F0070C524B81F885911A440CF13E
:10BAC000010381F87031142381F884318368326175
:10BAD0002046C1F87431FCF7B7F898F904B0BBF10F
:10BAE000FF3F19BF5FFA8BFBDA464FF00F0A4FF0AA
:10BAF000000B4FFA8BF229460120FBF793FF60B150
:10BB0000D0F804C03E4A002351688C4502F124025B
:10BB100003F1010316D0102BF6D10BF1010B5FFAE4
:10BB20008BFBD345E5D9013700220023052FC6E959
:10BB3000042308F1050806F128067FF47DAF03B061
:10BB4000BDE8F08FDAB2511E2E4B01EBC10E03EBB4
:10BB50008E0C4FEA8E0E9CF98431002BDDD101F062
:10BB6000070101930131264B8CF87011132103EB6F
:10BB70000E058CF885918CF88411816875611046EA
:10BB80000092CCF87411FCF75FF8DDE90023002C7B
:10BB9000C9D02846CDE90023FAF744FA3069FAF70C
:10BBA00041FA7468B169009AD0F80CC0019BED6845
:10BBB000C1F824C010460C34F2694B604FF0100CF1
:10BBC000C1E90333C1E90533C1E907338B620C6076
:10BBD000C1F808C04FF48051C2E90043C2E9023302
:10BBE000C2E90433C2E90633136291625562064921
:10BBF0001A46FCF751F80123337315E76847002014
:10BC00006801002000000020998C000870B40E4AE2
:10BC10000E4E0F4D4FF090444FF0010C36F8020BD2
:10BC2000002340FA03F1C90704D50CFA03F11460AC
:10BC3000918008320133102BF3D104F58064AC42BB
:10BC4000ECD170BC704700BF0C33002060FF0408CB
:10BC5000001800482DE9F04706460868BDF8207036
:10BC60009DF82480850AA5F58015542D0C4600F218
:10BC7000CC801946994B2B441D7E0B2D00F2C580BC
:10BC8000FEF7B6F96279B8F1000F40F0C080A179F3
:10BC90008C46934BA80103EB851595F870EEBEF129
:10BCA000010F71D04FF001084FEA410E85F8708EF8
:10BCB000C9004FF002080EF0020E01F0080185F8ED
:10BCC000718E142A59D8DFE812F0970158005800F5
:10BCD00058001500580058005800E201580058005C
:10BCE00058005301580058005800130158005800DC
:10BCF0005800C9001D18DFF8F491D5F8345ED5F866
:10BD0000208028F01008C5F82080D5F82080D5F8CC
:10BD100004A028F0200848EA0E1ED5F8188028F064
:10BD2000807828F4E6484D4548F4C04800F0FD818D
:10BD300009F500694D4500F0F88109F5E0594D45D8
:10BD400000F0F38167498D4204D001F580618D4296
:10BD500040F0F2814AF4406AC5F804A0C5F81880A2
:10BD6000AF63C5F820E0A96941F40061A961A96940
:10BD700021F48061A961A969A9611918012581F8D7
:10BD8000715E002581F8705E02F01F011A181CF028
:10BD9000020FD2F8342E3FD0042505FA01F1156ABE
:10BDA00025EA01051562156A29431162516C41F4B7
:10BDB0000041516495684C492940062906D0B1F5E7
:10BDC000803F03D0116841F0010111601A1802216F
:10BDD00082F8711ED2F8341E434A8D682A40062A22
:10BDE00006D0B2F5803F03D00A6842F001020A6033
:10BDF0000344012283F8712E21686379716001F197
:10BE00003402D01800213060D150BDE8F08794F89A
:10BE100006C08CF001013CE7012505FA01F1156A25
:10BE200025EA01051562156A294311622F498A42E4
:10BE3000BCD001F500618A42B8D001F540618A4268
:10BE4000B4D001F580618A42B0D001F580618A42A8
:10BE5000ACD001F500618A42ACD1A7E71918DFF830
:10BE60008C80D1F8341E0D6A25F480150D620D6AA0
:10BE7000D1F8049025F4001545EA0E5E0D6D25F00D
:10BE8000807525F4E045414545F4C04513D008F5DB
:10BE9000006841450FD008F5406841450BD008F5D2
:10BEA0008068414507D008F58068414503D008F512
:10BEB0000068414501D149F48029C1F804900D651D
:10BEC000CF64C1F820E00D6D45F400650D650D6D82
:10BED00025F480650D650D6D0D654EE7E8FC0408E1
:10BEE000C02900200040014007000100002C014053
:10BEF0001918DFF86C82D1F8341E0D6A25F48035EC
:10BF00000D620D6AD1F8049025F4003545EA0E4E15
:10BF10000D6D25F4803525F07005414545F060052F
:10BF200013D008F5006841450FD008F54068414539
:10BF30000BD008F58068414507D008F58068414579
:10BF400003D008F50068414501D149F48039C1F8B2
:10BF500004900D658F64C1F820E00D6D45F0080573
:10BF60000D650D6D25F004050D650D6D0D6504E77E
:10BF70001D18DFF8EC91D5F8345ED5F8208028F450
:10BF80008058C5F82080D5F82080D5F804A028F482
:10BF9000005848EA0E3ED5F81C8028F0807828F436
:10BFA000E6484D4548F4C04800F0B18009F5006905
:10BFB0004D4500F0AC8009F5E0594D4500F0A780F3
:10BFC00066498D4204D001F580618D4240F0BA800F
:10BFD0004AF4404AC5F804A0C5F81C802F64C5F88F
:10BFE00020E0E96941F40061E961E96921F48061D7
:10BFF000E961E969E961C0E61D18DFF86491D5F8E7
:10C00000345ED5F8208028F00108C5F82080D5F8E6
:10C010002080D5F804A028F002084EEA080ED5F8D2
:10C02000188028F4803828F073084D4548F06008DF
:10C0300013D009F500694D450FD009F540694D450C
:10C040000BD009F580694D4507D009F580694D454C
:10C0500003D009F500694D4507D12EF0080E41EADD
:10C060000E0E2EF0040E4AF4407AC5F804A0C5F86E
:10C0700018806F63C5F820E0A96941F00801A96143
:10C08000A96921F00401A961A969A96175E61D18D2
:10C09000DFF8CC90D5F8345ED5F8208028F480788D
:10C0A000C5F82080D5F82080D5F804A028F40078C1
:10C0B00048EA0E2ED5F81C8028F4803828F0730842
:10C0C0004D4548F0600829D009F500694D4525D057
:10C0D00009F5E0594D4521D020498D4203D001F5A5
:10C0E00080618D4234D14AF4405AC5F804A0C5F8A5
:10C0F0001C80EF63C5F820E0E96941F00801E961BF
:10C10000E96921F00401E961E969E96135E62EF4A4
:10C11000004E4EEA013E2EF4804E59E72EF4006E9A
:10C120004EEA012E2EF4806EDDE72EF0800E4EEAF0
:10C13000011E2EF0400E0DE601F580618D427FF468
:10C140000BAE07E601F580618D427FF443AF3FE718
:10C1500001F580618D42C8D1C5E700BF00400140B4
:10C16000002C0140204B10B5204C8446A3F6645EA1
:10C1700003F13000DA793AB15A7934F812100EEB43
:10C18000420289B2A2F8B81D0C339842F2D10CEBEE
:10C190004C030EEB830393F86B0D60B1ACF104021A
:10C1A000022A93F8691D09D9062905D80EEB410E1C
:10C1B000BEF8B80D80B210BD002010BD0629FBD816
:10C1C0000A4B33F81100BCF1050F80B2F3D1084BD4
:10C1D000084AB3F8AA3040F6B83101FB03F3B3FBC9
:10C1E000F0F3C2F8DC3310BD1C480020A02C012065
:10C1F0000075FF1F000000200448036E1BB1DB6ABE
:10C200000BB1603018470248704700BFC0290020BA
:10C210000C0C050838B5174CD4F8C83D1B883BB941
:10C22000154D002384F8D73D85F858306B6538BD2F
:10C23000D4F8CC2D002AF3DDD4F8D01D012A48888B
:10C2400006D001230C4DA4F8D40D84F8D63DE8E7C0
:10C250008A880132121A9A42F3D1074D28460023E8
:10C26000C5F88C3050F8603F1B69984741F008FAD8
:10C27000D7E700BFB83A0020C02900200648C36DA8
:10C280001BB1064B93F8D63D0BB10020704750F818
:10C29000603F5B68184700BFC0290020B83A002003
:10C2A00030B4174A174B92F858C003F6D85505EB2F
:10C2B0000C04C0E9004593F8D73D92F8580083423A
:10C2C00092F8580014D8834206D300231A46184621
:10C2D00030BCC1E90032704792F858001A1EC0F114
:10C2E000800330BC0CBF01200220C1E9003270473E
:10C2F0001B1A0022012030BCC1E90032704700BF88
:10C30000C0290020B83A00200D4B0E4A93F858106F
:10C3100092F8D70D93F85820904293F858200BD8F4
:10C32000904238BF93F858205B6D3ABFC2F180024B
:10C3300080180020184470475B6D801A18447047BD
:10C34000C0290020B83A002038B5124D124CD5F85B
:10C35000C82D937B012B06D0636D03F2FF736FF33F
:10C360000A03636538BD236E5B6A33B104F1600074
:10C37000984741F085F9D5F8C82D636D5288013B87
:10C3800013445242134003F2FF736FF30A036365D1
:10C3900038BD00BFB83A0020C029002070B51E4C3F
:10C3A0001E4D94F8583094F8581084B005F6D852C1
:10C3B0001344029395F8D73D03928B4220D894F80A
:10C3C0005820934214D294F858101E46C1F18001AF
:10C3D000F3B98C460122CDE9001610B9BCF13F0F2C
:10C3E00006D90023694602A841F0F8F895F8D73D30
:10C3F00094F85800C01AB0FA80F0400904B070BD3B
:10C4000094F858C0A3EB0C0C614600260122E2E729
:10C4100001EB030C0222DEE7C0290020B83A00201D
:10C420002DE9F043164685B0002935D0441E254D30
:10C43000254F04EB01084FF0000901E0A0452BD087
:10C4400095F8D70D14F8013F411C2844C9B280F873
:10C45000D83D0B0648BF002097F8583085F8D71D07
:10C460004ABF0146084685F8D79D994297F858304B
:10C4700036BFC3F18003C01AC0183F28DED997F831
:10C4800058309942DAD0114B5B78002BD6D000207F
:10C49000FFF784FFA045D3D1694602A8FFF700FF4C
:10C4A00020B1DDE9003213443F2B02D805B0BDE8CE
:10C4B000F0830246334602A841F090F805B0BDE88B
:10C4C000F08300BFB83A0020C029002000000020FF
:10C4D00030B585B0694602A8FFF7E2FE50B9084CB6
:10C4E00004F16005236E28465B6898470028F9D060
:10C4F00005B030BD0246012302A841F06FF8EEE717
:10C50000C029002070B5114D114C0023EB653BF0A4
:10C5100019FCC4F8D00DFFF76FFED4F8D03DC4F875
:10C52000C80D93B19A885B88D21A436802FB033323
:10C53000EB65FAF717F995F8583094F8D72D9A4229
:10C54000064601D0FFF7C4FF6E6570BDC02900200C
:10C55000B83A00202DE9F0410F4EF36D15468218D0
:10C560009A420E4A88BF1D1A92F8D72D96F8583075
:10C570009A4204460F4601D0FFF7AAFF326E0848E0
:10C580000023C6F88C302B46956A21463A46AC46C5
:10C59000BDE8F041604700BFC0290020B83A002044
:10C5A000202A00208C461346014662461846D1E7F1
:10C5B0002DE9F043DFF82881474D93B0FFF72AFEBD
:10C5C00098F8583095F8D72D9A4201D0FFF780FFA0
:10C5D000D8F85C700024C8F85440002F6CD03F4E4F
:10C5E0000AE098F8583095F8D72D9A4201D0FFF715
:10C5F0006FFF2034A7421BD922463146684601F01E
:10C6000095FB684641F0BAFB012201466846FFF7F8
:10C6100007FFA3B2002BE4D1D8F8AC30002BE0D058
:10C620009A881B6859690A4218BF12049A61D8E7B0
:10C63000FFF78AFE98F8583095F8D72D9A4201D026
:10C64000FFF746FF0023DFF89490C8F854301E46E9
:10C650001C4601E0A74229D92246494609A801F013
:10C6600065FB21220021684643F012F8202269462A
:10C670002046FFF76FFF2022054609A9684643F0D0
:10C68000F3F808B9202D00D00136A3B22034002BD6
:10C69000E0D1D8F8AC30002BDCD01A689B88516907
:10C6A0000B4218BF1B04A7429361D5D8B6FA86F097
:10C6B000400913B0BDE8F083FFF746FE98F8583004
:10C6C00095F8D72D9A4201D0FFF702FF0023C8F852
:10C6D00054300120EDE700BFB83A0020307905085A
:10C6E000C029002008B500210320FBF775FD72B6B4
:10C6F000FCF7CAFC154C08B5D4F8583E94F85E0E09
:10C70000ABB91420FEF722FF00BFD4F8583E5BB14E
:10C710001A689B88116994F85E2E0B4012B91BB100
:10C72000FFF7E0FF002BFBD0FAF74EF8ECE71968B3
:10C730009A880B69134020B1002BE2D10B6913409A
:10C74000FAE7002BDDD00B691340FAE7B83A002076
:10C75000F8B539F0D7FF1B20FBF7D4FF08B1292328
:10C76000C3801C20FBF7CEFF08B12923C380134CE4
:10C77000D4F8EC3013B10023C4F8EC30104B114E58
:10C78000C4F8E8600125002783F8607E84F8D4505F
:10C790003EF06EFF06F11C03C4F8EC300A4B5B7EE2
:10C7A000AB4201D02846F8BD5436C4F804613BF0D2
:10C7B00091FF064B83F823703846F8BDB84A002035
:10C7C000B83A0020E0030020B04B002000ED00E06C
:10C7D0002DE9F04F41F6946289B00021B948B94E75
:10C7E000B94D42F055FF4C220021B64842F050FFAF
:10C7F0004C220021B34842F04BFFB44B736201243A
:10C80000C6E90733356034713BF06CFEFFF77AFE02
:10C81000002108460AF07AFFF9F7A4FFB0F1000AF8
:10C8200040F32681AA4DDFF8C0C2002406F14C096E
:10C83000CDE901C42746264605F11C0B04E006F5A8
:10C840000066B24540F3AF80019AD2F8A430C2F836
:10C85000A830F9F7B9FF202259463046FFF77AFE93
:10C860009C491222584642F0FFFF0028E7D1BE4201
:10C8700024D00299984B01EB410203EB820302930F
:10C880004A1C1846C846F31B94490492039301F0CE
:10C890004DFA029B48F84C3B039B049AC9F80C7074
:10C8A000C9E90433D9F81C300292C9E908338C4B2A
:10C8B000C9F828300123C9F80830C146834BDFF896
:10C8C0002C82C9F81C3037461222A91818F80430F7
:10C8D000097F994202F101020BD00024202AF4D1F1
:10C8E0002037BA455946384654DBFFF733FE00225D
:10C8F000EBE70134152CF1D1D0197A492022FFF74A
:10C9000029FE00230A2207A97648CDF81CB001F0C1
:10C9100029FB80460798002301300A2207A90790C7
:10C9200001F020FB05900798002301300A2207A997
:10C93000079001F017FB04900798002301300A22AA
:10C9400007A9079001F00EFB0390079807A9013093
:10C9500000230A22079001F005FB074607980023F1
:10C9600001300A22194601F0FDFAB8F1000F11D08A
:10C97000DDE90432039943EA42127B0143EAC12311
:10C98000A8F2BC7843EA600342EA482243EA024341
:10C99000C9F81C30029B642B3FD0374606F5006671
:10C9A000B2453FF751AF029B642B36D0BE421BD03D
:10C9B000494C4A490C2202FB03445D1C2A4620468E
:10C9C00001F0B4F9F61B464BC9F82830C9E90376E3
:10C9D000D9F81C30C9F800400122C9E90833C9F868
:10C9E00014602B46C9F80820002B03F1010116DC66
:10C9F0004FEA4A03B3F1805F3BDB324B986828B9BA
:10CA00001A461B7913B11368002B75D10021084613
:10CA100009B0BDE8F04F0AF079BE642365214C26C9
:10CA20000193284BDFF8C8902D4F06FB01F41D1928
:10CA300032460021284642F02BFE3246002128468D
:10CA400042F026FE214E1F4B04F110014FF0010869
:10CA500043F80490CA18C5E90766C5F80880AF62B4
:10CA60006E6243F801A0019BC2F804A0991CBFE7C5
:10CA700021464C26134ADFF87C9006FB01F4151979
:10CA800000213246284642F003FE32460021284665
:10CA900042F0FEFD0B4A0D4E42F8049004F11001E5
:10CAA00001271046CAF100638A18BB404FF0020804
:10CAB000C5E9076685F80580AF606E624350536034
:10CAC0009BE700BF6051002074DB05080068214C23
:10CAD000B04B002050790508EC4B00206479050824
:10CAE000A5C50008CC4B0020C0290020747905089A
:10CAF0008C7905089C790508514900220023C1E979
:10CB0000102388640A46C86305460146D46C02F1C6
:10CB10004C03B4B19C689D644E1EB442C2E92355D7
:10CB2000DD6300F085804E1CB44273D113F8481CBD
:10CB300000293FF46BAF1A6443F8083C21461A46BB
:10CB4000E4E73F4A0226254615E0D36B16635B01F6
:10CB500018BF03F6FF73C2E9045514BF01EB13338A
:10CB6000334653631946916352F84C7FCB1A1C44E9
:10CB70004E1C0130CFB11379711E002BE5D1136922
:10CB800016635BB103F6FF73576901EB133353630D
:10CB90004FB107F6FF7701EB1731E4E757693346EA
:10CBA0005363002FF5D13146DDE7DFF89CC0CCF8A8
:10CBB000F4002448CCF8E8400139CCF8CC003E24FD
:10CBC00040203F25CCE93445CCF8E4108A0F8B0097
:10CBD000CCF8D800E1B140F2FF101B1842F100027E
:10CBE0005B0A43EAC25303F14002134403EBC10161
:10CBF000CCF8E030CB0DCCF8C430114BCCF8DC20B5
:10CC0000CCE93B334B02CCF8C810CCF8C030FDE681
:10CC10000123E8E78C427FF4F9AE00293FF4F6AE39
:10CC2000146CE66B0136E6631C6493641A466DE788
:10CC300000293FF4EBAE53F80C2C2146EDE700BF82
:10CC400060510020A8790508C0290020704700BF66
:10CC5000D0ED007AD0ED016A30EE677AE6EE877AA1
:10CC6000B0EE670AC0ED007A704700BFD0ED017AE0
:10CC7000D0ED026A30EE677A90ED000AE6EE877A30
:10CC800037EEC07AC0ED017AA6EE870A80ED000A81
:10CC9000704700BF90ED017AD0ED036AD0ED027AC3
:10CCA00030EE470AA6EE807A90ED000A80ED017A18
:10CCB00037EE676AE6EE867A37EEC07AC0ED027A22
:10CCC000A6EE870A80ED000A704700BFD0ED056A26
:10CCD000D0ED017A90ED066AD0ED025A90ED035A3C
:10CCE000C0ED066AB0EE407A26EEA70AD0ED007AD3
:10CCF00080ED057AA7EE870AD0ED077AA5EE860AC1
:10CD000090ED086AD0ED045AC0ED087AA5EE670AE6
:10CD1000A5EEC60A80ED070A704700BFF0EE406A34
:10CD2000D0ED007A90ED050A90ED067A90ED016A5B
:10CD3000D0ED035AA7EEA60AA6EE267AD0ED047A25
:10CD400090ED026A67EEC07AA5EEC07AE6EE267A2A
:10CD500080ED057AC0ED067A704700BF2DE9F047F7
:10CD6000DDF820A055460F4615F8011B002B06469E
:10CD700014460CBF4FF020094FF0300939B3002A98
:10CD80002BDD2B4600E09CB113F8012BA046013CA3
:10CD9000002AF8D1A8F1020854B144464946304669
:10CDA000B847013CFAD29AF8001008F1010459B1D1
:10CDB0003046B8472B4615F8011B0029F8D1A4EBE3
:10CDC0000A041819BDE8F0872046BDE8F087002A5C
:10CDD00002F1FF38E1DC0846F4E70024E8E700BF91
:10CDE00003685A1C02601970704700BF10B500F14B
:10CDF00000440246013C04E0B3EB0E0015D1A24210
:10CE000014D012F8013BA3F14100192811F8010BCD
:10CE1000A0F1410C98BF2033BCF1190F00F1200E96
:10CE2000EAD91B1A04D10028E9D110BD002010BD99
:10CE3000184610BD0278202A034600F10100F9D0FF
:10CE4000092AF7D02D2A29D02B2A03BF5A78B7EE0A
:10CE5000000A0346B7EE000AA2F13001C8B2092861
:10CE6000DFED4C7A10D8F2EE046A07EE101AB8EE35
:10CE7000C77A13F8012FA7EEA67AA2F13001C8B243
:10CE80000928F0EE477AF0D92E2A49D0197801F016
:10CE9000DF01452907D020EE270A70475A78BFEEF8
:10CEA000000A0346D8E710B459782D2962D02B29FF
:10CEB00054D0A1F13002092A03F1010355D800240E
:10CEC000002202EB820201EB420213F8011FA1F1E2
:10CED00030000928A2F13002F3D9B2F59A7F134647
:10CEE00028BF4FF49A73072A50D9DFED2B6A1A46F0
:10CEF000B7EE007A083A072A27EE267AFAD803F026
:10CF000007032BB1F2EE046A013B27EE267AFBD130
:10CF10006CB3C7EE877A5DF8044B20EE270A7047A2
:10CF20005978A1F13002D0B2092803F10103AED83B
:10CF3000F2EE046AF0EE665A07EE102AB8EEC77AEF
:10CF400013F8011F87EE266AA1F13002D0B209283A
:10CF500066EEA56A77EE867AEED998E79978A1F120
:10CF60003002092A03F10203A9D9B7EE007A67EE6D
:10CF7000877AD0E79978A1F13002092A03F10203F8
:10CF800088BFB7EE007AC4D8012499E7B7EE007ADB
:10CF9000B7E700BF0000000020BCBE4CF0B506792A
:10CFA00006F0E003402B03D145794FF0FF3406E053
:10CFB000602B4FF00105F8D1447905FA04F4002301
:10CFC000012006F00706AB4200D1F0BD052E0FD8B8
:10CFD000DFE806F00308101D242448B1C85CD75CC4
:10CFE00078400FE020B1C856D756C71B7842784129
:10CFF0000133E8E70028FBD031F8130032F8137052
:10D00000784080B220420CBF01200020F0E70028C9
:10D01000EED031F9130032F91370E6E70028E7D0BB
:10D0200051F8230052F82370DAE7037903F018036C
:10D03000102B1CD003D833B9B0F80B007047182B55
:10D04000FAD000207047104BB0F80B0093F9003075
:10D05000591C06BF0D4B1B78DBB203EB430203EBFD
:10D06000820303EBC30300EB430080B27047064B1F
:10D07000B0F80B0093F901305A1C06BF034B5B78E4
:10D08000DBB200EB4310F0E768040020F86F0020EB
:10D09000032870B518D80D4BC60003EBC000C94378
:10D0A000057D427D01F0010181EA0504A2420BD019
:10D0B00002693AB14D1B69421068928869410901C1
:10D0C0008A40826133445C7570BD00BFF86F0020F8
:10D0D0000379062B0FD1C9B20B2998BF074BC26841
:10D0E00094BF5956002101238B40134214BF0846B8
:10D0F0004FF0FF307047481C704700BFB0790508FB
:10D10000B5EEC00ADFED347AF1EE10FACCBF30EEA6
:10D11000270A30EE670ADFED317A20EE270A30B5B4
:10D12000FDEEC07A87B017EE904A054684EAE470B7
:10D13000002303A9A0EBE470CDE90033029339F09A
:10D140003DFE002CB4BF2D23202303A88DF8003012
:10D1500040F014FE012829D0022833D003281DD026
:10D1600003A9684642F09CFA684640F007FEC41ED8
:10D17000E4B222466946284642F068FB00232B555C
:10D18000284640F0FBFD2E232B5401300DEB04010B
:10D19000284442F0A1FA284607B030BD302303A945
:10D1A00068468DF8013042F07BFADDE743F2300249
:10D1B000302303A96846ADF801208DF8033042F012
:10D1C0006FFAD1E743F2300303A96846ADF80130A6
:10D1D00042F066FAC8E700BF6F12033A00007A44D3
:10D1E0000AF0D4B838B5054658B14C1E14F8011FE2
:10D1F000284619B9BDE838400AF0DEB80AF0C6F88A
:10D20000F4E738BD70B50546B0F8090037F0AAFF5D
:10D21000064B93F8306004462846FFF706FF16B128
:10D22000E368184470BDA368FBE700BFF86F0020F7
:10D2300038B505460C46FFF7E5FF2A7902F00703EB
:10D2400002F0E002602A29D1052B0CD8DFE803F0B8
:10D25000030B0F0B1B1B6A7901239340DBB202788F
:10D2600014B11343037038BD22EA0303FAE76A7965
:10D27000012393409BB2028814B113430380F2E769
:10D2800022EA0303FAE76B7901229A40036814B19A
:10D2900013430360E7E723EA0203FAE7052BE2D82A
:10D2A000DFE803F00303050507070470DBE70480EC
:10D2B000D9E70460D7E708B5202142F000FA034619
:10D2C000184623B10278202A03F10103F8D008BDE3
:10D2D00008B5CB0701D4FBF789FF08BD2DE9F34161
:10D2E000124D134F002305F8313F044600EB810631
:10D2F000B44203D10F4802B0BDE8F0813946284658
:10D3000042F0CEF92146684642F0E6F94FF00008B7
:10D310002021684642F0D3F928B96946284642F0F0
:10D32000BFF90434E4E780F80080F1E7F86F0020EB
:10D3300036ED0508297000202DE9FF479146044687
:10D340008A461E46FFF7C4FE421CBDF83070DDF869
:10D35000348005461FD0B9F1FF3F1FD0CDE9000949
:10D36000144A236831463846C0474A4620795FFA56
:10D370008AF1FAF757FB024600B10288D3B2039351
:10D38000C2F30323120BCDE90052029323680A4A29
:10D3900031463846C04704B0BDE8F0877B06FAD472
:10D3A0000C902368054A31463846C44604B0BDE8AF
:10D3B000F0476047F0DD0508FDDD050822DE0508C1
:10D3C0002DE9F043154685B06A1C8946BDF83060EA
:10D3D0000D9F194628D04FEA101800F00F0408F1ED
:10D3E0004008CDE90045174A43463046B847C0B12A
:10D3F000EBB20F2BD9F8000099F8051011D82A4686
:10D40000FAF758FB68B1038802780392C3F303224A
:10D410001B0BCDE90043029243460B4A00213046E4
:10D42000B84705B0BDE8F0837306FAD40309074A8C
:10D4300000F00F000C9040333046BC4605B0BDE80C
:10D44000F043604731DE050843DE05086DDE050860
:10D4500000B501EB020E714516D001390EF1FF3E09
:10D4600041F2210C11F8013F082280EA032003B2A7
:10D47000002B4FEA4000B6BF8CEA430380B298B25B
:10D48000013AF4D18E45EDD15DF804FBF8B5164DA7
:10D490006B78BE2B26D1022229464FF6FF70FFF78C
:10D4A000D7FF124FAC1C22884AB1A618BE4219D22F
:10D4B000052A17D92146FFF7CBFF3446F3E721466B
:10D4C0000222FFF7C5FF0222A118FFF7C1FF0634B1
:10D4D000074B641BA3F8524041F60F53C31A58423E
:10D4E0005841F8BD0020FCE700400008006000083B
:10D4F000F86F00204840082341B240000029C0B224
:10D50000B8BF5040013BF7D1704700BF30B5056848
:10D510008D42044618D901F1FF3E681E00231EF813
:10D5200001CF082183EA0C034FFA83FC5B00BCF1B6
:10D53000000FDBB2B8BF53400139F5D17045EED1D1
:10D540006A1C22602B7030BD00236A1C22602B7085
:10D5500030BD00BF08B5DFED2D0A41F03FFBDFED28
:10D560002C7AB4EEE70AF1EE10FA28DDDFED276A37
:10D570009FED287AF0EE407AF4EEC77AF1EE10FAD9
:10D5800030EE660AF6DCDFED247AB4EEE70AF1EE5F
:10D5900010FA2FDDDFED1E7A37EEC00A20EE007A9A
:10D5A0009FED1E6ADFED1E6ADFED1E7AE7EE066A6A
:10D5B00020EE076AE6EE877AA6EE270A08BDDFEDC1
:10D5C0001A7AB4EEE70AF1EE10FADCD5DFED0F6A55
:10D5D0009FED167AF0EE407AF4EEC77AF1EE10FA8B
:10D5E00030EE260AF6D4DFED0C7AB4EEE70AF1EE5F
:10D5F00010FACFDCDFED0E7AB4EEE70AF1EE10FAA6
:10D6000044BFDFED097A37EEC00AC7E7DB0FC94038
:10D61000DB0F4940E4CB1641DB0FC93F92E741B92C
:10D620009730083C15A82ABEDB0F49C0E4CB16C1D1
:10D63000DB0FC9BF38B5DFED2D7A2DED048B08EE79
:10D64000101A20EE270AB8EE488AF0EE609A28EE0B
:10D65000008A1546B0EE480AB0EE419A0446FFF73C
:10D6600079FFDFED237AF0EE408A38EE270AFFF7E4
:10D6700071FFF6EE007A68EEA78A012D88EEA97A8E
:10D6800028D0F7EE005A75EEC06AB8EE006A66EE72
:10D69000A77A20EE060A75EEC75AB7EE005A37EEA3
:10D6A000056A84ED099A85EE067ABDEC048B67EE77
:10D6B000877A66EE876A20EE070A25EE877AC4ED40
:10D6C000007AC4ED016AC4ED027A84ED030A84EDA8
:10D6D000047A38BDF8EE006A60EE266AF7EE007A4A
:10D6E00077EEC75AB0EE660AD7E700BF27D4D23626
:10D6F000DB0FC93F10B5DFED070A0446B7EE001A8D
:10D700000022FFF797FF0023A36163612362E361B7
:10D7100010BD00BFF304353FB0EEC07AF0EEE06A12
:10D72000F4EEC76AF1EE10FAB4BFF0EE475AF0EE2D
:10D73000665AF5EE405AF1EE10FAF0EE407A44D017
:10D74000F4EEC76AF1EE10FA8CBFB0EE475AB0EEB5
:10D75000665A85EE256A9FED1E2A9FED1E3A9FEDC3
:10D760001E4ADFED1E4ADFED1E2ADFED1E3A9FED59
:10D770001E5AA6EE423AE6EE223AA6EE034AF7EE2B
:10D78000005AE6EE044AE6EE235AA6EE245A85EE47
:10D79000250AF4EEC76AF1EE10FA48BF9FED137A3E
:10D7A000F5EEC00A48BF37EE400AF1EE10FA48BF66
:10D7B0009FED0F7AF5EEC07A48BF37EE400AF1EEE2
:10D7C00010FA48BFB1EE400A70479FED070AE0E744
:10D7D00039094E3DE3B59E3E88FA163E45FE7F3F31
:10D7E00099FB243F69A2163EA7DFA834DB0FC93F8F
:10D7F000DB0F49402DE9F04F17460E4617F8011B85
:10D8000089B0002900F051821446834600259A46CB
:10D8100009E05846B04701353C46274617F8011B3A
:10D82000002900F08D802529F3D16178302900F09E
:10D830008B8002340023A1F13000C2B2092A4FF0DC
:10D84000000260D96C2900F083807829E5D8572937
:10D8500040F2E980A1F158002028DED801A757F84E
:10D8600020F000BF45DA00081BD800081BD80008CC
:10D870001BD800081BD800081BD800081BD80008BC
:10D880001BD800081BD800081BD800081BD80008AC
:10D89000F9D9000879DB00081BD800081BD800085C
:10D8A0001BD800081BD800081BD800081BD800088C
:10D8B0001BD800081BD800081BD800081BDA00087A
:10D8C0001BD800081BD800081BD800081BD800086C
:10D8D00007DA00081BD800080BDB00081BD800087B
:10D8E0001BD8000845DA0008BEF1050FAAD8A1F13F
:10D8F00037000A2815D114F8011B02EB820200EB55
:10D900004202A1F13000C7B2092FA1F1610CA1F1CF
:10D91000410EF0D9BCF1050FE6D8A1F157000A2855
:10D92000E9D0572996D825297FF477AF27462521B6
:10D930005846B04717F8011B013500297FF473AF33
:10D94000284609B0BDE8F08FA1780123033472E7BF
:10D9500014F801EBBEF1780F3FF65FAFBEF1570F41
:10D9600068D9AEF1580120293FF657AF01A050F811
:10D9700021F000BFABDA00081BD800081BD8000854
:10D980001BD800081BD800081BD800081BD80008AB
:10D990001BD800081BD800081BD800081BD800089B
:10D9A000F9D900082DDC00081BD800081BD8000896
:10D9B0001BD800081BD800081BD800081BD800087B
:10D9C0001BD800081BD800081BD800081BDA000869
:10D9D0001BD800081BD800081BD800081BD800085B
:10D9E00007DA00081BD80008D7DB00081BD800089E
:10D9F0001BD80008ABDA00085AF8041B5846C9B215
:10DA0000B047013509E75AF8043B0093314600233B
:10DA10005846FFF7A3F90544FFE6534653F8042B95
:10DA200015609A46F9E600297FF47DAF284609B0D3
:10DA3000BDE8F08FBEF1000F82D0BEF1250F3FF49C
:10DA400075AFEAE65AF804EBBEF10F0F4FF0010094
:10DA500040F239810001BEFBF0FCBCF10F0FF9D898
:10DA6000002800F02D8105AFB9460EE058290CBF03
:10DA70004FF037084FF05708E04400FB1CEE000958
:10DA800009F8018B0DD0BEFBF0FCBCF1090FEDDCF9
:10DA90004FF03008E04400FB1CEE000909F8018B50
:10DAA000F1D1002189F800105FE0D146012159F839
:10DAB00004CBBCF10F0F40F201810901BCFBF1F076
:10DAC0000F28FAD8002900F0F58005AFB8460FE01E
:10DAD000BEF1580F0CBF4FF0370A4FF0570A82447F
:10DAE00001FB10CC090908F801AB0CD0BCFBF1F02C
:10DAF0000928EDDC4FF0300A824401FB10CC090903
:10DB000008F801ABF2D1CA462CE05AF8040B0928F8
:10DB10004FF0010109D901EB81014900B0FBF1F798
:10DB2000092FF8D8002900F0C28005AFCDE9023AEC
:10DB3000DFF89891B84600E07146B0FBF1F30A2B8C
:10DB4000B4BF4FF0300C4FF0570CA9FB01AE9C4412
:10DB5000092908F801CB01FB13004FEADE0EEBD8D0
:10DB6000DDE9023A002188F8001000973146584656
:10DB7000FFF7F4F8054450E65AF804CBBCF1000F67
:10DB8000C0F2828005AFB846BCF1090FE6464FF0FF
:10DB9000010108DD01EB81014900BCFBF1F009281E
:10DBA000F8D80029DED0CDE9023ADFF8209100E074
:10DBB0006146BEFBF1F30A2BB4BF30205720A9FB0E
:10DBC00001AC1844092908F8010B01FB13EE4FEAD8
:10DBD000DC0CEDD8C4E75AF8040B09284FF001011A
:10DBE00008D901EB81014900B0FBF1F7092FF8D802
:10DBF00000295CD005AFCDE90243DFF8D090B846EC
:10DC000000E06146B0FBF1F30A2BB4BF3024572487
:10DC1000A9FB01EC1C44092908F8014B01FB130086
:10DC20004FEADC0CEDD8DDE902439BE75AF8040B20
:10DC3000002832DB05AFB84609284FF0010109D9A9
:10DC400001EB81014900B0FBF1FCBCF1090FF7D8F1
:10DC5000002987D0CDE90243DFF8709000E06146EB
:10DC6000B0FBF1F30A2BB4BF30245724A9FB01EC1D
:10DC70001C44092908F8014B01FB13004FEADC0C96
:10DC8000EDD8DDE902436DE72D21CCF1000C8DF8D4
:10DC900014100DF1150805AF76E72D2140428DF8DF
:10DCA00014100DF1150805AFC6E70D4648E605AF9F
:10DCB000B84657E705AFB846CA4653E7604604E79B
:10DCC00005AFB946EDE6F446CDE600BFCDCCCCCCF1
:10DCD000F8B5114C0746606D0D461646A0B10F49C8
:10DCE000FFF780FA606D3946FFF77CFA0C49606DEA
:10DCF000FFF778FA0B49606D33462A46FFF77AFD45
:10DD00000949606DFFF76EFA94F8583013B101239A
:10DD100084F85930F8BD00BFF86F002081DE050897
:10DD20006FF40508E1D100088EDE05080EB400B5D9
:10DD300084B005AB019053F8042B0649039301A866
:10DD4000FFF758FD019B00221A7004B05DF804EB48
:10DD500003B07047E1CD0008F7B5114E07463046D5
:10DD6000002300F85A3F0C460E4B0F49002F18BFF6
:10DD70001946154641F094FC0C4F04EB45055A3604
:10DD8000AC4202D10A4803B0F0BD394634F8022B48
:10DD90006846FFF7CBFF6946304641F081FCEFE76C
:10DDA000F86F002092DE05089BDE0508A4DE05085A
:10DDB00052700020F7B50C4E0C4F002306F88B3F35
:10DDC000044600EB4105AC4202D1094803B0F0BD66
:10DDD000394634F8022B6846FFF7A8FF69463046FB
:10DDE00041F05EFCEFE700BFF86F002048DF050858
:10DDF00083700020F8B5084F4E1E054601F11F0440
:10DE000016F8012F28463946FFF790FFA64205F184
:10DE10000205F5D1F8BD00BFA9DE05080246531C76
:10DE2000084605D1034B1A681B790A600B717047CD
:10DE300001497BE72CDE050849DF050803685A1C09
:10DE4000026019700368090A5A1C02601970704751
:10DE500010B402681346511C016013F8021B0360E2
:10DE6000D31C5478036093781B0443EA0423141DE5
:10DE70000460D0785DF8044B0B4343EA00607047C0
:10DE8000A0F13003092B07D920F0200041381928D0
:10DE90008CBF0020012070470120704730380928CE
:10DEA0008CBF002001207047413819288CBF00200A
:10DEB00001207047613819288CBF0020012070476D
:10DEC000202805D0093804288CBF00200120704785
:10DED00001207047A0F14103192B98BF20307047F3
:10DEE000A0F16103192B98BF2038704702B310B519
:10DEF0008446841803E0981A15D1A44514D01CF860
:10DF0000013BA3F14100192811F8010BA0F1410ECA
:10DF100098BF2033BEF1190F00F12002EBD91B1A74
:10DF200004D10028E9D110BD002010BD184610BD55
:10DF30001046704770B5044608460D463FF01EFF78
:10DF4000064602E014F8013F43B132462946204616
:10DF5000FFF7CCFF0028F5D1204670BD1C462046B7
:10DF600070BD00BF2DE9F043064686469EF800C00E
:10DF7000BCF1200F7446ACF109050EF1010EF5D08D
:10DF8000042DF3D9BCF12B0F64D0BCF12D0F26D199
:10DF90000127102A94F801C004F1010423D04FF0A6
:10DFA000FF35B5FBF2F502FB05FE6FEA0E0E5FFAD8
:10DFB0008EFE9046002014F801CBBCF1390F4CF0D6
:10DFC0002009ACF1300C29D85FFA8CFC944528DA92
:10DFD000A84226461ED81BD000FB08C0EBE7102A3B
:10DFE0004FF00007DBD1BCF1300F0AD16078A0F10F
:10DFF0004105192D98BF2030661C78280CBF0234CB
:10E0000034466FF070454FF00F0E4FF01008D1E717
:10E01000F445E1D94FF0FF301F40CCE7B9F1600F74
:10E020000AD801B10E6067B923B16FF0004398427E
:10E0300028BF1846BDE8F083A9F157095FFA89FCAB
:10E04000C4E723B1B0F1004F28BF4FF00040404279
:10E05000BDE8F08300279CE701230A22002181E725
:10E0600070B50D461446FFF726F90646A0B1FFF736
:10E07000F3FF40F634039842A8BF1846B0F5617F1D
:10E08000B8BF4FF46170A0F561731922B3FBF2F3CE
:10E090002B702378013323703046FFF70CF90646C6
:10E0A000A0B1FFF7D9FF40F634039842A8BF184645
:10E0B000B0F5617FB8BF4FF46170A0F561731922AC
:10E0C000B3FBF2F36B70237801332370304670BDDD
:10E0D0002DE9F04116461F460446394630464FF4B6
:10E0E0007A7200233FF052FE3C4D3D4B054483FBCA
:10E0F00005602844E917C1EB601183FB01030B4461
:10E10000384EC817C0EB631086FB003CC317364E71
:10E11000C3EBAC0386FB03764FEAE37ECEEBE61E51
:10E12000C1EB0116A5EB860CC0EB0015A1EB850138
:10E13000617103EB4301A0EBC10040F2B55101FB5B
:10E140001E33B3F5896F84F806C020714FEA8E063E
:10E1500033DA40F2DA218B4237DCB3F5B77FB4BF54
:10E160004FF0000E4FF0010E204F0EEB4E0107EB6B
:10E17000C1017546C88A4FEA4E0808EB0E0C07EB42
:10E18000CC0C0CF1160C0B2101E03CF8020D98426E
:10E1900010DD0139F9D1F044012137F83800A170C0
:10E1A000013306F5FA6E1B1A7544E370228125804F
:10E1B000BDE8F0810131C9B2F1E703250B4F40F210
:10E1C0009650AE464FF00608D7E70225074F40F2BB
:10E1D0002940AE464FF00408CFE700BF80BC92C78D
:10E1E00089888888ABAAAA2A73B06D16600C0508C6
:10E1F0000C4B10B5D3E92E4354EA030209D1014672
:10E2000040F201130020C1F80230887108800881B3
:10E2100010BD054A1268121943F10003FFF758FFB9
:10E22000012010BDF86F0020642A00202DE9F04184
:10E23000044694421546084609D2B4FBF2F6154B43
:10E2400005FB16441B5D00F8013BBDE8F081B4FB03
:10E25000F2F69642B6FBF2F70CD20E4B05FB1767AF
:10E2600005FB1644DA5D00F8012B1B5D00F8013B4D
:10E27000BDE8F081BA42B7FBF2F807D9054B05FBC0
:10E28000187813F8082000F8012BE7E74046FFF75D
:10E29000CDFFF3E7CC79050830B5854CB4F8EC3404
:10E2A000B4F8F024B4F8F414B4F8F604B3F57A7FB3
:10E2B00088BF4FF47A7383B088BFA4F8EC34B4F805
:10E2C000EE34B3F57A7F84BF4FF47A73A4F8EE345A
:10E2D000B4F8F234B2F57A7F84BF4FF47A72A4F8BE
:10E2E000F024B3F57A7F84BF0023A4F8F234B1F5AB
:10E2F0007A7F6FD94FF47A718842A4F8F41400F24F
:10E3000088809A429CBF0023A4F8F03481429CBFCD
:10E310000023A4F8F434B4F80435B4F802259A4282
:10E3200084BF0023A4F80235B4F80C35002B3ED08E
:10E33000604DA979AA7800295ED1062A40F29C8016
:10E340002879002840F087809FED5B7A94F8E028D8
:10E3500007EE903A06EE902AF8EEE77AB8EEE66A13
:10E36000C6EE276A002973D1B4EEE67AF1EE10FA10
:10E370001DDD27EE277AFCEEC77ACDED017A9DF8F8
:10E38000043007EE903AF8EEE77AB4EEE77AF1EE71
:10E3900010FAC4BF0133DBB2002B7CD0102BA8BF16
:10E3A0001023DBB2934238BF134684F8E03862781A
:10E3B000032A1DD8414B03EB42132278C4F8E838F6
:10E3C000032A0ED83E4BEA2102FB0133C4F8EC3895
:10E3D00003B030BDB0F57A7F84BF0020A4F8F60406
:10E3E0008FE7374BC4F8EC380022227003B030BD01
:10E3F0000022324B6270E0E7072A13D0B3F57A6F40
:10E400009BD994F8E0080228B8BF022084F8E008FD
:10E4100093E700219A42A4F8F6143FF67CAFA4F8E3
:10E42000F01478E70622B3F57A6FAA7035D82A7906
:10E43000002ABCD194F8E02807EE903A07EE102AA3
:10E44000F8EEE77AB8EEC76A9FED1E7AC6EE276A45
:10E4500037EE077A88E7053A032AA8D99FED167A9E
:10E46000B7EE000A80EE070A40F0EAFB2B888342F1
:10E4700028BF03462B809AE7134800EB820090EDFB
:10E48000187A287900283FF461AF531F032B8ED9E7
:10E49000002A8CD0E4E7012383E794F8E028297967
:10E4A000022AB8BF022284F8E0280029C2D07EE701
:10E4B000F86F0020343B00206F120338B870002042
:10E4C0003871002017B7D138600C05082DE9F04FDE
:10E4D000984C85B094F8F038A3F11702022A00AFE7
:10E4E00000F28B82944BBB6094F80039FB60934B35
:10E4F000DFF858B203F1540899464FF0000A1EE0C5
:10E5000099F90420142A00F00883284641F06CFA97
:10E51000AA0322D5012800F00083082800F3FD8219
:10E5200016B115EA0B0F06D1F96828463EF016F928
:10E53000002800F0F28209F10C09C84513D0D9F87F
:10E54000005015F00106DBD0284641F04DFA0AF1E3
:10E55000010AAA035FFA8AFADCD40128DDDC09F19A
:10E560000C09C845EBD10AF1FF32022A00F2D5822C
:10E57000D4F88419D4F88809714B94F895C9C7F870
:10E580000CC021F0800620F08008C4F88469C4F82B
:10E59000888903F56A7A4FF47A794FF0000E4FF0CC
:10E5A000640B7960054633F8082CB2F57A7FB3F82E
:10E5B000462088BF23F8089CB2F57A7F33F8062CF2
:10E5C00088BFA3F84690B2F57A7F33F8042C88BF51
:10E5D00023F8069C33F8061CB2F57A7F84BF00222C
:10E5E00023F804EC9142B3F85A10B3F85C2098BFBA
:10E5F00023F806EC914293F86B2088BFA3F85AE009
:10E60000013A632A93F86C2088BF83F86BB001321B
:10E61000D2B2092A88BF83F86CE003F165010022B9
:10E6200013F8320011F801CF0132844538BF81F868
:10E6300000E0032AF4D1FA68012A18BF83F886E0C3
:10E64000EA339A45AFD1DFF808A179689AF8023029
:10E65000042B00F0988243B9BAF80030B3F5F07F8C
:10E6600084BF4FF4F073AAF80030FFF715FE0021C5
:10E6700094F8AF2961B9092A0AD0531E5D0003F04E
:10E68000030305F00805C3EB0313002A40F0D38110
:10E69000B4F8BE29B4F8BC391343B4F8C029134305
:10E6A0001BB213B10123A4F8C239264B3340002B0F
:10E6B00000F0D281F30700F14282750440F1D48169
:10E6C000214B1E4008EA0308C4F88469C4F888890D
:10E6D000320440F1D781002384F8073984F81739D0
:10E6E000DFF8709009F178064B4602E006339E424F
:10E6F0000CD01A780A2AF9D19978DA78914202D3A3
:10E700005A79002AF2D00A201FF076FD00234FF438
:10E71000806084F8403A0BF0C7FB002800F0468286
:10E72000CB469BF8051011B39BF80000E8B14B46AF
:10E7300015E000BFF86F0020600C05082479002068
:10E740004271002009600002F6DFFFFDBC020200FA
:10E75000343B0020C079002006339E4207D01A784F
:10E760008A42F9D15A79002AF6D01FF045FD0BF103
:10E77000060B5E45D5D19AF802B0BBF1080F00F048
:10E78000D18194F89539A17BA3F10103B3FA83F306
:10E790005B0984F8443A94F89639A3F10103B3FA7B
:10E7A00083F35B0984F84A3A94F8E934032BC8F3FD
:10E7B000C03288BF002384F8472A88BF84F8E93430
:10E7C000C04AD4F88439134008EA0202C4F88439F4
:10E7D000C4F88829002900F0CB81B4F8643A002BF2
:10E7E00040F0BC81D4F8683AB3F5000F24BF002391
:10E7F000C4F8683AD4F8703A23F4007323F00203A3
:10E800001BB140F20223C4F8703A94F86C3A94F8C1
:10E81000748A013B042B88BF0123ABF1050B88BF31
:10E8200084F86C3ABBF1030F40F238810025B8F14F
:10E83000000F22D0FD60DFF8B0B2454606E0A8F137
:10E840000603A3EB0A039D4240F22581D8461BF83C
:10E85000010F0028F3D00AF0EBF80028EFD08379FD
:10E860009B07ECD5FD6801233DB19AF8112052B900
:10E870009AF80520012A00D02BB19AF8063013B17E
:10E8800000238AF80630B4F8D23B03F00F02042AC2
:10E8900003D8C3F30313022B03D94FF42063A4F866
:10E8A000D23BB4F8D43B03F00F02042A03D8C3F3DD
:10E8B0000313022B03D940F60123A4F8D43B94F8A8
:10E8C000411C94F84D2C94F8403C914205D900220B
:10E8D00084F8412C53B1A4F8442C94F84C2C9A425F
:10E8E00004D2002384F8403CA4F8443C94F8363D1C
:10E8F00094F8422CDFF8F4C1D7F808A09A4284BFFC
:10E90000002384F8423C0CF1800B634613F8032D7E
:10E9100002EB4202524492F8348292F835E292F8C5
:10E92000365213F8010F9979DA784045A8BF40466E
:10E930007145A8BF7146AA42A8BF2A466345187010
:10E940009971DA70EDD103F1200CDC45DDD1D4F8FA
:10E950002429002A00F0FC800020012199F80030D1
:10E960002B2B08D199F80130043301FA03F3134239
:10E970001CBF9A43012009F106094E45EED108B1AA
:10E98000C4F82429504D6E4605F108082B4602E0D4
:10E99000434500F0AD8013F8012F072AF8D9002372
:10E9A00005F8013F0133082BFAD1B4F88E29B4F8E9
:10E9B0008C399A42B54602D3444BC4F88C39444B47
:10E9C000444DFF2284F8682D03F1540013F9082CFC
:10E9D000142A05D053F80C1C35EA010100F0D08050
:10E9E0000C339842F2D13C4B5A79022A01D10022D1
:10E9F0005A711437BD46BDE8F08F384ABA601146E7
:10EA0000DA0001EBC30393F87C1021B1D3F8803016
:10EA1000002B00F0D480BB68134493F87D20002ABB
:10EA20003FF462AD93F85C31002B7FF45DAD1823A9
:10EA300084F8F03858E5AA00A2EB95022848C2EB0A
:10EA40000212C3EB031392009B000180A4F8B229C9
:10EA5000A4F8B43901210BE646F0080648F008088E
:10EA6000C4F88469C4F88889300740F1B2801D4B2E
:10EA70001E4008EA03083204C4F88469C4F888898F
:10EA80003FF529AE94F80739002B00F09C80002355
:10EA900084F8173924E6FD680023E5E600228AF8A9
:10EAA00004200125B8F1000F7FF4C4AE9AF81130AC
:10EAB000002B7FF4E8AE9AF80530012B7FF4E3AE2B
:10EAC000DBE600BF3DD45418463B0020AE014A01AE
:10EAD0003079002001000200C44B0020600C0508C2
:10EAE000A8790020FE9FFFFD3B3B0020BD70002069
:10EAF00088B0E9462022FF21484640F0C9FD3B4A44
:10EB000004E0424549F823303FF44FAF12F8013F8B
:10EB100059F823100131F4D041E73549354836F032
:10EB200037FB25E59AF80630002B3FF42AAE9AF819
:10EB30001130012B04BF02238AF8113021E62E4B3D
:10EB40001E4008EA0308C4F88469C4F88889BFE550
:10EB50002B201FF051FBD4F82429FDE694F8600A1D
:10EB600009F066FF00287FF43DAEA4F8640A39E698
:10EB700022490B430A43C4F88439C4F888292CE697
:10EB800084F8682D2FE7BAF8203021F4845625F454
:10EB90008458B3F57A7FC4F88469C4F88889BFF4CF
:10EBA00064AD4FF47A73AAF820305EE5D4F8843966
:10EBB00023F0006328F00068C4F88439B0E5172317
:10EBC00084F8F03827E742F201031E427FF45FAF7A
:10EBD00086E5B1047FF57CAD094B1E4008EA0308C9
:10EBE000C4F88469C4F8888972E500BF463B0020F8
:10EBF000247900203CFF0508F79FFFFD0004040076
:10EC0000F6BFFFFD2DE9F04F2DED028BA84F97F8D1
:10EC10006C3D013B012B83B040F23381D7F89C3D22
:10EC2000A44EDFF8BC9203F2DC534E45C7F89C3D7E
:10EC300080F03B81012301939F4BDFF8A8B206F1DE
:10EC40001C0503F102089C4B5988002900F004813F
:10EC500008EB01025A4580F0FF80444608E0118825
:10EC600014460A44002900F0F7805A4580F0F480E9
:10EC7000052940F2F18035F81C3C6188C3F30B0391
:10EC80009942ECD163799B07E9D155F8141C23888C
:10EC900094F804A00093304636F07AFA35F81C1C3C
:10ECA000BAEB113F00F0DE800023019335F8181C09
:10ECB00055F8140C55F8044CC1F30B0138F072FCF4
:10ECC0001C364E45206005F11C05BCD3D7F88439AD
:10ECD0007A4CC7F88839FFF7F9FB3B787978784D9B
:10ECE000EA2203FB0242A4F1800303EB4113C7F8BD
:10ECF000EC28C7F8E8381FF087F84FF0FF33D7F853
:10ED0000EC086B6021F034F81FF0BEFA04F68803BB
:10ED100004F5106103E00633994200F0AD801A78E3
:10ED2000002AF8D19C78D878844202D358790028F8
:10ED3000F1D097F8BC3DB7F8C01D2A7203EB8303EE
:10ED4000642202FB01F103EB830364294FEA83038E
:10ED5000B8BF6421642B4FF00002B8BF6423594C44
:10ED6000C7F8981DC7F8B01DC7F89C2DC7F8A02D8F
:10ED7000C7F8A42DC7F8A82DC7F8AC2DA7F8B42D57
:10ED800087F8B62DC7F8943DC7F8EC4D25F0F6FD91
:10ED9000B7F9063E9FED4C7ADFED4C6ADFED4C8A09
:10EDA000B7F8F45D97F8F66D08EE103AB7F8023E42
:10EDB000B8EEC88A07EE903AB7F8003E28EE078A08
:10EDC00007EE103AF8EEE77AB8EEC77A67EEA67A61
:10EDD00027EE267A04F23C4338EE280A83ED017AC6
:10EDE000C3ED007AFEF7B6FBB0EE480AFEF7B2FBC1
:10EDF00097F8043E9FED377A07EE903AF8EEE77AFF
:10EE0000B0EE680AA7EE870AFEF7A4FB07EE905A59
:10EE1000DFED316AC7F8106EF8EEE77A04F24C4382
:10EE200086EEA77A04F58A6483ED000A84ED007A01
:10EE30000EF020F997F86C3D013B012B2DD9274AA4
:10EE400001981268C7F89C2D012387F8B53D03B0DF
:10EE5000BDEC028BBDE8F08F55F8141C304636F03F
:10EE600097F921E7009BA11D9A1F304636F0C6F99D
:10EE700000287FF41BAF17E7FA7B003A18BF012286
:10EE800057E7FBF74FFE00F5B71000F55870022268
:10EE9000C7F8880D87F88C2DC0E6FBF743FE0223E8
:10EEA000C7F8880D87F88C3DC9E7012301930DE76A
:10EEB000F86F002094FE050800400008387100201B
:10EEC00068040020B479002088C3E43A17B7D13829
:10EED000DB0FC93F35FA8E3CC0C9FB48642A0020CD
:10EEE0001C0706080060000838B50122184D841878
:10EEF0000328034685F8142EE4B217D9FF2824D03E
:10EF0000144A002341F2024100E034B10233402BA5
:10EF100022F8021B04F1FF34F7D11D44FF2385F8CA
:10EF2000183EBDE838400E200BF05AB9EA2205F52C
:10EF3000A07003FB02002B70C5F8EC0820F018FF4E
:10EF40001FF0CCFE1FF0AEFFDAE70023E5E700BFBD
:10EF5000F86F0020107E0020054BD3F85C2E0121B5
:10EF600042F4001283F8591EC3F85C2E704700BFAC
:10EF7000F86F00202DE9F0470568C5F30A0386B055
:10EF800004460E46002B5ED1CDE902330493B5F161
:10EF9000006F4FF00103059324D3424BB3F8E020F8
:10EFA0004FF6FF739A421BD03F4BD3F8E0253F4BFF
:10EFB00003EA422303F100639D4213D2012303932A
:10EFC0002B4603F17843DB0A01A902A8049336F02B
:10EFD00049FA002837D04FF0FF3006B0BDE8F0877F
:10EFE000334BE9E72F4BB3F8E0104FF6FF7399422C
:10EFF0000FD02D4B2D4AD3F8E03502EA432202F11F
:10F0000000639D420BD20A210520FCF72BFC38F04F
:10F0100023FF284B9D42F6D901334FF4802213443D
:10F020009D42F0D2022303934FF6FF73994207D01B
:10F030001D4BD3F8E0251D4B03EA4223EB1AC0E732
:10F040004FF48023FAE7D6E900A91B4E337B012B4E
:10F0500007D00123337338F0D5FE074620B10023D3
:10F0600033736FF00200B8E7DFF850803061D8F8F2
:10F07000143043F00103C8F81430C5F800A0BFF302
:10F080006F8FC5F8049038F0BDFED8F8143023F027
:10F090000103C8F8143037730028E2D1236808331D
:10F0A00023609AE70075FF1F0070FF1F00FEFF013D
:10F0B00000000408FFFF030868040020002002404D
:10F0C0002DE9F0415A4E3378B12B8AB075D1FEF755
:10F0D000DDF980F00104E4B2564B574DB3F84332EA
:10F0E000564FADF8003004F00104BD4267D3002C48
:10F0F00000F09B801022002106A840F0C9FA504B76
:10F1000004969B1B05934F4B5A69002A05DA4E4A19
:10F110009A6002F188329A605B69474D4FF48073C0
:10F120000222694604A8ADF824303EF09BF8022282
:10F1300069464FF6FF70FEF78BF94FF00008044662
:10F14000BD424AD3022201A904A80025ADF804500B
:10F150003EF088F8022201A92046FEF779F940BA6C
:10F16000C043ADF80800022204A802A93EF07AF8D4
:10F17000089888B106ABC0F108022946184440F04F
:10F1800087FA9DF9240018B906A904A8FFF7F2FE32
:10F1900000238DF8240008939DF825302BB1294BCE
:10F1A0005A6942F000425A615B699DF92400B0FA45
:10F1B00080F040090AB0BDE8F08101248CE7A988FD
:10F1C000AB69A868D3F80080C1F30B0138F0EAF905
:10F1D0001C35804518BF012487E7AE888DF80D8067
:10F1E000C6F30B06B31DADF808302B88C3F30B0232
:10F1F000ADF80A201B0B062202A904A88DF80C30DA
:10F200003EF030F8062202A92046FEF721F9A9684F
:10F210000446324604A83EF025F8A9682046324646
:10F22000FEF716F91C3504468AE70120C2E700BF45
:10F2300000400008600C050894FE05081C0706083D
:10F240000060000800200240230167452DE9F047D7
:10F25000874CFFF73BF994F86C3D013B012B40F2E2
:10F26000C280D4F89C3D834E012203F2DC53C4F8E3
:10F270009C3D84F8602E0325FFF722FF70B13378A0
:10F28000B12B0BD1FEF702F9013D00F0D18000282F
:10F2900040F0D180FFF714FF0028F0D1013DEBD101
:10F2A000754E764C764DDFF8DC910A273221052029
:10F2B000FCF7C0F94FF4FA7A7368C3F30803002B24
:10F2C00040F0A980EFF31183002B40F0A4804FF0B1
:10F2D000E0202368816922689342FAD12A6891422A
:10F2E000F7D8D9F800004FF47A7202FB00F8A8EBC7
:10F2F0000108B8FBF0F802FB03887368C3F3080346
:10F30000002B40F09180EFF31183002B40F08C80B4
:10F310004FF0E0202268816923689A42FAD12B6875
:10F320009942F7D8D9F800C04FF47A7000FB0CF37B
:10F330005B1AB3FBFCF300FB0233A3EB0803B3F54A
:10F340007A7FDAD3BAF1010AB6D1FA210620FCF7A6
:10F3500071F94FF47A7A7368C3F30803002B4ED126
:10F36000EFF31183002B4AD14FF0E020236881692D
:10F3700022689342FAD12A689142F7D8D9F800005E
:10F380004FF47A7202FB00F8A8EB0108B8FBF0F822
:10F3900002FB03887368C3F30803C3BBEFF3118355
:10F3A000ABBB4FF0E0202268816923689A42FAD112
:10F3B0002B689942F7D8D9F800C04FF47A7000FB57
:10F3C0000CF35B1AB3FBFCF300FB0233A3EB080363
:10F3D000B3F57A7FDED3BAF1010ABCD1013F7FF4E5
:10F3E00065AF38F039FDFBF79DFB00F5B71000F570
:10F3F00058700222C4F8880D84F88C2D31E7FBF791
:10F4000065FB7368C3F308038046002BC6D0FBF787
:10F410005DFB0346DAE7FBF759FB7368C3F30803A8
:10F420008046002B3FF46FAFFBF750FB034684E7A9
:10F4300000283FF435AF94F86C3D013B0022012BCE
:10F4400084F8602E0BD90D4B0122196884F8B52D74
:10F450000023C4F89C1D84F8613EBDE8F087FBF7EB
:10F4600061FB0223C4F8880D84F88C3DEBE700BFF4
:10F47000F86F00200040000800ED00E0642A002042
:10F4800054430020F037002010B50A4C012384F8C3
:10F49000143EA373FFF7DAFEFFF7B4FB41F202421A
:10F4A000FF23A4F8182E84F81A3EBDE810400E2061
:10F4B0000AF096BEF86F002090F89230DFED6B6A8C
:10F4C0006B4A07EE903A90F8963005EE103A90F8B5
:10F4D000943004EE903A90F8953005EE903A90F81A
:10F4E0009830F8EEE77AB8EEC55A04EE103A67EEB7
:10F4F000A67A25EE265AF8EEE44AF8EEE55AB8EE7A
:10F50000C44A25EE275A64EEA64A65EEA65A24EEB2
:10F51000264AF0B5B7EE007A90F8917064EE854A0D
:10F5200065EEA75A24EE274A00F16F06014602F164
:10F530001A050024B0EE476AB0EE473A137807EE9A
:10F54000903AF8EEE77A67EE857A67EE867AFDEE16
:10F55000E77A17EE903AFA2BA8BFFA2323EAE3736F
:10F560000B72537807EE903AF8EEE77A67EEA47ADA
:10F5700067EE867AFDEEE77A17EE903AFA2BA8BF8F
:10F58000FA2323EAE3734B72937803EE903AF8EE92
:10F59000E33A63EEA57A67EE877AFDEEE77A17EE37
:10F5A000903AFA2BA8BFFA2323EAE3738B7293886D
:10F5B00007EE903AF8EEE77A67EE847A67EE867A9D
:10F5C000FDEEE77A17EE903AB3F57A7FA8BF4FF4D5
:10F5D0007A7323EAE3738B812B68D5ED007A002BD5
:10F5E000F8EEE77A3FDD90F8973002EE903AF8EEC9
:10F5F000E22AB0EE436AA2EEE66A63EE863A83EE52
:10F60000A76AA2EEA66A013465EEA77A67EE877A4A
:10F6100067EE867AFDEEE77A17EE903AFA2BA8BFEE
:10F62000FA2323EAE373BC4206F8013F00DDF0BD94
:10F63000012C13D190F8933007EE103A90F89B30DC
:10F6400006EE103AB8EEC77AB8EEC66A27EE267A0A
:10F6500026EE266A0435083208316FE7B7EE007AE5
:10F66000B0EE476AF6E7B7EE006ACCE70AD7233C6C
:10F67000A60E050890F899306BB3B0F864308BB1E2
:10F6800090F89A2002EB82036421C3EB0313B3FBCF
:10F69000F1F3A0F86430962312FB03F3B3FBF1F30C
:10F6A000A0F8663043884BB190F89A3003EB83039F
:10F6B000C3EB03136422B3FBF2F34380B0F8503082
:10F6C0004BB190F89A30962213FB02F36422B3FBFD
:10F6D000F2F3A0F85030704790F821304BB3438BD1
:10F6E00083B190F82230FA2213FB02F203EB83037A
:10F6F000B3F57A7FA8BF4FF47A7364218383B2FB9A
:10F70000F1F24283838843B190F82230FA2213FB4E
:10F7100002F36422B3FBF2F38380C3884BB190F809
:10F72000223003EB8303B3F57A7FA8BF4FF47A73DB
:10F73000C380704770B50B4C002504F56A7694F8C9
:10F74000913013B12046FFF7B7FE2046FFF792FF36
:10F7500001353046FFF7C0FF042D04F1EA04EED175
:10F7600070BD00BF3871002010B5064C4FF4807298
:10F77000002104F662603FF08BFF0023C4F8643F71
:10F7800010BD00BFF86F0020034BD3F8680F08B11D
:10F7900007F012BE704700BFF86F002008B50B4697
:10F7A00005490246D1F8680F28B10449FEF722F84E
:10F7B000BDE80840E8E708BDF86F0020E1D1000887
:10F7C000024B0146D3F8680FFDF70CBDF86F00201F
:10F7D0000048F5E7ECE905080CB4C30607B500D509
:10F7E00061B9049805A90191FFF7D8FFFFF7F0FF71
:10F7F000012003B05DF804EB02B070470020F8E789
:10F8000008B5FFF7DDFFBDE80840E1E710B50446A5
:10F810000348FFF7D5FF2046BDE81040F0E700BFE2
:10F82000AEDE050810B508460749FDF7DFFA0028E7
:10F8300015BF0124002405480548FFF7E7FF2046CF
:10F84000BDE810400AF0C4BBB3DE0508BCDE050805
:10F85000E3DE0508034B0146D3F8680F08B107F053
:10F8600095BD7047F86F00200CB407B510F020006C
:10F870000BD079B92320FFF7EDFF049805A901917A
:10F88000FFF78CFFFFF7A4FF012003B05DF804EB46
:10F8900002B070470020F8E70FB407B504A951F88B
:10F8A000040B0191FFF77AFF03B05DF804EB04B09D
:10F8B0007047194B1B682DE9F0415BB31748184F8F
:10F8C000DFF86480FFF79CFFFFF75EFFFCF7A2FC08
:10F8D0000025FCF7D3FC044640B113200AF080FC5D
:10F8E000FFF776FFBDE8F0410E4889E73B78012B32
:10F8F000F3D04046FFF7D0FF792D05F1010602D184
:10F90000FFF766FF2646FFF73FFF6420FBF71EFE6A
:10F910003546DEE7BDE8F0811C2A0020FFDE050841
:10F920008E48002019DF0508BEF805080FB407B59A
:10F9300004A951F8040B0191FFF730FFFFF748FFCE
:10F9400003B05DF804EB04B070472DE9F041037992
:10F9500003F0E002402A4AD009D82ABB03F007038B
:10F96000052B1CD8DFE803F0161B161B090F602AB5
:10F9700044D0802A3ED0BDE8F081D0F8051021485F
:10F98000BDE8F041D2E7D0F8052051421E48BDE85D
:10F99000F041CBE7B0F80720B0F80510F6E7B0F972
:10F9A0000720B0F90510F1E74679184D184805EB26
:10F9B000C605FFF705FF95F8707200240123A742E2
:10F9C00002D8BDE8F04103E7D5F86C6256F8242070
:10F9D0004FEA84084AB113B90E48FFF7F1FE56F812
:10F9E00008100D48FFF758FF00230134E7E741797D
:10F9F0000A48C5E7827941790948C8E7BDE8F0417E
:10FA0000084893E71FDF050835DF0508600C050887
:10FA10004CDF05085DDF05082CF4050860DF0508EC
:10FA200071DF050888DF05082DE9F04385B0FCF794
:10FA3000E3FB02698389018802928268019242880D
:10FA4000009242681B4EDFF88080DFF880901A4FEA
:10FA500004461A48FFF76AFF002515B91848FFF752
:10FA6000CFFED8F800309D4213DA3378052B96BFCD
:10FA700009EB83030022D3F8DC23B3880093738857
:10FA8000294638460135FFF751FF062D06F10606D7
:10FA9000E3D138F057F94288838864689B1A03FBE6
:10FAA0000444FCF731FC02460648214605B0BDE897
:10FAB000F0433BE7647F00200AE00508A0DF05086B
:10FAC000FEDF050819E0050884480020600C0508E1
:10FAD0000249034801F5B2610EC927E70070FF1F14
:10FAE00036E0050870B5134C134D144E002294F8FF
:10FAF0000B3503F0010302B170BD002BFCD00121D6
:10FB00002846FFF713FF752025F05FFB01463046BE
:10FB1000FFF70CFF1A2025F058FB01460848FFF7B5
:10FB200005FF1B2025F051FB01460648FFF7FEFEAE
:10FB30000122DCE7F86F00204AE0050856E00508DE
:10FB400069E005087CE005082DE9F047BE4BBF4F92
:10FB50001A68BF49BF4BC048B2FBF3F296B0FFF73B
:10FB60009BFEBB6803F00303022B00F03181032BE3
:10FB70000CBF03250025B94BDFF88483DFF884939D
:10FB8000DFF864A30FCB0AAE86E80F00B44B0593F1
:10FB9000012DB44BC8BFFC68069316AB03EB85037D
:10FBA000C8BF04F00104012D53F8301CD8BFAE4A81
:10FBB000AE48AF4EC4BF16AB03EB84044FF0000752
:10FBC000C8BF54F8442CAB4CFFF766FEB4F8902F36
:10FBD0004FF47A73B2FBF3F103FB11220A20B4F95C
:10FBE000923F92B2B2FBF0F2A348FFF79FFEA34A06
:10FBF000A349A448FFF750FEFFF7EAFDA17BA24A04
:10FC0000A24BA34806EB8101D31AD1F80414B4F82F
:10FC10005220FFF78BFEFFF7DBFD9E48FFF7D0FD7C
:10FC200094F8941F9C48FFF737FE9C48FFF7C8FDE7
:10FC3000B4F8962F94F8981F994892B2FFF72CFECB
:10FC4000FFF7C6FD97499848FFF726FE3D4694F812
:10FC5000073503F00103002F00F0BC80002D40F0B9
:10FC6000EE809248FFF7CCFD914FD4F8A08FDFF8DB
:10FC70009892012507F1180A0123AB4013EA080FF7
:10FC800014D019F8052057F825305AF8251053F8E4
:10FC900022208848FFF700FE012D05D194F8C11FEE
:10FCA00011B18548FFF7F8FDFFF792FD0135062DEC
:10FCB000E2D1824D824815F8E43C55F8E87C06EB29
:10FCC0008303D3F89C14FFF7E7FD27B13A7A797ADA
:10FCD0007C48FFF7E1FDFFF77BFDFCF78DFA01693A
:10FCE00021B182687848120DFFF720FEFFF770FD02
:10FCF000764B774819684FF47A73B1FBF3F1FFF74D
:10FD0000CBFD07A8FEF774FA38B107A90EA83DF09D
:10FD100085FB70480EA9FFF7BFFDFFF759FD55F8A9
:10FD2000588CB8F1000F00F08D8007EE908ADFED5F
:10FD30006A6AB8EEE77AC6EE877AFDEEE77A17EEE2
:10FD4000903A95F8600530B1644A039392ED0D0A3C
:10FD50003EF076FF039B55F8D87C5FB107EE907AB2
:10FD6000DFED5D6AF8EEE77A86EEA77AFDEEC77AF8
:10FD700017EE907AB5F862156429A8BF6421CDE921
:10FD8000000742465648FFF7D1FDB5F864255548AF
:10FD90006423B2FBF3F103FB112295F8753506EBF2
:10FDA000830692B2D6F8B034009395F874354E4E6F
:10FDB000FFF7BCFD4D48FFF703FDD4F85C4E01256D
:10FDC000002C40F0A380FFF703FD16B0BDE8F087DC
:10FDD0000125D0E6002B3FF441AF15B14046FFF7B7
:10FDE000EFFC01214846FFF757FD94F89C3F06EBD6
:10FDF00083035046D3F80C14FFF74EFD94F8BA383D
:10FE0000DB0702D53A48FFF747FD94F80436032B89
:10FE100009D03848FFF740FD94F80436012B02D191
:10FE20003548FFF739FDD4F858355B7B0125AB42E7
:10FE30002F467FF60CAF3148FFF72EFD07E7FFF79F
:10FE4000C7FC11E743467CE7040000200010024095
:10FE50008FE0050840420F0099E00508541005089E
:10FE6000ABE00508B0E0050883FE0508B5E005082D
:10FE7000600C0508F86F0020BDE00508F0FF0120C8
:10FE800000080000DFE005080060000800400008EE
:10FE9000F1E0050808E105081AE1050822E1050876
:10FEA00024E1050838E105083DE105085CE10508A5
:10FEB000CC100508C8F6050861E10508F0800020AF
:10FEC00065E105086EE1050878E10508642A00206F
:10FED00093E10508ADE10508002474496804002099
:10FEE000C0E1050806E20508F7E505082BE205086C
:10FEF0001AF4050847E105084FE1050854E1050833
:10FF00005DDF050842E105089404002094FAA4F09E
:10FF1000B0FA80F005FA00F024EA000409F038FF96
:10FF200001463046FFF7B8FC4AE72DE9F04FDFF80D
:10FF3000788198F8033099B0002B00F098805148F0
:10FF4000514EDFF868B1DFF86891DFF868A1FFF77C
:10FF500057FC00252F460BA9E8B211F011FC9DF8C3
:10FF60003430002B53D0139C54B107EE904A9FEDD0
:10FF7000470AF8EE677A80EE270A3EF061FE0446F3
:10FF80000B9A29465846FFF787FC109A002A70D032
:10FF900002FB04F04FF47A73B0FBF3F30993DDF83E
:10FFA00048C0BCF1000F66D00CFB04F142F21073A4
:10FFB000B1FBF3F198F80330082D18BF7F18002B20
:10FFC0005BD01798079015980690169805900A230D
:10FFD00011984FF47A7EB0FBFEFE0998CDF810E040
:10FFE000B1FBF3FE03FB1E11CDE902E10999B1FB60
:10FFF000F3F103FB1100CDE90010BCFBF3F3214644
:020000040801F1
:100000005046FFF793FC0023C6E90D33B362013578
:10001000192D06F140069ED198F8033023B31C4CED
:100020001C48D4F87C25D4F87815D2084FF47A739C
:10003000B1FBF3F3D4F88015FFF778FC0A221648D9
:1000400097FBF2F102FB1172FFF770FC134B1B7868
:10005000432B06D1D4F88425D4F888151048FFF72F
:1000600065FC0023C4F8803519B0BDE8F08F0D4859
:1000700066E7099293E761469CE721464846FFF709
:1000800055FCC0E741E20508108000208096184B1F
:10009000F0800020E8E2050808E305084547002055
:1000A0002CE305089FE20508F86F0020A9E2050887
:1000B000C8F30508B8E2050870B5224C2248FFF7DE
:1000C0007FFB94F86035002B37D0204B93ED0D0A61
:1000D0003EF0B6FD01461E48FFF728FC1D4D1E48A8
:1000E000FFF76EFB1D4B95F819091D4A00280CBF40
:1000F00010461846FFF784FB95F819390BB3B4F88E
:100100001E161848184E194DFFF7C6FB94F81C062A
:1001100000280CBF30462846FFF772FBB4F82016C3
:100120001348FFF7B9FB94F81D0600280CBF3046B2
:100130002846BDE87040FFF763BB0E48FFF760FB41
:10014000CCE770BDF08000206AE305086804002059
:1001500084E30508F86F002093E305089DDF050898
:1001600056E30508A4E3050863E305085AE3050818
:10017000CBE3050889E305080EB403B503AA52F8DA
:10018000041B0192FDF7A4FD064BD3F8682F1AB9A2
:100190000549586DFDF726F802B05DF804EB03B091
:1001A000704700BFF86F0020ECE905082DE9F04723
:1001B00098460B7903F0E005402D81460F46164620
:1001C00032D1644DDFF8A881DFF8B091002416E049
:1001D0003B7903F00703013B042B04D8DFE803F06D
:1001E00014171A1D2100315D5A48FFF755FB7B7922
:1001F000013BA34202DD4846FFF7E2FA01347B7976
:10020000A342E5DCBDE8F08731572846EDE736F834
:100210001410FAE736F91410F7E756F824104046A0
:10022000E3E756F82410F0E703F00703052B57D84F
:10023000DFE803F0031F27292C3E3478602D55D0CA
:100240002CD8002D75D1B7F80550B7F80760414894
:100250002146FFF721FBAC4239DBB44237DCB8F171
:10026000000FCFD0324629463B48BDE8F047FFF7A4
:1002700013BB96F90040602D38D00FD8002D58D10F
:1002800051E03488DAE7B6F90040F4E7D6F800A088
:10029000202D54464DD034D9602D27D0802DB1D19A
:1002A00032782E4B2E48002A14BF3146194635E0CD
:1002B000202D34683DD0EFD821462648FFF7ECFAD0
:1002C000D7F80510A14202DB4B42A34221DDFFF724
:1002D0007FFA3A68234923464846BDE8F0474BE792
:1002E000202D25D01ED9602DD8D100247B7944FA49
:1002F00003F3DB07BDE8F0474CBF1B481B48FFF783
:10030000CBBA51461A48FFF7C7FAD7F805108A4505
:10031000DDD8B8F1000F3FF475AF1648BDE8F047DF
:10032000FFF7BABA0024B7F90550B7F907608EE7AE
:1003300000247A79104B03EBC20393F87022A24297
:10034000C5DDD3F86C3253F82400BDE8F047FFF761
:1003500037BA00BF49DF05081EED050897F9050803
:100360002CF40508F1E305089DDF050856E30508B0
:1003700032DF0508EBE30508600C050822E10508FB
:1003800070B50546084616460C46FCF73BFF33465B
:10039000024621462846BDE8704007E70EB403B583
:1003A00003AA52F8041B0192FDF792FC044B054985
:1003B000586DFCF717FF02B05DF804EB03B070470F
:1003C000F86F0020ECE905080049E7E70BE40508B1
:1003D000F8B5064608460C46FDF73EFE20210546C8
:1003E00020463FF06CF9044618B93046BDE8F840A5
:1003F000EAE7124F124E3B7832789A4204F1010438
:1004000001D0FCF765F80F4B20461D603DF0B6FCAF
:10041000012201462046FCF703F83B7832789A42E5
:1004200001D0FCF755F820463DF0A8FC2A460146CD
:10043000BDE8F8400448FFF779BA00BF182A002049
:100440008F480020142A002022E405082DE9F041FD
:10045000064688B008460D46FDF7FEFD20210446FD
:1004600028463FF02CF920B9304608B0BDE8F041ED
:10047000AAE7FDF7F1FD2246054601460F48FFF7C2
:1004800055FA85B1202D2A46694628BF20222046EC
:10049000FCF760F8E84606460027B74208DBAD1BCC
:1004A0003444002EEDD1FFF793F908B0BDE8F08198
:1004B00018F8010BFFF7CEF90137EEE738E405082D
:1004C00010B504460748FFF79BF9FCF771F820B117
:1004D000BDE810400448FFF793B920460349BDE842
:1004E00010405BE750E405085AE4050862E405089B
:1004F0002DE9F041144BD3F82C3688B00446F3B103
:100500001A6804A9D56A18466A46A847064688B1FB
:10051000DFF8408004AC6D46002735F8022B34F834
:10052000021B40460137FFF701FABE42F5DC08B076
:10053000BDE8F08105492046FFF730FFF7E70449A1
:1005400008B0BDE8F04129E7F080002083E4050809
:100550009BE4050869E4050870B5054608460C46A5
:100560003DF00CFC024668B1132804D1084821462E
:100570003FF07AF930B12846054B064A0649BDE8F6
:1005800070400BE7BDE8704001490448FFF7CEB961
:10059000A2E40508B6E40508C1E40508EBE4050893
:1005A00070B5054608460C463DF0E8FB024668B1CA
:1005B000042804D1084821463FF056F930B12846B6
:1005C000054B064A0649BDE87040E7E6BDE87040C5
:1005D00001490448FFF7AAB9F9E40508FEE4050853
:1005E000C1E405080EE505082DE9F04307469BB078
:1005F00008460C463DF0C2FB20220646002101A819
:100600003FF046F82EB3402E07D03B4940233246F8
:1006100038461BB0BDE8F043C0E601AD04F1400828
:100620004FF000090222214668463FF02FF90023CF
:10063000102209A968468DF80290FDF793FC099BEA
:100640000DF10202934223D10234A04505F8010BBB
:10065000E8D109AC4122002120463FF019F8274D8E
:10066000002E3CD095F83066D6B1202205F23161DB
:1006700001A83FF05DF998B105F231612046FDF720
:10068000B9FB1F4A1F4923463846FFF787FE04E09F
:100690001A781D493846FFF781FE1BB0BDE8F0838C
:1006A0001A4B93F83030D3B9CEB9194E01AB1A4674
:1006B00003CAA24230607160134606F10806F6D103
:1006C00001232046124985F85136FDF793FB114866
:1006D000FFF79CF810482146FFF728F9DDE795F869
:1006E00051361BB995F83036002BF3D00849204617
:1006F000FDF780FBEEE700BF21E50508F080002054
:100700005FE50508C1E4050843E50508F86F00202A
:100710002187002069E5050878E505082DE9F74FF0
:10072000834608460C463DF029FBDFF81881064653
:10073000D8F8847928B1024633492046FDF7D6FB24
:1007400080B93946314836F0F9FA3149314821EA61
:10075000070136F0F3FA3049304803B0BDE8F04FF6
:1007600036F0ECBA23782D2B2D4B03BF013406F164
:10077000FF364FF0010A4FF0000A4FF000094FF02A
:10078000FF3553F8041B51B1324620460193FDF763
:10079000ADFB019B00280ABF4D460021012109F154
:1007A000010989B9B9F11D0FEBD11E4922465846FE
:1007B00003B0BDE8F04FF1E53B43C8F884391A496E
:1007C0001A4B12E01A4913E0114A0123AB401A40B8
:1007D000002AF7D007EA0302BAF1000FECD027EAAB
:1007E0000303C8F884391349134B002A18BF19466C
:1007F000124B134803EB8503D3F8C42403B0BDE8C0
:10080000F04FFFF793B800BFA4E20508B0E5050874
:100810003DD45418BAE50508C22BABE7C6E5050878
:1008200024110508D4E50508A8E50508A1E5050893
:1008300085E5050891E5050898E50508600C0508BB
:1008400091EC0508F86F00202DE9F74F019008465C
:100850000E46174698463DF091FA0446E8B93F48DF
:100860003F4DFFF719F8204609F0ACFA3B681842F3
:1008700006D0204609F0B8FA01462846FFF70CF8E2
:100880000134172CEFD13B6813B93648FEF798FFB7
:1008900003B0BDE8F04FFEF79BBF02463249304639
:1008A000FDF724FB0546A8B93048FEF789FF2C4622
:1008B0002F4D204609F086FA10EA080F06D0204690
:1008C00009F092FA01462846FEF7E6FF0134182C9B
:1008D000EFD1DDE733782D2B03BF013604F1FF3470
:1008E000012500254FF0000948F4000B484609F0A7
:1008F0007BFA2246824601463046FDF7F7FA00BBF6
:10090000484609F05FFA1BEA000F1AD08DB1B9F121
:10091000170F1CBF3B6840EA03081648C7F8008061
:10092000FEF74EFF1248514603B0BDE8F04FFEF708
:10093000FDBFB9F1170F1CBF3D6885433D600E48F0
:10094000EEE709F10109B9F1180FCFD10B49019870
:10095000324603B0BDE8F04F20E500BFE5E50508ED
:10096000F6E50508EFE50508A4E20508FBE505083E
:10097000F7E5050898E50508A8E50508D4E50508A4
:10098000014A40F202235FE7687A0020014B024AE5
:100990005AE700BFFFFF7F00607A002010B50446D1
:1009A000012020F079FC20B920460449BDE8104020
:1009B000F4E4BDE810400248FEF7B8BF06E60508BB
:1009C00015E6050870B5054608461646FDF744FBD2
:1009D0000D4B041E93F8742A0EDB944205DA0B4883
:1009E0002146FEF7A3FF204670BD2EB1FF2C03D198
:1009F0000748FEF79BFFF6E70649013A2846FFF74E
:100A0000CDFC4FF0FF34EEE7F86F002020E605083C
:100A100031E6050844E605082DE9F04F074691B098
:100A20008248834D0E46FEF781FF8249C5F854D6B1
:100A3000002385F858360622012391F8741A3046AF
:100A4000402485F8594606F06FFC0A20FAF77EFD2F
:100A500095F858360C2BDAB240F2E4809DF80C6021
:100A6000FE2E2CD0FF2E15BF0F24152400250125A6
:100A7000944240F0D780611EC9B268462EF00AFA4F
:100A800004F140030DEB030414F8413C834240F0B1
:100A9000C4806A1E012A9DF80D3012D903F01F0789
:100AA00061375C096448FEF78BFE022D39D0013CAA
:100AB000042C34D8DFE804F00B2D2F33310002254D
:100AC000D6E79DF80E709DF80F401E46EAE75B489A
:100AD000DFF8C091DFF8C0A1DFF8C0B1FEF790FEEB
:100AE0005748FEF76DFE6C464FF0000814F8011BE6
:100AF000484608F10108FEF7CFFEB8F10C0F16D0FA
:100B00000AFB08F3B3F1553FF0D85846FEF758FEFC
:100B1000ECE74C48DCE74C48DAE74C48D8E74C486F
:100B2000D6E700238DF83F300DF11F00D0E7FEF728
:100B30004FFE022D3AD06422B6FBF2F102FB1162A5
:100B40003B464448D2B2C9B2FEF7F0FE85F001033D
:100B50005B42DBB2012B59D83F4A404B9DF8101045
:100B60003F48404E00290CBF11461946FEF7DEFEF5
:100B70009DF811103C4B3D4800290CBF31461946E9
:100B8000FEF7D4FE022D41D19DF812403848FEF701
:100B900017FE8CB1FF2C1FD00A23B4FBF3F103FB2B
:100BA00011423448D2B2FEF7C1FE08E032483A465C
:100BB0003146FEF7BBFECFE73046FEF721FE9DF83B
:100BC00013402E48FEF7FCFD44B1FF2C21D02C48E9
:100BD0002146FEF7ABFE04E02A48EEE72148FEF787
:100BE0000FFE204E204FDFF89C800DF113050024EE
:100BF00015F8013F7BB1FF2B14BF3A464246214610
:100C000021480134FEF792FE042CF1D111B0BDE869
:100C1000F08F1C48E3E73246F1E71C493846FFF7FE
:100C2000BDFBF3E71A48FEF7EBFDEFE78AE60508A0
:100C3000F0800020F86F00209BE60508A6E6050876
:100C4000D4E60508ADE60508B5E60508BDE60508E5
:100C5000CCE60508E6E6050873E605086AE6050839
:100C60001DE705087AE6050887F5050834E7050855
:100C70003BE705084FE7050802E7050857E70508C1
:100C800049DF05087EE6050867E7050872E70508FD
:100C900082E70508A9DE0508ABAAAAAA97F9050804
:100CA0002DE9F843DFF8A89007460C4620463DF0B2
:100CB00065F8064660B91E4B1E4893F8F0281E4B97
:100CC00003EB8203D3F83415BDE8F843FEF72EBEDC
:100CD000024649462046FDF709F960B1DFF8648015
:100CE000002558F8041BB1B9224638461349BDE81F
:100CF000F843FFF753BB1248124C134DFEF760FD4B
:100D000054F8041B19B12846FEF7C6FDF8E7BDE804
:100D1000F843FEF75DBD32462046FDF7E7F80135A2
:100D20000028DED1024B094C83F8F058BEE700BF23
:100D3000F86F00208BE70508600C0508D4E505086E
:100D4000FBE5050898110508F7E5050883FE050889
:100D5000A4E2050838B50D4604461A49052228467E
:100D6000FDF7C4F868B9184B93F8582022B901214F
:100D700083F8581083F85920BDE838401348FEF72F
:100D80003FBD134903222846FDF7B0F8A0B90E4D28
:100D900095F8583063B195F859304BB10D4920465C
:100DA000FFF7FCFA002385F8583085F8593038BD34
:100DB0000948FEF725FDF5E720460849BDE838401B
:100DC000FFF7ECBADEF40508F86F002095E7050898
:100DD00025F60508ABE70508E2E70508F6E705088C
:100DE00070B5184C94F8583005467BB194F85930DA
:100DF00063B11549FFF7D2FA28461449FFF7CEFA36
:100E0000002084F8580084F8590070BD104B93F806
:100E10005126AAB193F8302692B903F2316203F257
:100E20005C6503F25166106851682C4603C40832B1
:100E3000B2422546F7D1012283F8972608F03CFDFF
:100E40000120E2E7F86F0020ABE7050805E8050898
:100E5000F080002008B5034610460AB9002008BDFE
:100E6000DB0601D50029FAD0FEF7D0FCF6E7F8B58D
:100E70000D4E96F83030054693B9F8BD25B123885C
:100E8000C3F30B039D4204D0D4E90201A2883EF0D3
:100E9000DDFC1C34BC42F1D3002386F83030ECE793
:100EA000024C034FF6E700BFF86F002094FE0508E0
:100EB0001C0706082DE9F04F164685B0CDE9010163
:100EC0001A4600213046FFF7C5FF314C009006F06E
:100ED00010034FF00009A2460393FEF755FC237957
:100EE000029A03F01803934203D0002A44D1182B2E
:100EF00042D14FF00D0B0BFB09A3B3F8090034F0FE
:100F000031F980462046FCF790F8D8E902210746DF
:100F1000024401442046FCF741F880F00101009AA8
:100F20000546C9B23046FFF795FF039B009003B119
:100F300015BB0BFB09FBB3065AF80BB00ED56DB908
:100F400014485946FEF7A8FCD8F8082001982B460B
:100F50003A442146FFF72AF9FEF73AFC0E48594673
:100F6000FEF79AFCD8F80C20019800233A44214659
:100F7000FFF71CF9FEF72CFC09F1010940F22D23C3
:100F8000994504F10D04A8D105B0BDE8F08F00BF6C
:100F9000BC23050823E8050824E805080149FFF7F4
:100FA000FDB900BF2EE8050838B50C4605461549C1
:100FB0002046FBF71BFF30B9FEF7BCFB1248BDE82B
:100FC0003840FEF71DBC11492046FBF70FFFA0B9C2
:100FD0000F4B83F8D10183F8D90183F8BB0283F862
:100FE000C30283F8A50383F8AD0383F88F0483F865
:100FF000970483F809050748E1E72846BDE838402B
:10100000CCE700BF3DE8050843E805085EE80508B1
:10101000F86F002066E805082DE9FF4707460846F7
:101020000D463CF0ABFE082845D105F1FF3801AE76
:10103000073531464246B14612F8010FFCF750FF22
:10104000AA4201F8010BF7D10023DFF880A08DF848
:101050000C30A84517D11C49484620F0ADF81A4875
:101060001A49082310F8012B11F8014B10326A4479
:10107000013B02F80C4CF5D115488DF80C3001A954
:10108000FEF754FC14E018F8010FFCF729FF06F8EE
:10109000010B0446014650463EF011FB28B12146A3
:1010A00030463EF00CFB0028D3D03846FFF776FFE1
:1010B00004B0BDE8F0870028D1D0384604B0BDE8C0
:1010C000F047FFF781B900BFF0780020508705088E
:1010D00082E8050807B5009313460A460249FFF760
:1010E0005DF903B05DF804FB89E8050820B10078DC
:1010F000B0FA80F040097047012070472DE9F74FA2
:1011000081460846FFF7F2FF0E46054670B10024FF
:1011100001A9204635F052FE013401464846FFF74A
:10112000EDFF122CF4D103B0BDE8F08F0846FCF7B8
:1011300093FFC4B2112C70D8701C3C4D3C4EFCF790
:10114000BAF805EB4408670098F898A68346B8B942
:10115000AAF102014B424B413D4495F89826B25CFE
:10116000002B53D095F89936192040F2EE2100FB60
:1011700003133048214603B0BDE8F04FFEF7D6BB5D
:10118000017830463EF09BFA78B1032C94BF0022E0
:101190000122294902EB4202831B0A4452FA83F3DB
:1011A00093F8A8A5BAF1030F04D1484603B0BDE8EF
:1011B000F04FF3E65846FCF77EF8F0B1BAF1020FB3
:1011C000F3D1FCF749FF40F6CA0380B29842A8BFAA
:1011D000184640F2EE239842B8BF1846A0F2EE201F
:1011E0001923B0FBF3F088F89906AAF102025342E2
:1011F0005341EA1982F898A6AEE7BAF1020FF4D18A
:10120000484603B0BDE8F04FFFF7DEB80B48214673
:1012100003B0BDE8F04FFEF789BB094911232A4608
:10122000484603B0BDE8F04F54E700BFF08000200F
:1012300060890508A2E80508600C0508B2E8050801
:10124000BFE805082DE9F04F0346A1B00846FFF7B7
:101250004DFF054628B1184621B0BDE8F04FFFF715
:10126000B3B8DFF8C4920B90FF238DF82830D9F87B
:10127000BC36ADF83000CDE9050093F838200D906C
:101280008DF838200F90ADF8400011930991074672
:101290004FF0FF38934909A83EF0AAF9044618BB5D
:1012A000914F01460AAC0B0190481A57002310F9E0
:1012B000016BB24240F0D28010464E1C35F068FD02
:1012C000314602463846FEF731FB022E4FF001014F
:1012D000E9D19DF938A09DF92830534540F0C580EB
:1012E0008348FEF723FB4DE02378002BD2D0032F59
:1012F000D4BF00260126062F00F2A980DFE807F000
:101300000447509104475000042F10D079492046DB
:10131000FCF710FE58B14FF4806008F0E5FD00289E
:1013200000F0B48190F90400012306930AE07249A9
:101330002046FBF75BFD70B9D9F8BC3693F938004D
:10134000042F22D0119B119320AB03EB061606F855
:10135000580C01379EE7204635F06EFC0028EFDA86
:1013600001230A2212A92046FCF7FCFD40B2002806
:1013700003DB129B1B78002BE2D060482246711CD5
:10138000FEF7D4FA21B0BDE8F08F0023DBE720465A
:10139000FCF762FE20AB03EB061646F8540CD8E7C8
:1013A00057492046FCF7C6FD5649B0F1000A2046D1
:1013B00018BF4FF0010AFCF7BDFD08B14AF0020A60
:1013C0003301DFF868C1079320AB03EB0616BCE8D6
:1013D0000F0006F850AC12AE0FC6BCE80F000FC6E7
:1013E000BCE80F000FC69CE8030086E80300002657
:1013F0000DF1480AB346DAF8001020463EF082FAB2
:1014000010B19AF804301E430BF1010BBBF1070F2A
:101410000AF1080AEFD1079B80336B4403F84F6C45
:1014200097E739492046FBF7E1FCA0B13749204650
:10143000FBF7DCFC00288CD02046FCF70DFE0328CF
:10144000804686D901463248FEF770FA9AE731485D
:101450002246082194E7012305937AE70133072BFD
:101460007FF425AF2C4801318AE70B9B1BB9AAF109
:1014700014025542554100235F1CE368002B62D1E2
:1014800094F900B0584608F0FFFCD4F8049018B165
:101490000668002E40F08A80B9F1000F237A14BF4D
:1014A0004E464FF46146666023B91C48FEF73EFA8B
:1014B00003232372627A2AB1194807923946FEF74C
:1014C00035FA079A0292237ACDE9006300231A467F
:1014D0001946584608F0B3FDE06048BB114839464C
:1014E000B2E700BF36ED050849E9050848120508CE
:1014F00066E90508E2E80508EDE80508F1E80508F1
:101500000CE90508A9F505080FE90508F1E5050846
:1015100015E905082DE9050854E905087FE90508DE
:101520009AE90508B5E90508F080002010120508C1
:101530005849594A5948B9F1000F18BF0A4633466D
:101540003946FEF7A9F9022F04F110044FF0010308
:1015500092D1119E0D9F4DB15148FEF751F933685C
:101560001B6A1BB14F493A4630469847059B002BF2
:101570004FD04D49474BBAF1140F18BF19464B488D
:10158000FEF7D4F9BAF1140F09D1059B002B42D014
:101590003368DB691BB14649002230469847069BF9
:1015A000002B42D13146384635F05EFBE660B9F19A
:1015B000000F2CD04946304603F018F93D4AB36875
:1015C0003D483946FEF7B2F994F80890B9F1000F9A
:1015D0000CD03279914509D038484B463946FEF750
:1015E000A5F9336849469B6930469847637A23B129
:1015F000727933483946FEF799F9F36A002BA2D085
:1016000030483946FEF792F90023F3629BE7214AFE
:10161000D5E72049B3E7B8F1000FC0DB3368DB69D9
:10162000002BBCD028494246B7E706F0ADF80520AC
:10163000F9F78CFFDFF89490DFF894A000254FF0C5
:10164000030B9AF8743AAB42ACD919F8014FC4B104
:10165000204607F0EDF9804698B12046F7F752F89A
:10166000EBB2044610B180F806B0C37120460121E8
:10167000F6F744FD98F80630DB07204603D5F6F769
:10168000CBF90135DDE7F6F7C1F9FAE74FF0FF30A6
:101690004AE600BF83FE0508C7E80508D1E905084A
:1016A00087EA0508ED470108D5E80508B0EA05080E
:1016B000D1D20008D0E80508EFE9050814EA0508CA
:1016C00037EA05086EEA050891D000083B3B002088
:1016D000F86F00202DE9F74F05460846FFF706FD95
:1016E0000B46044618B9324A92F8C07627B9284604
:1016F00003B0BDE8F04F51E42E49DFF8C090DFF8A9
:10170000C080DFF8C0A001AA18463DF09EFF264623
:1017100010B906F045F808E056B9012201462846FE
:10172000FFF750F9421C04461AD103B0BDE8F08F10
:10173000FCF792FC2F28834634D80FB106F024F82A
:10174000BBF1060F13D098F8741A01235FFA8BF2DD
:10175000E0B205F0E9FD59465046FEF7E7F80027EC
:10176000144901AA002001363DF06FFFD0E7D8F8F8
:1017700088391B0112D5FF2C0ED0E1B22846FFF7A5
:101780004BF9E8E72846FFF747F9013798F8743A2C
:10179000F9B28B42F6D8DEE70027F7E70648FEF7F6
:1017A0002FF8D8E72F2249462846FEF7F7FDD7E75E
:1017B000F080002036ED050806E60508E4EA050895
:1017C000F86F0020D3EA05082DE9F74307460846DD
:1017D000FFF78CFC0B46044628B1384603B0BDE841
:1017E000F043FEF7F1BD2F49DFF8B89001AA184683
:1017F0003DF02BFF26460546A04665B92A4B3246EA
:10180000D3F8BC06A1B239F0F5FA68BB27493846CF
:10181000FEF7C4FD28E0B8F1000F06D0B8F1010FC3
:1018200025D03846FEF7D0FD1EE028463CF0A6FA4B
:101830001F49064602462846FCF758FB50B31D498F
:1018400032462846FCF752FB30B31B493246284645
:10185000FCF74CFB10B3194932462846FCF746FB0F
:10186000F0B13846FFF79AFB03B0BDE8F083B31E32
:101870005A425A4129463846FFF7A4F8421C04460A
:10188000F2D001AA494600203DF0DFFE08F1010830
:101890000546B2E74646F4E70126F2E70226F0E7FE
:1018A0000426EEE736ED0508F080002010EB050871
:1018B00004EB050807EB05080AEB05080DEB050826
:1018C0002DE9F74380460846FFF710FC0B46054616
:1018D00028B14046FEF778FD03B0BDE8F0832F49FC
:1018E000DFF8B89001AA18463DF0AFFE2F46044637
:1018F0002E467CB9022DECD1A7F57A73B3F57A7F29
:1019000021D927494FF4FA634FF47A724046FFF722
:10191000E1FBE1E74DB1012D10D001AA49460020BD
:101920003DF093FE01350446E3E70122214640469F
:10193000FFF748F8431C0646EFD1CDE72046FCF7F9
:101940008BFB0746E9E7174DD5F8C436B8B25B689C
:101950009847FF2EBCEEC00A05F5DA650CD1124B94
:10196000F8EE407A93F8743AA34212DC10EE101AA3
:101970000E48FDF7DBFFAFE7F8EE407A05EB860592
:1019800010EE102A0A48C5ED007A3146FDF7CEFF69
:10199000A2E7E5EC017A0134E6E700BF36ED050881
:1019A0001EEC0508F0800020F86F00203BEB0508D6
:1019B0002EEB0508F8B507460846FFF797FBC8B1B8
:1019C0001F4B9E6B0136304608F00EFA3446054632
:1019D000F0B90134182CA8BF0024204608F004FAFE
:1019E0000546A8B9B442F4D138461649BDE8F840D6
:1019F000FEF7D4BC0846FCF72FFB044608F0F4F9C8
:101A0000054628B921461048BDE8F840FDF78EBFCD
:101A10000B4B9C6308F0AEFB0C482A462146FDF7B1
:101A200085FF172C09D80A4B0C2202FB043393F8CC
:101A3000F005BDE8F84008F0D3BB0020F9E700BF8F
:101A4000680400204AEB05085EEB050874EB050806
:101A5000600C050838B5124D04460846FFF746FBF2
:101A600060B1104B104893F900104B1C0ABF0F4B8C
:101A7000C9B21978BDE83840FDF758BF0846FCF7F1
:101A8000EBFA032804D8C0B2FDF72EFA2946E4E7A2
:101A900020460749BDE838400322FEF77FBC00BF5F
:101AA00083FE0508680400208DEB0508F86F002010
:101AB0009DEB050838B5124D04460846FFF716FBA6
:101AC00060B1104B104893F901104B1C0ABF0F4B2B
:101AD000C9B25978BDE83840FDF728BF0846FCF781
:101AE000BBFA032804D8C0B210F0CCFD2946E4E7C5
:101AF00020460749BDE838400322FEF74FBC00BF2F
:101B000083FE05086804002089EB0508F86F0020B3
:101B100098EB05082DE9F74F444BDFF828911A7828
:101B200089F800205A7893F830300091054689F8FA
:101B300001200BB904F040FE33F04EFB00263C4C74
:101B4000B0460D233A4A0099734352F803A0504619
:101B5000FCF7F0F9002841D0B8F1000F01DDFDF7E6
:101B600037FE34485146FDF797FE002221462846AD
:101B7000FEF706FCFDF72CFE237903F01803082B73
:101B800046D0102B49D02046FDF7DFFE284B0D2212
:101B900002FB0633B3F8090033F0E4FA8346D8B108
:101BA0002046FBF742FADBE90221074602440144E2
:101BB0002046FBF7F3F978B9019051461E48FDF72E
:101BC0006BFEDBF80810019A28461346CA19214615
:101BD000FEF7ECFAFDF7FCFD08F10108013640F2D2
:101BE0002D239E4204F10D04ABD10020FFF73FF9F5
:101BF000FF2389F8003089F80130B8F1000F11D1C6
:101C0000009A0E49284603B0BDE8F04FFEF7C6BB68
:101C10000B492846FFF71EFFB5E709492846FFF79D
:101C200049FFB0E703B0BDE8F08F00BFF86F0020B8
:101C3000BC23050828E80508B8EB0508D4E5050825
:101C400083FE0508680400202DE9F74F804608460A
:101C50000F463CF093F8044620B1012825D13B788B
:101C60002A2B22D1A948AA4EAA4FFDF7C9FD00256B
:101C7000B1464FF00D0A04F001040AFB05F33846A3
:101C800059F80310FDF708FE314622464046FEF79C
:101C900077FB0135FDF79CFD40F22D239D4206F1B7
:101CA0000D06EAD103B0BDE8F08F3D2138463DF086
:101CB00006FD002800F0238103469A4613F8012D03
:101CC000202AFAD0AAEB070A0130054610F8013B9A
:101CD000202BFAD0DFF838B25FFA8AFA4FF0000909
:101CE0000D2303FB09F352465BF8031000913846BD
:101CF0000BEB0304FCF7FAF8064670BB00990846A4
:101D00003CF03CF8824528D1277907F0E0014029D2
:101D100000F0898012D871B366797F4A02EBC6065B
:101D2000002796F870220092BA463B46009ABA42C3
:101D300002D9BAF1000F62D02BB12DE06029ECD0AE
:101D4000802900F0A48040467449FEF727FB204616
:101D500003B0BDE8F04FFDF7F8BD09F1010940F20D
:101D60002D239945BCD16E493A46404603B0BDE8A3
:101D7000F04FFEF713BB07F00703042B1CD10B46F3
:101D80000A222846FCF7EEF8D4F8053083420146D3
:101D9000D9D32046FBF74CFA0D2303FB09F9614820
:101DA0005BF80910FDF778FD00222146404603B09C
:101DB000BDE8F04FFEF7E4BA052B0DD101230A224E
:101DC0002846FCF7CFF8D4F8053083420146BADB49
:101DD0005B428342B7DCDCE72846FCF73DF917F0AD
:101DE000050F0BBFB4F80520B4F90520B4F807308F
:101DF000B4F9073090420146A5DB9842EAE7D6F8ED
:101E00006C1251F8270060B129460193FAF7EEFFF2
:101E1000019B30B9394620464FF0010AFBF708FA1A
:101E20005346013782E76379009307F00707013FC4
:101E3000009BB342B0DDAA4615F8013B202BFAD037
:101E40002046FBF7DFF90546042F04D8DFE807F04A
:101E5000030E0E141D005046FCF7FEF8A8552C2169
:101E600050463DF02CFC0136451CE1E75046FCF79E
:101E7000F3F825F81600F2E700230A220021504665
:101E8000FCF770F845F82600E9E70123F5E7284656
:101E90003BF074FFE37994F805A0A779DB070646C9
:101EA0000AD52046FBF7AEF90378014623B1324646
:101EB00028463DF0D9FCE0B9DEB1B74219D320463F
:101EC000FBF7A0F93A4600213DF0E2FBB2453FF6B0
:101ED00063AF1549324628463DF0C6FC00283FF462
:101EE0005BAF2046FBF78EF9324629463DF0AEFC4B
:101EF00052E70E493A464046FEF750FA23E7394684
:101F0000404603B0BDE8F04F04E600BFC8EB05084B
:101F1000BC23050828E80508600C050816EC050830
:101F2000D4E505080BEC050897F90508DBEB050877
:101F30002DE9F04F914687B00C461A4600218046A5
:101F4000FEF788FF4D4606460027B9F1000F66D020
:101F50002946062220463DF0EBFC0028324614BFFD
:101F60000121002140460CBF4FF0010A4FF0000A4A
:101F7000FEF770FF064628780BF050F88346F8B15C
:101F800068790BF04BF8AB78EA789BF805E095F8A8
:101F900001B04FF461714FF0190C1CFB03131CFBD3
:101FA0000212297900B14079CDE90410CDE902325D
:101FB000CDE900EB1B4A3B4651464046FDF754FC39
:101FC00020780BF02BF88346F8B160790BF026F8F7
:101FD000A378E2789BF805E094F801B04FF46171C2
:101FE0004FF0190C1CFB03131CFB0212217900B1EA
:101FF0004079CDE90410CDE90232CDE900EB094A80
:102000003B4651464046FDF7E7FB0137142F04F1EC
:10201000060405F1060598D107B0BDE8F08FCA4661
:10202000CEE700BF24EC05082DE9F041054686B057
:102030000846FFF75BF80F46064638B100235C49B7
:102040001A46012006B0BDE8F04171E70846FCF7EA
:1020500003F81328044600F3A18006254543781CA5
:102060008DF81760FBF727F9524E074660B1FBF772
:10207000F3FFC0B20AF0E8FF30B17319027983F8B8
:10208000C82901238DF817303846FBF714F90746A5
:1020900068B1FBF7E1FF0D2809D8062303FB0463B1
:1020A00083F8C9099DF8173001338DF81730DFF830
:1020B0000081A91C0DF1170241443846FBF7D0FFFF
:1020C000FBF7F9F8074668B1FBF7C6FF012809D806
:1020D0009DF81730062202FB0462013382F8CC0916
:1020E0008DF817303846FBF7E6F880B1FBF7B4FF00
:1020F000C0B20AF0A9FF50B19DF81730017906224D
:1021000002FB0462013382F8CD198DF817309DF877
:102110001720042A4FF006032FD103FB046300228B
:10212000A3F8CC29062505FB04651CF0ADF895F84D
:10213000C8090AF073FF95F8CB1995F8CA791923E5
:102140004FF46172804695F8CD0913FB012613FB0D
:1021500007270AF063FF437998F80520039395F861
:10216000CC390097CDE90163134895F8C939214668
:10217000FDF7DCFB06B0BDE8F081052A05D103FBC5
:102180000463002283F8CD29CCE7062ACAD008EBE5
:102190000502002348F805309380C3E7074913235D
:1021A0003246284606B0BDE8F041FEF793BF00BFB7
:1021B000C0790020F86F002024EC05083DEC0508EC
:1021C0002DE9F04F904689B01A460C460021814611
:1021D000FEF740FE3B4EDFF8F0B008F1540307462F
:1021E0004546079394F9040007F04EFE00285DD0A1
:1021F000B8F1000F63D029460C2220463DF098FB31
:1022000000283A4614BF0121002148460CBF4FF078
:10221000010A4FF0000AFEF71DFE074695F904007B
:1022200034F0B6FDEA7906EB82020346D2F81027B5
:1022300004922A7A06EB82025146D2F810270392C2
:10224000AA7906EB82024846D2F8102702926A79F0
:1022500006EB8202D2F8102701922A6800925A46B1
:10226000FDF702FB94F9040034F092FDE27906EBED
:1022700082020346D2F810270492227A06EB8202E9
:102280005146D2F810270392A27906EB8202484603
:10229000D2F810270292627906EB8202D2F8102758
:1022A0000192226800925A46FDF796FA079B0C3578
:1022B000AB4204F10C0495D109B0BDE8F08FC246E1
:1022C000D0E700BF600C050843EC05082DE9F04796
:1022D00080468CB00846FEF709FF054638B100235A
:1022E00059491A4601200CB0BDE8F04768E7CDE92E
:1022F00009000B90079107A854493DF079F906466B
:1023000034F09AFC431C04460ED12B460A2208A93D
:102310003046FBF727FE089B1B782BB9C4B2132C61
:1023200096BF333444B264B2204607F06BFD0546D5
:1023300028B94046FEF732FE0CB0BDE8F0874349AD
:102340008DF8284007A83DF053F9B0B300230A22C6
:102350001946FBF707FE02260990DFF8F090DFF838
:10236000F4A00027494607A83DF042F9F8B1FBF771
:1023700073FE374A002352F8041B88421FD1DBB298
:102380000AEB8302D2F81027904210D1022F20D0FE
:10239000032F23D05A1E012FD2B215D00B2A03D8F7
:1023A0008DF829300136F6B20137042FDAD1052E27
:1023B0001AD84046FEF708F8BEE70126CDE70133FC
:1023C000102BD8D10023DBE7052AEDD88DF82A3071
:1023D000E8E7092BE8D88DF82C30E3E79A1E0D2AA0
:1023E000E2D88DF82B30DDE709AB03CB2860186805
:1023F0006960A860204634F0CBFC164A9DF82B108B
:1024000002EB81010346D1F8101704919DF82C10BE
:1024100002EB8101D1F8101703919DF82A1002EB0D
:102420008101D1F8101702919DF8291002EB810269
:102430000021D2F810270192099A00920846064A14
:10244000FDF7CAF978E700BF2479002036ED0508CA
:1024500070130508600C050843EC05082DE9F04FE2
:1024600090468BB00C461A4600210746FEF7F2FC58
:102470004546099000264FF0190A4FF46179B8F1EA
:10248000000F4BD029460A2220463DF051FA002881
:10249000099A14BF0121002138460CBF4FF0010BEF
:1024A0004FF0000BFEF7D6FC2A890692EA880592C7
:1024B0002A790492EA780392AA7809901AFB029288
:1024C00002926A781AFB029201922A7800923346AD
:1024D000134A59463846FDF7C7F922890692E28821
:1024E000059222790492E2780392A2781AFB029272
:1024F000029262781AFB0292019214F80A2B00925F
:102500003346074A594638460136FDF765F91E2E0F
:1025100005F10A05B3D10BB0BDE8F08FC346DCE787
:1025200060EC05082DE9F04380468BB00846FEF7C5
:10253000DDFD0F46044638B100235E491A460120EE
:102540000BB0BDE8F04389E70846FBF785FD1D2881
:10255000054600F3A5800A264643781C8DF82740DF
:10256000FAF7A9FE10B101238DF82730FAF7A3FE80
:10257000514C074668B1FBF76FFD0D2809D80A23B7
:1025800003FB054383F8F0069DF8273001338DF8EF
:102590002730DFF82091711C0DF12702494438469D
:1025A000FBF75EFDFAF787FE074668B1FBF754FDBF
:1025B000232809D89DF827300A2202FB054201335F
:1025C00082F8F3068DF827303846FAF774FE07468E
:1025D00068B1FBF741FD0D2809D89DF827300A2284
:1025E00002FB0542013382F8F4068DF827309DF88E
:1025F0002730062B0CD009EB06020023404649F891
:102600000630536013810BB0BDE8F043FDF7DCBE2C
:102610000A2606FB054600233846A6F8F636A6F835
:10262000F836FAF748FE074618B1FBF715FDA6F88D
:10263000F6063846FAF73FFE30B1FBF70DFD0A23E8
:1026400003FB0543A3F8F8061C4B4FF0FF325A601A
:102650000A2303FB05424FF46170B2F8F836069383
:10266000B2F8F636059392F8F436049392F8F336FE
:10267000039392F8F216192313FB0101029192F8C9
:10268000F11613FB0103019392F8F0360093002139
:102690000B4A2B460846FDF79FF80BB0BDE8F083C8
:1026A00008491D23224640460BB0BDE8F043FEF723
:1026B00011BD00BFE0870020F080002068040020EA
:1026C00060EC05083DEC05082DE9F04F2DED088B79
:1026D000DFF828A195B0804691461E460C46154667
:1026E000002794ED008AB5EE408AF1EE10FA7DD015
:1026F000D4ED019A94ED029AD4ED038AB9F1000F5A
:1027000049D0D5ED00BA95ED01BAD5ED02AA95ED07
:1027100003AAB4EE6B8AF1EE10FA6CD1F4EE4B9A88
:10272000F1EE10FA67D1B4EE6A9AF1EE10FA62D1C6
:10273000F4EE4A8AF1EE10FA0CBF01210021324674
:102740008B46404681F00101FEF784FBB0EE6B0A38
:10275000064611A8FAF7D4FCB0EE4B0A07900EA873
:10276000FAF7CEFCB0EE6A0A06900BA8FAF7C8FC9E
:10277000B0EE4A0A059008A8FAF7C2FC0599069A35
:10278000079B039002910192009352463B465946A3
:102790004046FDF769F8B0EE480A11A8FAF7B0FC18
:1027A000B0EE690A83460EA8FAF7AAFCB0EE490A11
:1027B00006900BA8FAF7A4FCB0EE680A059008A8EA
:1027C000FAF79EFC069B059A0390CDE900B30292AE
:1027D0003B465246002140460137FCF7FDFF082FDB
:1027E00004F1100405F110057FF47BAF15B0BDECCA
:1027F000088BBDE8F08F0021A1E700BF83EC05083E
:102800002DE9F14FDFF898B106460C462046FEF759
:102810006DFC074638B100235A491A46012001B021
:10282000BDE8F04F50E7584905222046FBF75EFB14
:1028300060B9544B00221A601A611A621A631A6452
:102840001A651A661A6701B0BDE8F08F042259466E
:102850002046FBF74BFB05462046002D45D1FAF7F5
:102860002AFD07460028EED03BF088FADFF834A1B5
:102870005FFA80F85AF8049BB9F1000F07D1434979
:102880002246304601B0BDE8F04FFDF787BD424615
:1028900049463846FBF72AFB013584460028E9D132
:1028A000384A0346174600210133082B42F8101B13
:1028B000FAD1374B03EBC505D5F880E0BEF1000F28
:1028C00005D13448344C4946FDF730F89EE795F879
:1028D0007C50AC45F5DA0EEB0C130FCB07EB0C1468
:1028E00084E80F000CF1010CF3E7FBF7B5FB0728B8
:1028F00005463DD82046FAF7DEFC074658B3FAF7FE
:1029000099FA204B03EB051383ED000A01243846A6
:10291000FAF7D1FC074638B1FAF78CFA194B03EBFA
:10292000051383ED010A01343846FAF7C4FC074663
:1029300038B1FAF77FFA134B03EB051383ED020A64
:1029400001343846FAF7B7FC38B9304601B0BDE873
:10295000F04FFDF739BD0446D9E7FAF76BFA094B9A
:10296000032C03EB051383ED030A3FF454AFECE7AC
:102970000A4907233A46304601B0BDE8F04FFEF75A
:10298000A9BB00BF0C8900200FE90508D4E50508A4
:10299000600C05089CEC050883FE05083DEC050865
:1029A00097EC0508981105082DE9F74F92460C465B
:1029B0001A4600218146FEF74DFADFF870B08046D6
:1029C00056460025BAF1000F2ED03146042220468B
:1029D0003CF0AEFF0028424614BF012100214846CA
:1029E0000CBF01270027FEF735FA738801933AF8E8
:1029F0002530009380462B465A4639464846FCF718
:102A000033FF6388019334F8043B00935A462B4606
:102A1000394648460135FCF7DFFE042D06F1040671
:102A2000D0D103B0BDE8F08F5746EAE7A6EC050821
:102A30002DE9F34105460846FEF758FB0C460746CC
:102A400038B1002333491A46012002B0BDE8F041F5
:102A5000AAE731492046FAF7C9F970B92D4B04228B
:102A60004FF47A704FF4FA61013A1880598003F1FB
:102A70000403F9D102B0BDE8F0812046FBF7ECFA7F
:102A80000328064641D82046FAF715FC074698B1B8
:102A9000FBF7E2FA4FF0010804463846FAF70BFC60
:102AA00020B1FBF7D9FAB8F1000F09D1284602B0DE
:102AB000BDE8F041FDF788BC40F2EE248046ECE72B
:102AC000A4F2EE2240F2DC539A4203D8A0F2EE22A6
:102AD0009A420AD9114940F6CA0340F2EE2228462A
:102AE00002B0BDE8F041FEF7F5BA0D4B0D4A03EB1D
:102AF00086030021A3F89C48A3F89E08CDE9004076
:102B000033460846FCF768FEB4E7074903233A4614
:102B1000E5E700BF8C8900200FE90508B7EC050840
:102B2000F0800020A6EC0508BFE805082DE9F04F6D
:102B30000E46154689B01A4600210446FEF78AF96A
:102B4000B04681462F464FF0000B002D7CD0394611
:102B50000C2240463CF0ECFE00284A4614BF0121FE
:102B6000002120460CBF4FF0010A4FF0000AFEF78B
:102B700071F997F90B20049297F90A200392B7F99B
:102B800008200292B7F906200192B7F904200092BA
:102B90008146384A5B4651462046FCF765FE98F967
:102BA0000B20049298F90A200392B8F908200292A7
:102BB000B8F906200192B8F9042000925B462D4A2C
:102BC000514620460BF1010BFCF706FEBBF1080F46
:102BD00008F10C0807F10C07B7D1DFF89C804FF023
:102BE000000B0C2303FB0BF985B3002755F80900F4
:102BF00056F80920012303FA07FA42403AEA020292
:102C000014BF1946002110EA0A0F07D000975B464F
:102C1000424620460791FCF727FE079956F80920FF
:102C20001AEA020F05D000975B4642462046FCF7A1
:102C3000D3FD01370E2FD9D10BF1010BBBF1080FDA
:102C4000CFD109B0BDE8F08FAA46A8E72F4656F8C5
:102C50000910012303FA07F20A4206D000975B46E7
:102C6000424601212046FCF7B7FD01370E2FEED179
:102C7000E2E700BFC5EC0508DDEC0508F0B5064647
:102C80008BB00846FEF732FA0D46044620B3002307
:102C90003D491A4601200BB0BDE8F04046E72D291A
:102CA00003D0A1F13003092B49D8052C05DD3046AE
:102CB0000BB0BDE8F040FDF787BB2846FBF7CCF929
:102CC0000AAB621C03EB440424F80C0C15F8013F1A
:102CD000303B092BFAD9144629780029DFD1062C7C
:102CE000E5D1BDF81C20BDF91C30072ADFD8BDF99D
:102CF0001E50A5F5FA7292B2B2F5FA6F18D8BDF966
:102D00002070A7F5FA7292B2B2F5FA6F10D8BDF939
:102D100022C065450CDC67450ADBBDF924E00EF1F5
:102D2000640292B2C82A03D8BDF92640112C11DDE5
:102D3000164930460BB0BDE8F040FDF72FBB202907
:102D400002D101352246C6E730460BB0BDE8F0405F
:102D5000FEF724B90E4A0C2000FB032264B2A2F84D
:102D6000B058A2F8B278A2F8B4C882F8B6E882F8EF
:102D7000B7480846CDE903E4CDE9017C054A009552
:102D8000FCF72AFD0BB0F0BD9C890020F2EC050891
:102D9000F0800020C5EC05082DE9F04F89468DB084
:102DA000164600211A460746FEF754F8DFF8DCA065
:102DB00005460024C4EBC40309EB030259F80300E1
:102DC00091889279089040F30748ADF824108DF867
:102DD0002620B8F1000F54D0002E55D0F218F0582C
:102DE000918893790A90ADF82C1007220AA908A8B7
:102DF0008DF82E303CF09CFD00282A4614BF01219E
:102E0000002138460CBF4FF0010B4FF0000BFEF7CE
:102E100021F89DF82E3006939DF92D3005939DF9EC
:102E20002C3004939DF82B3003939DF92A300293A4
:102E30009DF8293001939DF82830009305462346DC
:102E4000524659463846FCF70FFD9DF8263006934A
:102E50009DF9253005939DF9243004939DF8233086
:102E6000CDE902839DF8213001939DF82030009335
:102E700052462346594638460134FCF7ADFC102C27
:102E800098D10DB0BDE8F08FB346DEE708ED050838
:102E90002DE9F04FDFF8A4828BB006460D46284698
:102EA0003AF06CFF034630B99649024601200BB058
:102EB000BDE8F04F70E7944905222846FBF716F865
:102EC0000446C8B9914D0146702205F60C103CF03D
:102ED000DFFBC5F8AC48C5F8B848C5F8C448C5F824
:102EE000D048C5F8DC48C5F8E848C5F8F448C5F846
:102EF00000490BB0BDE8F08F042241462846FAF79E
:102F0000F5FF044630BB2846FAF7D5F9814600287C
:102F1000EFD03AF033FFDFF828B282465BF8047B4B
:102F20003FB97B492A4630460BB0BDE8F04FFDF76C
:102F300035BA524639464846FAF7D8FF40B92046D6
:102F40001DF09AF87348744D3946FCF7EFFCA6E77C
:102F50000134E3E7714907222846FAF7C7FF07461D
:102F600000287AD1202128463CF0A9FB044670BBFA
:102F70006B486C4DFCF790FC214628460134FCF769
:102F80008BFC0E2CF8D1FCF723FCDFF8B891664FD0
:102F9000DFF8B481002529464846FCF77DFC0C2665
:102FA000DFF8A8A16E430024F25960480123A34032
:102FB00013420CBF414651460134FCF76DFC0E2C08
:102FC000F2D10135FCF704FC082DE4D191E7584912
:102FD000574D01AA3CF039FB02AC002848D0022F23
:102FE00011D1029A072A07D8039C0D2C04D8037824
:102FF000722B13D06E2B25D04E4908230022304669
:10300000FEF768F875E7FBF727F801AA44F8040B08
:103010002946002001373CF018FBDEE73B490C2332
:1030200003FB02110123D1F8AC18A3400B4337492D
:103030000C2000FB02123949C2F8AC383046FFF7C9
:1030400027FF56E7314B0C2000FB02330121D3F858
:10305000AC38A14023EA0103E9E728463449344F5C
:1030600001AA3CF0F2FA02AD002480B1082C03D191
:103070003046FDF7A9F93CE7FAF7EEFF01AA45F85B
:10308000040B3946002001343CF0DFFAEDE7082C50
:10309000EED1029B0F2B30D8DDF80CE0BEF1070F0C
:1030A0002BD8DDF810C0BCF10D0F26D8059F07F115
:1030B0006402C82A21D8069DFF2D1ED807986428CF
:1030C0001BD80899642918D8884216DA099C032C61
:1030D00013D8C3EBC3020D4B134483F8111983F8C3
:1030E0000CE90D4983F80DC983F80E7983F80F595F
:1030F00083F8100983F81249A0E70F493046FDF71D
:103100004DF9F6E6FC8900200FE90508F080002063
:10311000D4E505089CEC050883FE050825ED0508A7
:103120002DF405082DED05089C89002032ED0508D9
:1031300036ED050838ED0508F2EC050897EC0508B2
:103140009811050849DF050885F20508F0EC050827
:103150002DE9F04F924689B00C461A4600210746E9
:10316000FDF778FE002607905546B3464FF0190943
:103170004FF46178BAF1000F28D029460622204684
:103180003CF0D6FB0028079A14BF012100213846E5
:103190000CBF4FF0010B4FF0000BFDF75BFE6A799F
:1031A000079019FB028205922A7919FB0282049288
:1031B000EA780392AA7802926A7801922A780092B9
:1031C0003346124A59463846FCF74EFB627919FBE2
:1031D00002820592227919FB02820492E27803921C
:1031E000A27802926278019214F8062B009233467C
:1031F000064A594638460136FCF7EEFA0A2E05F122
:103200000605B7D109B0BDE8F08F00BF3EED050857
:103210002DE9F04F074689B00846FDF767FF8B465A
:10322000044638B1002354491A46012009B0BDE8CC
:10323000F04F8DE7514B084693F84CAC93F84D9CFA
:1032400093F8368DFAF708FF0928054600F38B80BE
:10325000062646430BF101008DF81F40FAF72BF8C4
:10326000474C834648B1FAF7F7FE0D2805D8A31955
:1032700083F87C0901238DF81F305846FAF71BF8B4
:10328000834668B1FAF7E8FE504509D8062303FBE8
:10329000054383F87D099DF81F3001338DF81F30F9
:1032A0005846FAF708F8824668B1FAF7D5FE48455D
:1032B00009D8062303FB054383F87E099DF81F30D8
:1032C00001338DF81F305046F9F7F5FF814668B19C
:1032D000FAF7C2FE804509D3062303FB054383F8B2
:1032E0007F099DF81F3001338DF81F30DFF888808B
:1032F000311D0DF11F0241444846FAF7B1FE9DF819
:103300001F30062B0BD008EB06020023384648F886
:103310000630938009B0BDE8F04FFDF755B803FBC8
:1033200005424FF4617092F88119192313FB0101D2
:10333000059192F8801913FB0103049392F87F39E9
:10334000039392F87E39029392F87D39019392F8B3
:103350007C39009300210B4A2B460846FCF73CFAC7
:1033600009B0BDE8F08F084909232246384609B064
:10337000BDE8F04FFDF7AEBE6C8A0020F86F00206C
:10338000F08000203EED05083DEC05082DE9F04FEA
:103390000F468BB0144600211A460646FDF75AFD2B
:1033A0000546002C00F0DD8022783B789A4218BF59
:1033B0000121024608BF002130460CBF4FF0010832
:1033C0004FF00008FDF746FD23789E4A054641462A
:1033D0003046FCF749FA3B789A4A41463046FCF7BA
:1033E000FBF9002C00F0BF8062787B789A4218BF0E
:1033F00001212A4608BF002130460CBF4FF00108CA
:103400004FF00008FDF726FD63788F4A05464146D8
:103410003046FCF729FA7B788B4A41463046FCF768
:10342000DBF907F1C9030593A31C0693822307F177
:10343000020A04F1CA0B07934FF000093B784B4591
:1034400000F39380002C00F0F68097F8EA3094F8AF
:10345000EA209A4218BF01212A4608BF00213046BF
:103460000CBF4FF001084FF00008FDF7F3FC94F893
:10347000EA30764A054641463046FCF7F5F997F8BA
:10348000EA30724A41463046FCF7A6F9002C00F0BB
:10349000D48004F1EA0307F1EA0204F1FA014FF0E3
:1034A000010833F802CF32F8020F844518BF4FF0FD
:1034B00000089942F5D188F001012A46C9B2304688
:1034C000FDF7C8FC0821054604F1EC00FAF772FC90
:1034D0005F4A034641463046FCF7C6F997F8EA10C2
:1034E00007F1EC00FAF766FC594A034641463046BC
:1034F000FCF772F9002C00F0A2804FF0FC094FF0AD
:10350000010807EB090104EB0900F9F76FFC09F169
:103510000409002818BF4FF00008B9F58E7FF0D1DC
:1035200088F001012A46C9B23046FDF793FC082114
:1035300004F1FC00F9F7D2FE464A03464146304604
:10354000FCF792F997F8EA1007F1FC00F9F7C6FECC
:10355000404A0346414630460BB0BDE8F04FFCF709
:103560003BB9A04637E7A04655E7079BFB180993F0
:10357000002C5ED0079B0998E31819460893F9F7C9
:1035800035FC059B5A789BF800309A42069A06BF94
:10359000B0FA80F84FEA58184FF00008AAF1020379
:1035A000023A0AF10E0133F802CF32F8020F8445D5
:1035B00018BF4FF000088B42F5D188F001012A4670
:1035C000C9B23046FDF746FC6278069905469BF87D
:1035D0001800FAF7C1FB02909BF800300193089B9A
:1035E00000931D4A09F1010341463046FCF73CF9BE
:1035F000059B7A78587E5146FAF7AEFB059A029001
:1036000012F8013F019309F10109099B059200930A
:10361000114A4B4641463046FCF7DEF8069B103314
:103620000693079B09330AF1100A0BF1010B07936C
:1036300004E7A046DCE7A04621E7A0464EE7A04607
:1036400080E700BF57ED050869ED050897ED05080F
:10365000AFED0508C6ED05087EED05082DE9F04F34
:103660008FB0044602AA0846B1493BF0EEFF05467A
:1036700040B903460246AF494120FFF787FE0FB02D
:10368000BDE8F08FAC49F9F7B1FB064628BBA84965
:1036900002AA3BF0DAFFFAF7DFFC0828054606D954
:1036A000A649082332462046FDF714FDE7E7A44C5F
:1036B00094F84C3C83420CDC84F84C5CDFE73146E8
:1036C000384628F09DFD013694F84C3CB342F6DCB8
:1036D000F2E7064604F64C47F6E79A492846F9F71A
:1036E00085FB0646E0B9924902AA3BF0AEFFFAF725
:1036F000B3FC0828054603D9934908233246D2E78C
:103700008F4C94F84D3C834202DC84F84D5CB6E764
:1037100030462946013633F067FA082EF8D1F4E72F
:103720008A492846F9F762FB064600BB804902AA8F
:103730003BF08BFF0028A2D0FAF78EFC0828054644
:1037400003D9834908233246ADE77D4C94F8363DD2
:10375000834209DD014604F64C4028F095FD2946D8
:1037600004F64C4028F09EFD84F8365D87E77949E1
:103770002846F9F73BFB064618BB714BDFF8B091C2
:1037800093F8367D06AD0146102228463BF080FFB7
:10379000A846BE4202AA80F20A81494600203BF0B8
:1037A00054FF10B96C493A460AE1FAF755FC013664
:1037B00028F8020BEDE795E80F00684C84E80F004D
:1037C0005DE767492846F9F711FB0646C0BB5C4B2D
:1037D000DFF85C9193F8367D06ADBE4202AA80F216
:1037E000F380494600203BF030FF014610B95D49A7
:1037F0003A46E5E0032228463CF048F8AA464FF056
:10380000000828463AF0BAFA404502D80136043595
:10381000E3E79AF80000FAF763FB08F101080AF8F9
:10382000010BEEE7504DB6000446B4423FF427AF1B
:1038300006AB19192819032228F0CCFC0434F4E74C
:103840004A492846F9F7D2FA0746002840F0AC80EA
:10385000DFF8EC80364998F84C6C02AA3BF0F5FE94
:1038600000283FF40CAFFAF7F7FB451E01D4AE4237
:1038700003DC3F493346012215E72D4902AA002007
:103880003BF0E3FE014600283FF4F9AE0026082293
:1038900003A88DF814603BF0F9FF0DF10C0903A8A3
:1038A0003AF06CFAB0421BD8214902AA00203BF042
:1038B000CCFE00283FF4E3AE037898F84DAC0193BA
:1038C0000026B14656451A4902AA4FF0000080F280
:1038D00085803BF0BAFE834650B9264952466FE0D8
:1038E00099F80000FAF7FCFA013609F8010BD6E75F
:1038F000A6B99BF80030303B092B0FD91E49F9F7C8
:1039000075FA38B11D495846F9F770FA70B11C497B
:103910005A4655E04FF001094FF0FF365846FAF786
:103920009BFB002830DA17495A4649E0B146F3E7D5
:1039300036ED0508447C0020DDED0508E3ED0508C3
:10394000F86F0020EEED0508F7ED050805EE050817
:1039500011EE050823EE050812EF0508307D002062
:103960004DEE050832EF0508407D002077EE050892
:103970007CEE050852EF050893DE050888EE050881
:103980008FEE0508C4EE05080EAB03EB46030136C7
:1039900023F8200C96E72049524611E033F8022B19
:1039A00024F8022F013730E01C492A4608E01C4960
:1039B00000203BF04AFE00283FF4FDAE19493A468C
:1039C0002046FCF7EBFC5AE6154900203BF03DFE93
:1039D00000283FF427AF14493A46F1E73BF035FEA3
:1039E0000028D8D1114C05EBC500823020440822B4
:1039F00003A928F0EFFB0198FAF772FA08EB050328
:103A000004EB051483F8160D06ABBE42C6DC454434
:103A100085F82E9D33E600BFD9EE0508FCEE0508BB
:103A200036ED05082FEE050859EE0508447C002008
:103A30002DE9F04F89B00F4690460021139A039369
:103A40000646FDF707FA87EA08086FEA0803DFF879
:103A50008490069304460025284606F0B3F9129B8D
:103A6000184230D0069BDFF870B0034014BF4FF00F
:103A7000010A4FF0000A049310EA07030CBF4A46FC
:103A80005A4628460593079206F0AEF9039B079A1B
:103A90000090804651463046FBF7E6FE049BB3FAA1
:103AA00083F1224649093046FDF7D4F9059A039B74
:103AB000CDF800800446002A0CBF5A464A465146BB
:103AC0003046FBF789FE0135172DC5D109B0BDE899
:103AD000F08F00BF77EF050891EC050870B504463C
:103AE00008460E463AF04AF9314605460246204657
:103AF000FAF7FCF968B9635D1846FAF7E1F900B91D
:103B000033B901352C44204601340378202BFAD0F8
:103B100070BD0020FCE708B504460948FBF750FEDD
:103B2000FBF732FE074BD3F8BC0606F0FFF903F0B3
:103B30000FFE012C01D134F08FF9F5F757FB00BFD0
:103B40007EEF0508F080002010B5044608460B46BD
:103B5000FDF7CCFA28B9094903221846FAF7C6F945
:103B600028B90748FBF752FE0120FFF7D4FF204693
:103B70000449BDE81040FCF711BC00BF8AEF0508FE
:103B80008EEF0508F6E705082DE9F74F064601AA6E
:103B900008462F49DFF8C880DFF8C890DFF8B0A0EA
:103BA0003BF053FD4FF0000B04465D4601271CBB64
:103BB000BBF1000F28D1274C002D44D026482946C0
:103BC000FBF7B4FE94F830300BB902F0F5FD31F09C
:103BD00003FB002384F85930FBF7ACFD15B12846F0
:103BE000FDF745F99FB13046FDF7FAF878B1FBF7DC
:103BF0002DFB0020FFF78FFFBBF1000F0AD02046FE
:103C0000FAF72AFA85B2C5B93046FDF7C7F903B00D
:103C1000BDE8F08F41462046FAF78CF980B9494655
:103C20002046FAF787F90028EED05F4601AA5146F0
:103C300000203BF00AFD0446B9E74FF0000BF5E722
:103C40004FF0010BF2E70548FBF7E0FDBFE700BFCF
:103C500036ED0508F86F0020B9EF0508DCEF050820
:103C6000B0EF050815F5050810B50C46FDF7B8F8D6
:103C700078B1084B01229A73FBF7E8FA0648FBF784
:103C8000C5FD06492046F9F7B1F810B10020FFF74D
:103C900042FF10BDF86F0020F2EF0508B3DE050803
:103CA000F0B5032985B005460C46164614D80B4FCF
:103CB0003970FBF78DFD0A492846FDF7CBFE09490F
:103CC000224601A8FAF732F801AB3246082128460D
:103CD000FDF7F0F8FF233B7005B0F0BD680400204D
:103CE00083FE05088DEB0508F0B5032985B0054670
:103CF0000C46164614D80B4F7970FBF769FD0A493C
:103D00002846FDF7D7FE094922466846FAF70EF81D
:103D10006B46324610212846FDF7CCF8FF237B7016
:103D200005B0F0BD6804002083FE050889EB050896
:103D300010B586B00E4B04930E4B03930E4B0293BB
:103D40000E4B01930E4B0F4A0F49009304460F4B45
:103D50000F48FBF7A1FDFBF73BFD3CB10D4A0E49B7
:103D60000E4806B0BDE81040FBF7E0BD06B010BD40
:103D700039F005083EF0050849F0050852F005083D
:103D80005EF00508F9EF050803F00508FF6F002055
:103D90000EF00508A2E40508F9E4050868F0050836
:103DA0000120C5E72DE9F04F0A4689B000210546FC
:103DB000FDF750F8394C059094F9000003F02AFD06
:103DC0008146608831F0CEF9354BD0F808B093F8D1
:103DD000307017B15F46D0F80CB0A379012B38BF13
:103DE0000123069300262279637906FB02331BF830
:103DF0000380002F3BD0FB5C059A0793434514BF1B
:103E00000121002128460CBF4FF0010A4FF0000AA3
:103E1000FDF720F8079B0590013653B303F00F021E
:103E20001B094033CDE9006302924B461D4A5146BF
:103E30002846FBF719FDB8F1000F24D008F00F0356
:103E40004FEA1818029308F14003CDE90063154AC0
:103E50004B4651462846FBF7BFFC069BB342C2DCEB
:103E6000114B0834A342A7D109B0BDE8F08F3B46FF
:103E7000C2E7002FDFD00D4A00964B465146284638
:103E8000FBF7F2FCD7E76B06E7D4084A00964B46EF
:103E900051462846FBF7A0FCDFE700BFB01305083A
:103EA000F86F002095F00508C0140508ABF0050870
:103EB00038B50B4D05EBC0050C4695F9500703F0DE
:103EC000A9FC01460748FBF7E7FC95F8563733B1E4
:103ED000611C0548BDE83840C9B2FBF7DDBC38BD00
:103EE000600C05082CF4050848DF050873B50E467C
:103EF00010490546F8F77AFF18B93070012002B072
:103F000070BD2C78602C8CBF613C413C082C0FD8D4
:103F1000013501230A2201A92846FAF723F8019B5B
:103F2000AB4205D00F2803D8013440EA0410E4E77F
:103F30000020E4E72CDE05082DE9F04F0A468DB09D
:103F400000218346FCF786FF704CDFF8CC9103908C
:103F500004F1B00A0025A37A99F83060AB4200F36F
:103F6000938010345445F5D140F2162031F0FAF820
:103F7000D0E902450DF1180A002E4FF015024FF05E
:103F80000001504604BF254634463BF081FB002724
:103F90002E78002E3ED069780591304604F020FD41
:103FA00095F90290049009F1010253425341002C0B
:103FB00000F0A98005990022A05CB04240F09F80EB
:103FC000224492F90280C14540F0978052788A429B
:103FD00008BF012301220AF8072003F0010383F040
:103FE0000101039A05935846FCF734FF059B0390A3
:103FF00044B1474A0499CDE900B230464246F9F748
:10400000DFF9059B434A0499CDE900B230464A46A0
:10401000F9F7D6F90137152F05F10305B8D184B3A7
:10402000DFF8EC80DFF8EC90564604F13F0716F815
:1040300001ABBAF1000F21D12078F8B194F9023028
:1040400001331BD0617804F0CBFC039A05460121B3
:104050005846FCF7FFFE94F902200390534620785F
:104060002946CDE900B8F9F7ABF920785346CDE9F8
:1040700000B94FF0FF322946F9F7A2F90334BC42E8
:10408000D5D10DB0BDE8F08FE08831F06BF8D0E904
:104090000231627A207A002E08BF194605FB002201
:1040A00008BF33468F562BB39E56039A0493B742EC
:1040B00014BF0121002158460CBF4FF001084FF0FA
:1040C0000008FCF7C7FE049B039043B1104B324637
:1040D000CDE900B3294643462046F9F72DF90D4BAB
:1040E0002946CDE900B33A4643462046F9F724F97C
:1040F000013530E74FF0FF36D7E700236AE7033298
:104100003F2A7FF459AF4FF0FF3868E7A40400203E
:1041100069F80008D9F70008F86F00202DE9F04F82
:1041200080468BB008460D4639F028FE0246B8B3EB
:10413000A7492846F9F7DAFE044688BBFBF748FB97
:10414000A448A54DA54EA64FDFF8D882FBF758FB33
:10415000142032F05DFD04F00702E1103046013218
:104160000131FBF799FB95F81D9095F91C00B9F109
:10417000000F0ED003F04EFB4A4601464046FBF7C7
:10418000D5FB0134102C05F12405E4D10BB0BDE8BA
:10419000F08F03F03FFB01463846FBF7C7FBF0E723
:1041A0002846904905AA3BF050FA054620B9014639
:1041B0004120FFF7C1FEE9E78B49F8F717FE20B968
:1041C0008A494046FCF7EAF8E0E7894E0B270024CD
:1041D00031682846F8F70AFE002808BF3446013F38
:1041E00006F11006F4D154B982492846F8F7FEFDCD
:1041F00028B181492A464046FCF7D0F8C6E700209E
:1042000078498DF8130005AA3BF01FFA0646002CEA
:104210004ED000284AD0F9F71FFF031E43DB227956
:10422000062A3BD1E168012202FA03F008423AD0A3
:104230007248DBB240FA03F1C90734D59A40013A1B
:1042400010403BF0D1FB0546E08830F08BFF6C4915
:10425000D0E9022391F83010002918BF1A46217ABC
:10426000637A05FB0133D118002712F903900291FC
:1042700003975C4905AA00203BF0E7F98346002834
:104280003FD1604901239CB3029A204692F9002055
:10429000CDE900312946F9F74FF877E75D1E13B1F4
:1042A000A37A9D42D0DB58493246A4E7574EFAE73D
:1042B00068B10DF11301FFF719FE28B19DF81350F5
:1042C0002846F4F71FFA20B95149324693E74F4E7A
:1042D000FAE72846F3F7D2FB8146284604F06CFB48
:1042E0000390284604F0A4FB254607460294C0E745
:1042F000CDE900319DF813004A463946F9F760F8D8
:1043000044E73949F8F772FD064600282FD1ACB1D1
:10431000404FEDB2207972B22946F3F783FB0028B3
:104320003FF434AF0288037800933146C2F303238D
:104330003846120BFBF7FAFA0136EBE73868797961
:10434000344C72B2F3F7B6FB00283FF41FAF02887B
:10435000037800933146C2F303232046120B013643
:10436000FBF7E4FA102E38687979EAD10EE72A498A
:104370005846F8F73BFD002877D05846F9F76CFE11
:10438000824642B29CB12079E9B2F3F74BFB002898
:104390004ED129462046F8F79BFE26681F49CDF8E6
:1043A00000B0034632464046FBF7F8FFEEE65FFA00
:1043B0008AF60F2E3868797936D99DF81330184966
:1043C000CDF800B01A09403203F00F03EBE700BF4D
:1043D000BFF00508C4F0050868010020DAF0050800
:1043E000F7E5050836ED0508A4E20508ECF0050838
:1043F000A404002087F8050800F10508FE811300D9
:10440000F86F0020D9F700080FF1050883FE0508B2
:104410001FF1050831F10508F1E5050853F105081C
:1044200076F10508B9F60508F3F744FB0028C4D077
:1044300006AE31465046F9F7F1FC08A94846F9F7AF
:10444000EDFCCA4520D04FFA8AF38CB1029A294676
:1044500013702046F8F73CFE276800960246154880
:1044600008AB3946FBF762FA90E64FF0FF3ADFE718
:10447000039A114893709DF813200096110908AB18
:1044800002F00F024031EDE75CB129462046F8F713
:104490001FFE26680246094808AB3146FBF746FA7C
:1044A00074E69DF813200648110908AB02F00F02CC
:1044B0004031F3E79EF10508C1F10508E9F105086F
:1044C00004F205082DE9F04387B00709DDF83880CC
:1044D00091461E46403700F00F0439B304F080FACD
:1044E000C379174ACDE9004305463B464946304665
:1044F000C047C0B12868F3F70DFCAA796B79114960
:1045000012F0020F4FEA93030F4A18BF0A46E979E7
:1045100000940133CDE90321CDE901030B4A3B4669
:1045200000213046C04707B0BDE8F083084A0E942A
:104530003B4649463046C44607B0BDE8F0436047B5
:1045400020F205089EDF050883FE050832F2050803
:1045500054F205082DE9F04F07468BB040F21620C3
:104560000C4630F0FFFD2246054600213846FCF798
:1045700071FC434BD5E9024593F83030002B08BF5E
:10458000254606464FF015024FF0000104A808BF6B
:104590001C463BF07DF805F13F03039395F800902E
:1045A000B9F1000F31D095F801A0002C65D022465A
:1045B00000231178494558D128336B4492F8018083
:1045C000012203F8182CD045324614BF01210021E6
:1045D00038460CBF4FF0010B4FF0000BFCF73AFCD4
:1045E000064654B1B8F1000F07D0264B00935A4647
:1045F0003B4641464846FFF765FF234B00935A462A
:104600003B4651464846FFF75DFF039B03359D42FD
:10461000C4D13CB3DFF86C90DFF86CA0651C0DF1E1
:104620001008403418F8013BCBB915F8013CB3B180
:1046300016B13046FBF7EAF8297815F8010CCDF8E9
:1046400000903B460022FFF73DFF002215F8010CC9
:10465000CDF800A03B461146FFF734FF0026033596
:10466000A542DFD10BB0BDE8F08F0133152B02F16D
:1046700003029ED14FF00008A5E7A046A3E700BFC4
:10468000F86F002069F80008D9F7000810B501316B
:10469000144604F0A5F928B9064B1A681B79226064
:1046A000237110BDC27904492046BDE81040F9F7D6
:1046B0003DBB00BF2CDE05082DF20508224BB0F5EE
:1046C000FA6F1A680346A8BF4FF4FA63B3F57A7F0E
:1046D000B8BF4FF47A73D20416D540F2DC52904240
:1046E00015D007EE903A40F2DB529042F8EE677A2E
:1046F0001FD8DFED166A9FED167A9FED160A77EE4A
:10470000E67AA7EE870A7047B0F57A7F02D89FED68
:10471000120A704707EE903ADFED106A9FED107AAB
:104720009FED100AF8EE677A77EEE67AA7EE870A31
:104730007047DFED0D6A9FED0D7A9FED0D0A77EE64
:10474000E67AA7EE870A70478079002000007A4455
:10475000D62000C000E082440000000000407A44FF
:10476000661000400000404200A0BB44D62000403C
:1047700000008344704700BF704700BF00207047AF
:1047800001207047704700BF704700BF704700BFEF
:10479000704700BF9FED010A704700BF0000000096
:1047A00000207047064B1B78834206D9054B00EB6F
:1047B000400003EBC003586970470020704700BFFA
:1047C000351E0020741D0020034B00EB400003EB5E
:1047D000C003587C704700BF741D0020024B18783E
:1047E000003818BF01207047351E002003681B6980
:1047F00003B11847704700BF70B5094C236873B107
:104800000546002606E099681A681E7321609047E5
:10481000236823B15A68AA1A002A1846F3DA70BD31
:10482000B0A50020704700BF08B5254B1B68DB040E
:104830000AD5B5EE400AF1EE10FA12D19FED210A29
:104840003AF0FEF980B208BDDFED1F7AB4EEE70A58
:10485000F1EE10FA1CDA9FED1D0A3AF0F1F980B280
:1048600008BDDFED197AB4EEE70AF1EE10FAE5D4EF
:104870009FED177AB4EEC70AF1EE10FA14D870EE75
:10488000677A9FED147A9FED140AA7EE870AE4E792
:1048900070EE677A9FED117A9FED110AA7EE870AF5
:1048A0003AF0CEF980B208BDDFED0E7A9FED0E7AB8
:1048B00070EE677A9FED0D0AA7EE870ACDE700BF7D
:1048C000807900200080BB440000404200007A4410
:1048D00000E0824466BEFFBE0060BB4438DFFF3E9E
:1048E00000407A440000834466BEFF3E00A0BB4403
:1048F00070B58E4B1B6813F004032DED048B40F054
:10490000C4809FED8B8A8B4C1D4694F8B13094F88F
:10491000B02013F001037BD1002A74D1D4ED2D7A9D
:104920009FED857ADFED856A854B67EE877A94ED9A
:104930002F7A1E78E8EE267A0D2E38EE477AC4EDEF
:104940002D7A84ED2E7A02D17E4B00229A809FED43
:10495000787A9FED7D9AF0EE488A0023D4ED347A80
:10496000D4ED356A94ED338A37EE677AE6EE877ACE
:1049700037EEC87AC4ED347AA6EE878A84ED338A9E
:1049800084ED308A0BB184ED2E8A94ED367AD4ED25
:10499000387ADFED6E5AD4ED396A94ED370A84ED3A
:1049A000368A38EE477AB0EE676A97EE256AE6EE09
:1049B000867A37EEC07AC4ED387AA6EE870A84ED9F
:1049C000370A3AF03DF902B282EAE273A3EBE273EE
:1049D0009BB2092B40F2A280002AACBF0A380A30F1
:1049E00005B20D2EA4F8E85000F08380242E73D079
:1049F000382E05D1B0EE480A3AF022F9514B988092
:104A0000BDEC048B70BD84F8B23084F8B03085E71B
:104A1000002A3FD094ED2F9A494B1E780D2E78EE48
:104A2000498A09D1DFED4A7A94ED300A20EE270A4F
:104A30003AF006F9434B988094F8B23093B394F867
:104A4000C420CABB94ED307A002D42D094F8C53012
:104A500077EE487A06EE903A77EE897AF8EEE66AD3
:104A6000F0EEE77A67EEA67ADFED3A6AF4EEE67AE0
:104A7000F1EE10FA1ADD9FED2E9AF0EE687AE9EE6B
:104A8000077A2B46B0EE677A68E72A4C012594ED49
:104A9000298A3AE794ED2D9A012384ED2F9A84F820
:104AA000B030B9E76DB194F8C42042B99FED209AB7
:104AB000B0EE687A2B4651E7022A08D03DB1012AB0
:104AC0002ED094ED307A9FED1A9A012346E794EDAB
:104AD000307A9FED179A41E7DFED1D7A94ED2E0AAB
:104AE00020EE270A3AF0ACF8BDEC048B154B588049
:104AF00070BDDFED167A9FED160A124C69EE277A2B
:104B000028EE800AFDEEE77A17EE903A23803AF01D
:104B100097F8BDEC048B6080E58070BD002560E7F0
:104B20009FED039AB0EE687A134617E7987F00204E
:104B300000000000B0A50020CDCC4C3FCDCC4C3EB9
:104B400045470020484700209A99993E0000C842F6
:104B5000CDCCCC3D00401C462DE9F04F6B4B1B7873
:104B600087B0002B00F0CB80694D6A48A968FAF73E
:104B7000DDFE69686848FAF7D9FE684B6848D3E9F2
:104B80000031C91A674B1A68B1FBF2F2FAF7CEFE90
:104B9000FAF71EFE6448FAF733FE6448FAF730FE6F
:104BA0004FF00008624B1B785FFA88F4A34222D8CA
:104BB000FAF70EFE5F4D604E002455F8041F304694
:104BC0000134FAF769FE162CF7D1FAF701FE5B4DB6
:104BD000594E01242B4669681B683046C91A0134B6
:104BE000FAF75AFE162C05F10405F3D107B0BDE81B
:104BF000F04FFAF7EDBD524B142603EB840306FB8E
:104C0000045693ED3B0AB6F80E903AF019F896F870
:104C10001EA01AF0010F0CBF2D2252221AF0020F13
:104C20000CBF2D2354231AF0040F0CBF4FF02D0C92
:104C30004FF0560C1AF0080F0CBF4FF02D0E4FF02E
:104C4000430E81B21AF0800F4FF03C0BB1FBFBF129
:104C500005914FF064010CBF4FF02D0A4FF0530A3D
:104C600080B201FB09F1671CCDE902A10490CDE9F6
:104C700000CE34483946FAF70FFEB37FDB073AD54A
:104C80005C23314A6343D118D05891ED010A70B1C9
:104C9000DFED2E7AB8EE400A20EE270A07EE900AE2
:104CA000F8EE677A80EE270A39F0CAFF00B2642274
:104CB00090FBF2F102FB11022548FAF7EDFD1421F9
:104CC00001FB075701FB0454F988628A0491218B88
:104CD0000391E18A0291A18B0191A18A009102F0D6
:104CE000030319214B431B48218A9208FAF71EFE41
:104CF00008F1010856E71848FAF762FDDFE71748A0
:104D000007B0BDE8F04FFAF77BBD00BFC818002020
:104D10003C460020A3F20508B3F205085C470020DA
:104D2000CAF20508F0370020F7F2050853F305082A
:104D30006C7A0020E446002003F40508E8460020D1
:104D4000B0A50020AFF305085C43002000401C46DE
:104D5000CCF30508E1F30508D8F3050807F40508C6
:104D60002DE9F84F00261F4DDFF88090DFF880A076
:104D700007460C46B0462046FCF7B8F9D5F800B017
:104D800048B921465846F9F7D5F820B96868214650
:104D9000F9F7D0F880B15846FAF712FD696811B1F9
:104DA0005046FAF779FDA96811B14846FAF774FD43
:104DB000FAF70EFD4FF001080136362E05F1100509
:104DC000D9D12046FCF792F948B9B8F1000F06D1C5
:104DD000224638460449BDE8F84FFBF7DFBABDE884
:104DE000F88F00BF084005082FF4050829F40508CE
:104DF00023F4050870B5224C2378012B00D070BD38
:104E0000204B1B68002BFAD01F4D2B6828465B688F
:104E100098470028F3D01D4B1D4E1A68338892889E
:104E20009A421BD31B49096800224968EA622A6832
:104E300003FB01F12846D368984738F021FC164A55
:104E40003388526801333380002AD8D011689388A0
:104E50004A69134218BF1B048B6170BD0E4A0F4B89
:104E600052681B7800212170002AC8D091881268EE
:104E7000C3F340031B0101FA03F3936170BD00BF4C
:104E80008E4800201C2A0020202A0020884800206C
:104E90008C480020804800206C2A0020782A0020BE
:104EA000154B1B78222B154B05D093F8B10000F061
:104EB000010038F044BC124AD3F80C1192F8742265
:104EC000013A18BF012291B110B40C688888216999
:104ED0005DF8044B08420B490CBF10B2012008805A
:104EE00093F8B1004A8000F0010038F028BC054971
:104EF00010B208804A80D8E745470020B0A50020BE
:104F000018490020484700202DE9F84FAE4C2DED00
:104F1000048BA36820469847002800F0D980B4F994
:104F20000E30A17D06EE903AB4F9103007EE103A3B
:104F3000B4F9123007EE903AF8EEE66AB8EEC77AA6
:104F4000F8EEE77A0929C4ED126A84ED137AC4ED0C
:104F5000147A04F1480600F0BF809C4D30461FF0E3
:104F6000ABFDAB8D002B40F0C180994B1B685B07FC
:104F700000F1E880AB6A94ED137AB3F9022094ED66
:104F8000128AD4ED147AB5F800B0DFF86C828F4F36
:104F900006EE902A8F4AF8EEE66A92F8B293B3F9D9
:104FA0000420B3F9003037EE667A06EE102A06EEDA
:104FB000903A894B84ED137AB8EEC66AF8EEE66A49
:104FC00093F800A0B4F8443077EEC67A38EE668ADB
:104FD00009EE103A0025A945B8EEC99A84ED128A67
:104FE000C4ED147A1AD0BBF1000F23D1D8ED008A9A
:104FF000A8EC018A78EE688AA94568EE898AC6ED30
:10500000038A00F0A2800135032D07F10C0726D09A
:10501000A94506F1040696ED008AE4D1BAF1040F21
:10502000E1D1B0EE480A39F00BFE6C4B1880BBF1B1
:10503000000FDBD0D7ED027A97ED037A78EE676A3E
:1050400097ED018AE7EE267A77EEC86AC7ED027A15
:10505000A7EE268A87ED018A86ED008AC6E794EDE1
:10506000137AD4ED167A94ED126AD4ED156A27EE10
:10507000077A67EEA77AA6EE067ABAF1040FE6EE93
:10508000A67A94ED146AD4ED176AA6EE067AE6EED7
:10509000A67AB1EEC70AB1EEE77AD4ED006A26EE41
:1050A000800A26EE878A84ED180A84ED198A0CD1CD
:1050B000DFED4B8A494D20EE280A39F0C1FD28EE7C
:1050C000280AA88039F0BCFD2881012384F86830C3
:1050D000BDEC048BBDE8F88F3C4D04F12001304657
:1050E0001FF082FCAB8D002B3FF43FAFD5F828E0DA
:1050F000DFED3C6A3C483146AEF102020EF1040C91
:105100000027B3F5C87F1CBFD0ED007AB8EEE77A70
:10511000D1ED007AE1EC016A08BFB0EE667A77EE75
:10512000877AFDEEE77AE0EC017A22F8027F944577
:10513000E7D1012B1CD0013BAB85254B1B685B07DE
:105140007FF518AF31F06CFC14E7BAF1040F7FF46F
:105150005AAFB0EE480A39F073FD9FED240A1F4B99
:1051600028EE800A588039F06BFD1C4BD8804AE746
:105170001F48DFF888C0D0F81811B4F80C80D0E9C7
:105180004420C8318CFB01A9C917C1EBE911C83211
:10519000A1EB0801AEF804108CFB0281D217C2EB20
:1051A000E112C830AEF800208CFB002CC017114A69
:1051B000C0EBEC10AEF80200C2F80A30D781FAF763
:1051C00063F9AB8DB7E700BF9C7F0020BC7D00205A
:1051D00080790020047500204547002048470020C2
:1051E00000007A4400000000C0A600200AD7233C3B
:1051F000B0A50020B0790020CCA600201F85EB517F
:105200002DE9F04F2DED048B274C94F82861022EE8
:1052100093B0074640F02882DFF898B0DFED235ABC
:10522000BBF812509FED226A012384F8293194F8CB
:105230002C3107EE905A06EE903AB8EEE75AF8EEA7
:10524000666A04F5987004F5BC720023F0EC017AEC
:1052500077EEC57AF4EEE57AF1EE10FA88BFF0EE5B
:10526000657AF4EEC67AF1EE10FAB8BFF0EE467A3F
:10527000022B21D0B0EEE77AF4EEC76AF1EE10FA15
:1052800000F3BE82B0EE667AF5EEC07AF1EE10FA67
:10529000ACBF37EEC77A37EE277A0133032B82EDA6
:1052A000007A1ED00432D1E7B0A500200000FA43F6
:1052B0000000FAC3F078002094F82D1107EE101AC0
:1052C00094F82E11B8EE477A09B9F1EE677AF0EE4C
:1052D000E74AB4EEE47AF1EE10FAD5DD0023C4F823
:1052E0008031D64BD4ED4F7A1A68FDEEE77A12F48E
:1052F000805217EE903A40F09282BBF81410994217
:1053000000F3FF82B3F5FA6FD4BFC1EB0300C1F520
:10531000FA604FF47A73C1F5FA6100FB03F3B3FB53
:10532000F1F394F84017002940F00B8303EB83015D
:1053300003EB410342F6F7208342194600F3A682AD
:1053400013F57A7F00F3DE82B4F9483707EE903A1E
:10535000F8EEE77AC4ED617A002A40F0A282B4F850
:1053600070375A0640F1D58040F62B021A40B44BF4
:1053700094ED5F5AD3ED033AD3ED027A93ED044AEC
:10538000D3ED096AD3ED052AD3ED064A93ED077AEA
:10539000D3ED085A94ED5E2A0CBF94ED603A9FED70
:1053A000A93A37EE840A33EEA21A77EEE31A77EEC3
:1053B000A39A72EEC48A33EEE26A77EEC47A72EE92
:1053C000842A34EEA64A77EE653A67EE847A74EE64
:1053D000E60A26EE236AB0EE674AA0EE204AF0EE17
:1053E000463AE0EE203A34EE879A74EEC74A37EE3A
:1053F000257A35EEE68AA1EE474AE1EE073A75EEE8
:10540000A65AF0EE466AD1EE076A34EE464AB6EE88
:10541000001A77EEA33A24EE014A61EE633AA8EE51
:10542000884A36EEE77AB0EE668AE9EE893AA0EE6F
:10543000608AA0EE207A23EEA36A77EE887A27EEC0
:10544000017A67EE817AF0EE466AA1EEA57AD4EE93
:10545000046AA4EE046AE2EEA47A23EE871AF0EE60
:10546000464AB0EE666AA7EEE76AE7EE474A67EE9D
:10547000272AB0EE418AA4EE278A63EEA71AB0EE7F
:10548000620AE7EEE74A75EE055AA7EE076AA4EE50
:10549000630AE7EE476AF0EE610AA4EE671AE4EEEB
:1054A000070A65EE885A25EE066AE2EE245AE4EE13
:1054B000471A72EE024AE4EE232AE7EEA76A25EEC7
:1054C000005AA1EE246AA2EE205A71EEA11A72EEE1
:1054D000A22A66EE836AF0EE004AE1EE835AA2EE5B
:1054E000836AE5EE246A83ED0A4AC3ED0B3A83ED45
:1054F0000C7AC3ED0D7A544BC4ED5E5AC3ED005ADD
:1055000083ED016AC3ED026A84ED5F6A0AB9C4EDF6
:10551000606A0EF05FF994F8B130DB076BD44B4A48
:10552000DFF83CC10FA902F1080512F8010F04EBE6
:105530008003D3ED4C7AFDEEE77A013117EE903A15
:10554000B3F5FA6FA8BF4FF4FA63B3F57A7FB8BF2B
:105550004FF47A73A3F57A73C3EBC3135B00ACFB10
:1055600003E39B097F3B012808BF5B42954201F89A
:10557000013CDAD14FF0000C35488DF844C0654647
:1055800062464FF0010E10F8013F04EB8303D3EDA8
:105590004C7AFDEEE77A0EFA02F117EE903AB3F587
:1055A000FA6FA8BF4FF4FA63B3F57A7FB8BF4FF430
:1055B0007A73A3F57A73C3EBC3135B00B3F5FA3FB9
:1055C00041EA050102F10102A4BF4DB24FF0010C06
:1055D000082AD8D1BCF1000F01D08DF844501D4BE2
:1055E00093F87412D3F89822032900D01AB1117BD2
:1055F000002900F043840022DFF868801546164B2E
:1056000084F828211B78002B00F0DA8098F800300D
:10561000472B07D104EB8603104AD3F880379B1140
:1056200022F8163004EB8503D3F880379B11C4F8B9
:105630008C3713B0BDEC048BBDE8F08F807900206F
:10564000EC0500200000000024AD002067430508A1
:105650006F430508184900200C7E002048470020B1
:10566000D34D62104547002001239E4284F88831C3
:1056700000F0998094F88931002B40F0C68094F8AE
:105680008A310093002BB6D0002384F88A31B24BC4
:10569000B24A1D781168002D40F0CE808F4240F252
:1056A000E38294F88B31002B00F0AD85DFF8D492C3
:1056B000DFF8D48201969FEDAA8ADFF8A8A2DFF86E
:1056C000CCB24E46C1460EE0A64841469847032D4F
:1056D0004DDD94F88B31A6EC010A01359D4209F1AC
:1056E000040980F2E982DBF82C10DAF80430072D87
:1056F000D4BF1BF805805FFA85F80029E4D0414645
:105700009848984704EB4803BBF81A10B3F8D8310F
:10571000994215D807EE903ABBF81C30B8EE677A7C
:1057200007EE903AF8EE677AF4EEC77AF1EE10FAE7
:1057300088BFF0EE477AFCEEE77A17EE903A99B21E
:10574000D4F80032180507D5012303FA08F8DBF86E
:105750002C3018EA030F04D1BCEEC00A10EE103A48
:1057600099B207EE901A032DB8EE670AB1DCB5EED8
:10577000400AF1EE10FAACD0B9F8003007EE103A5A
:10578000B9F80230B8EE477A07EE903A30EE470AA1
:10579000F8EE677A20EE080A77EEC77A80EE277A6D
:1057A00037EE080A95E70FF03BFE6F4BDFF8E0811C
:1057B0001B780222154684F82821002B7FF426AF9F
:1057C000F5F7B0F9C7F101031844684B1B68DF69AE
:1057D00004EB8603F909D3F880374FEAA31CBCEB2E
:1057E000D71F1CBF8B019911B20088422244CBBF46
:1057F000800103F1FF33C2F88007C2F8803705E764
:10580000002142F8041B013320E5DFF858A1DAF843
:105810000C3050469847002384F889312FE7B3F5C0
:10582000FA6FA8BF4FF4FA63B3F57A7FB8BF4FF4AD
:105830007A73A3F57A7374E5DFF8548194F88C21B8
:1058400098F800C08F4201D9013D1D70D4F8B432E0
:10585000002A00F0A18043498869002808BF384623
:10586000002B40F0D8829FED420A9E464FF44871CB
:10587000BCF13E0FC4F8B402A4F8B81284EDAF0A2C
:1058800000F08B843B4B83F800E0ADE0B4F95E3769
:1058900007EE903AF8EEE77AC4ED617A002A3FF419
:1058A0005EAD354BDB78002B7FF459ADD4F8FC218D
:1058B00094F86C3702F08072002B40F0F682002AD8
:1058C0003FF44DAD9FED267A2C4A77EEC77AFDEE78
:1058D000E77A17EE903A1BB21B0382FB0312DB1729
:1058E000C3EBA213C5F5FA6212B202FB03F343F352
:1058F0000F332B4407EE903AF8EEE77AC4ED617A65
:105900002DE51146DFF874E0C8178EFB01C3C0EB2C
:10591000A31004EB40034FF47A78B3F948C7B3F906
:105920004A3708FB1011A3EB0C0301FB03F38EFBBA
:105930000301DB17C3EBA11363441BB207EE903ADC
:1059400006E594F8411703FB01F10D4B83FB0103BE
:10595000C917C1EB6313E9E4847D0020807D00203A
:1059600000007A44647D00200C7E0020ACA500205D
:1059700000409C4450860020887D0020D34D62105A
:105980001F85EB5140A700208C890020F078002073
:105990004547002000247449002B00F035824FF663
:1059A000DC70FB1A9842A8BF1846B0F5487FB8BF14
:1059B0004FF4487007EE900A1FED0A7AF8EEE77A86
:1059C000A3EB000E87EE270ABEFA8EFE81B24FEAE5
:1059D0005E1EA948A4F8B812BCF13E0F80F800E0A2
:1059E00084EDAF0A00F0A383BCF1270F03D139F097
:1059F00027F9A24B1880A24D2B68DA0400F1F3813D
:105A000094F8C332022B00F04983042B00F03A8350
:105A1000012B00F01C82D4F8D0229A49BB1A8B4289
:105A200038DC974238D007EE903A974BDFED976A13
:105A300093F828309FED967A9FED965AB4F8C422D9
:105A400006EE103AF8EE677AB8EEC66A67EEA67A06
:105A500037EE467AF7EE006A27EE057A77EEE65AD9
:105A6000B4F8C632E7EE256A9A4227EE277A87EE27
:105A7000266A40F06D82884BB3F90020B3F902101A
:105A8000914240F05182B3F90420B3F906109142DB
:105A900040F03682C4F8D072804B9F4200F2AC8155
:105AA00018F024FB81460EF015FB94F8B12094F811
:105AB000ECB298F8003012F0010200F0B980724A9E
:105AC0000028527EB8BF40425FFA80FA52459CBF20
:105AD000012284F8ED2294F8EE22EAB1BBF1010F25
:105AE00021D094F8ED1284F8EF12E1B9B9F1000F6A
:105AF00019D16B490878CDE9012319F0BBFADDE92A
:105B0000012380B967480099006890F83600003892
:105B100018BF0120009007E094F8EF1219B9B9F10D
:105B2000000F00F0E881002184F839155E490098E3
:105B300084F8F8024878002874D094F8D406002835
:105B400070D194F8D50600286CD194F8D6060028B8
:105B500068D153480078CDE9002319F08BFADDE9CC
:105B60000023514900285DD12868C00600F16183F7
:105B7000087942004B2AA8BF4B228245D2B280F05E
:105B800079839245C0F05C83484ADFED497A92ED13
:105B90000B7AB0EEC77AB4EEE77AF1EE10FA40F184
:105BA0004F8392ED057AB0EEC77AB4EEE77AF1EE64
:105BB00010FA40F1458392ED117AB0EEC77AB4EE57
:105BC000E77AF1EE10FA40F13B83D4F82C270AB9BA
:105BD000C4F82C774988D4F82C07D4F83027BAF1C8
:105BE0004A0F88BF4908121A4FF47A753A4405FBE8
:105BF00001F18A4202D9012184F8D416002800F06C
:105C00002B831F2B07D11D4B012199804FF47A71F3
:105C1000B2FBF1F2DA80BBF1010F00F0AA8201229F
:105C20001546ECE41F2BF6D1144B00225A60F2E724
:105C30001C4884F8ED22012184F83915016884F8A4
:105C4000EF2291F83610003918BF01211F2B84F87C
:105C5000F81201D1094B5A60BBF1020F00F0A78284
:105C6000002384F8EC32DAE7DFF8488094F88C21DE
:105C700098F800C0EAE500BF5086002048470020A1
:105C80008079002090D00300F0780020BD37863660
:105C9000000080430000803BEC050020404B4C009E
:105CA000A8950020E4780020D878002094AC00204B
:105CB0000000C84245470020D4F8FC21DFF868C343
:105CC000019EDCF80000049002F4807194F88C21AD
:105CD0000291002A40F0CD80914694F8051284F894
:105CE00004920391002B00F0A2829AF80000BBF806
:105CF0001250DFF838A30A920138C1B20791BF48A9
:105D000003990B97A0FB010E09EE105A0EF0FE0549
:105D100005EB5E054D1BEDB20595BBF81A50B84872
:105D20000195BBF81C500695049DC178DFEDB58A3E
:105D30009FEDB58A05F596754FF0000ECDE9085632
:105D4000CDE90CC04E46B8EE499ADDF81C900AF138
:105D5000D80B0AF5907875460A461F4630E0BCEE2F
:105D6000E77A17EE103A98B2019B98422FD3069B20
:105D700098422CD8089BCBF80030002A00F0B48160
:105D8000032D00F308811646F4EEE87AF1EE10FADE
:105D900088BFF0EE687AF4EEC87AF1EE10FAB8BF78
:105DA000F0EE487AB9F1010F40F2FF800135BD42B3
:105DB000EAEC017A0BF1040B08F1060800F03881D7
:105DC000924B03EB8500D0ED007A002EC7D1002A5C
:105DD00000F0D380032D00F3DE80032D00F0A081BE
:105DE000F0EE497AD0E7D4F8FC31DB073FF508AE96
:105DF00004200CF0EBFC03E6814B9A78002A7FF438
:105E00004FAE01229A704BE69FED810A96464FF401
:105E100048711346DDE54FF6DC7EC31A9E45A8BFE8
:105E20009E46BEF5487FB8BF4FF4487E07EE90EA25
:105E30009FED787AF8EEE77A1FFA8EF1A3EB0E0E5B
:105E4000BEFA8EFE87EE270A4FEA5E1E10E5D4F8F2
:105E5000C832FB1A002BFFF6DEAD07F59C4320335A
:105E60000320C4F8C832F6F77DF98008A4F8C6020A
:105E7000D1E5B1FA81F94FEA59192EE701201073E3
:105E8000D3F8A8320FAAC3F89C2040F20312C3F83B
:105E9000A410A3F8882019460922C3F8A02051F8BD
:105EA000880B32F0C5FDFFF7A6BB9FED5B7A5B491F
:105EB00077EEC77AFDEEE77A17EE903A1BB21B0336
:105EC00081FB0301DB17C3EBA113002A00F07B81E8
:105ED000C5F57A7212B202FB03F343F30F332B447E
:105EE00007EE903AF8EEE77A0123C4ED617A84F880
:105EF0006E37FFF734BABBF1010F3FF414AEF8E58B
:105F000007EE902A94EDB97A84EDBA6AF8EEE77A52
:105F100077EEC77AA6EE277A84EDB97ABDEEC77A16
:105F200017EE102ADA80B5E507EE902A94EDB77ADD
:105F300084EDB86AF8EEE77A77EEC77AA6EE277AAC
:105F400084EDB77ABDEEC77A17EE102A5A809AE52B
:105F500007EE903A94EDB57A84EDB66AF8EE677A7A
:105F600077EEC77AA6EE277A84EDB57ABCEEC77ACB
:105F700017EE103AA4F8C4327DE5029B5BB9DBF85A
:105F80000000049B181A0028C0F2AB80032DDCBF70
:105F9000002684F80462E8B207921BF0CBF807EE03
:105FA000900A079AF8EE677AEEE6FCEEE77A94F844
:105FB000983217EE901A88B2059928F811002BB97B
:105FC000039B022B15D9012084F89802B8F802002F
:105FD000B8F800C0124B8444B8F8040084440FFAA7
:105FE0008CFC23F815C00F4B83FB0CE0A0EBEC708E
:105FF00080B207EE900AF8EE677AD7E6ABAAAAAAB3
:10600000887D002000A00C4500803B4440A7002074
:1060100000409C440024744900007A44D34D62102F
:106020004CA8002056555555642A0020E0A60020B3
:10603000DDE90B7CB1460A9A099E0D98B9F1000F73
:106040005DD00369DCF80010C160002B00F0C8804F
:10605000CB1A016A8B4200F3BA80DFF8908298F87D
:1060600000C0BCF1280F07D1D4ED4F7A8F4DFDEE63
:10607000E77A17EE903AEB80039B013384F8053200
:10608000FFF7E4BBF4F74EFDD4F8CC32884AC01ACF
:106090009042C4BF0023A4F8C432BCE4854B864AB6
:1060A000DB7B04EB8303D3ED4B7AFDEEE77A17EE4F
:1060B000903A1BB2B3F5FA6FA8BF4FF4FA63B3F589
:1060C0007A7FB8BF4FF47A73A3F57A73C3EB832357
:1060D000A2FB0323C3F38F13A4F8C432A4F8C6327F
:1060E00099E4DAED007A4FE6029B002B3FF44CAEC8
:1060F00051E794F80532714884F804220393DCF8E0
:1061000000106F4DC3680161C91A2B6843F0040386
:106110002B6043689942C4BF002380F825309CE778
:106120006848038807EE903AF8EE677A2CE65F4DF0
:106130006548019280FB03C0DB17C3EBA0036348F3
:10614000A5F804E0A0FB0101C908E98047F6FF714A
:106150008B42A8BF0B462B8038F072FD94F8C21218
:10616000B4F8C032019A2881002940D0AB81EA817D
:1061700041E4574B1B6893F869305345BFF44FAD6A
:10618000022384F8EC32534B00225A60DA615A63DE
:1061900043F8502F5A609A6041E54F4DA5FB0050DF
:1061A000424D400968804D4880F800E0C0E7036830
:1061B00093F86C30002B3FF432ADD4F8003259051F
:1061C0003FF52DAD4CE584F86E27FFF78BBB3C49BE
:1061D000012380F825300B6823F004030B603CE7B3
:1061E000374D0161296841F00401296031E76420DD
:1061F0003B4900FB03F381FB03011944DB17C3EBAD
:1062000061239BB2B2E7DFF8E8C094F88C21DCF898
:106210000030D4F8FC31002A3FF46BAF83F4807374
:10622000C3F3002994F8053284F8049203932348B9
:1062300004E7002A7FF49CACB9F1000F7FF498AC1E
:10624000D4F82C1729B1D4F83027521A3A44C4F89C
:1062500030270022C4F82C271F2B7FF4DCAC134A14
:10626000002393804FF47A71D4F83037B3FBF1F305
:10627000D380D0E41B48DFED1C7A90ED007AB4EEB9
:10628000E77AF1EE10FABFF67FAC90ED017AB4EE4A
:10629000E77AF1EE10FABFF677AC90ED027AB4EE41
:1062A000E77AF1EE10FAFFF66CAC6DE44847002097
:1062B00060E31600F0780020D34D6210887D002046
:1062C000547E0020B07D002067666666CDCCCCCCC5
:1062D000E478002094AC00201F85EB51508600200C
:1062E0000308208088AC00209A99193E4547002079
:1062F000642A00202DE9F843974B1B685A0701D404
:10630000BDE8F883DFF89082944F98F80030944C01
:1063100097F83860372B04BF924B1E8063681A7859
:10632000012A054607D0042E00F20B81DFE806F0B3
:106330008EB29BA6160093F904208B4B642101FBBF
:10634000023393F85920202A00F0BE80874A0123A7
:1063500084F8883113704FF47A7771E0D4F89C3068
:1063600083489847002800F0B5808249D4F8A030CF
:10637000081D9847D4F8AC90B9F1000F40F3BA80EB
:1063800007EE909A9FED7C0ADFED7C0AF8EEE77A43
:1063900027EE800A38F07AFB79499FED7A7A7A4ABB
:1063A0000878F7EE007A77EEC07A67EE877A92ED9A
:1063B000007A002800F0A78077EEC77AC4ED297A2A
:1063C00098F80030372B17D107EE909A9FED6F0A9F
:1063D000DFF89081F8EEE77A27EE800A38F030FC9B
:1063E000D4F8A83094ED290AA8F80200A8F80430DF
:1063F00038F026FCA8F8060094F88030002B4ED127
:10640000052387F8383098464FF47A77012384F8CB
:10641000883104EB8606F4F785FBD6F89037401BED
:10642000984204EB880388BFC6F89007D3F89037EA
:10643000C4F88C37002F3FF463AF0A2FB8BF0A2788
:10644000534B1B681B681F61BDE8F883D4F88C3080
:106450004748984700283DD0012387F838309846B0
:106460004FF47A77D2E7D4F8943041489847032321
:1064700087F838309846B4F88470C7E7D4F8983075
:106480003B48984730B3042387F8383098464FF498
:106490007A77BBE7D4F8903035489847D0B10223DB
:1064A00087F83830F4F73EFB04EB8606401BD6F83D
:1064B0009037834219D2C6F89007D4F89837C4F8B9
:1064C0008C374FF47A77B8E79B699B691B047FF59B
:1064D0002AAF3BE797F83830244A0121022B11708C
:1064E000E0D098464FF47A7790E7D4F89837C4F81C
:1064F0008C37E6E7224B1B78002B7FF461AF00233B
:10650000C4F8A4305CE7DFF894C0224BB3F800E095
:10651000BCF8003001339BB277EE877A9E45C2ED1E
:10652000007AACF80030EAD807EE103AB8EEC77A35
:106530000123C7EE876AACF800000B70C2ED006A59
:10654000DDE7D4F888300A489847002387F83830C8
:106550009846B4F8827059E7987F0020EC05002037
:10656000B0A50020484700203C3100200C7E0020D0
:10657000B4A5002058A6002008942537B1DC423E7F
:10658000FC950020D048874AF89500200AD7233C84
:10659000ACA50020FE950020454700200096002075
:1065A00070B5104D104C2E1D15F8010BFF2814D09E
:1065B00006F032FE2279617980EA0203DBB2994269
:1065C0000BD0801AB0FA80F02268400900011AB19D
:1065D00091881268814091616371AE4204F10804B0
:1065E000E2D170BD58AD002008700020034B93F835
:1065F000AC2793F8AD1734F0FDBB00BFB0A5002069
:1066000010B5124C23681B6B9847114B114A9978AF
:1066100040F2DC500023032998BF1046A360A4F881
:106620000530F4F759FF0C4B93F8AE37012B0AD025
:1066300007D9023B012B08D8084B0322C3F80C25CD
:1066400072B6F2F7D3FD31F007FC10BDB48700201D
:10665000343B0020FCA60700B0A50020002000402D
:10666000034B93F8B10010F0010000D07047C7E76A
:10667000B0A5002038B50C4D95F8B13013F00104E9
:1066800000D038BD094B01229A73F8F7DFFDF8F707
:10669000B9FA95F8AF37002BF3D085F8AF47BDE8CE
:1066A000384025F02BBD00BFB0A50020F86F0020BA
:1066B000F8B5384C2368002B57D00A2801D00D2894
:1066C00051D1354D95F8B0370BB1F9F781F8334E0C
:1066D0002321304638F0F3FF08B1801B2060236887
:1066E000002273B902B12360F9F73EF895F8B0378C
:1066F000F3B1BDE8F8402A48F9F762B801220B4629
:10670000EFE7591E705C2028F8D092B90022254C82
:10671000224FF2543726013E0DD13146224B9C4286
:1067200012D2E3682068984795F8B137002BDBD187
:10673000F8BD2360EAE721683846FDF7CFF9014646
:106740000028EBD11034E6E795F8B03723B11749AC
:106750001748F9F711FDC7E71648F9F731F80F4860
:10676000F9F74EF8C0E7FF2BE2D8A0F120025E2A2D
:10677000DED80BB92028DBD05A1C2260074AD0543F
:10678000054B93F8B037002BD2D0BDE8F840F9F7AD
:1067900061B800BF5C7F0020B0A500205A7E0020B9
:1067A000AEDE0508084005086843050843F40508FF
:1067B0005FF4050865F4050838B5074C074DAC4291
:1067C00003D3074B01221A7038BDD4E90210A28806
:1067D00039F03CF81C34F2E794FE05081C07060863
:1067E000287000202DE9F04F0E4693B09F49834654
:1067F00030461746FDF772F90546002840F01F8124
:106800009B493046FDF76AF90546002840F019819A
:1068100098493046FDF762F90546002840F013819B
:1068200095493046FDF75AF90546002840F00D819C
:1068300092493046FDF752F9002805460ABF012467
:10684000082435467F4207F010078D4928463C430F
:10685000FDF744F9002800F0FA8044F02004894B49
:106860001B780BB9FFF7A8FF2EF0B6FC14F0090F48
:1068700000F038838448F8F7C9FF0020FDF758FA84
:1068800014F48073049340F0EC808048F8F7BEFF66
:106890007F48F8F7B5FF04F01803182B05D17D48A1
:1068A000F8F7B4FF7C48F8F7ABFF01230393F8F740
:1068B0008FFF7A497A48F9F739F87A497A48F9F72F
:1068C00035F804F48473082B07D178495846F9F752
:1068D000FFF876495846F9F787FE14F080030793CE
:1068E0000ED1734B93F8B427002A724A03F2B473A3
:1068F00006BF0121134600216F4A2046F8F76CFFBE
:106900006E492046FDF74EFA6D492046FDF722FEFE
:106910006C492046FDF710FB6B4BD3F800A06B4B86
:1069200014F010061D6840F09E806948F8F76EFF6D
:106930000296684BCDE905336AEA05034FF000087B
:106940000993069B53F8049B0693B9F1000F21D0DD
:10695000099B029A012707FA08F73B400CBF012167
:10696000002120460893FAF775FA65EA0A033B42CC
:1069700014BF01210021584A02904B462046F8F7E7
:1069800073FF0899544A00394B4618BF012120462D
:10699000F8F722FF08F10108B8F11D0FD1D165EA1F
:1069A0000A034FF000080693059B53F8049B0593D8
:1069B000B9F1000F24D0012707FA08F73D420AD0A9
:1069C0006AEA05033B42454A4B4614BF01210021B8
:1069D0002046F8F749FF1AEA070F11D0069B029AE2
:1069E0001F400CBF012100212046FAF733FA391E5F
:1069F00002903A4A4B4618BF01212046F8F7ECFEB8
:106A000008F10108B8F11D0FCED1354B354A364992
:106A10002046FBF7D5FB079B002B6DD0134B22467E
:106A200018215846FAF746FA039B002B00F0B8816C
:106A30002E48F8F7EBFE2E48F8F7E2FEB0E101240D
:106A400000E70224FEE60424FCE68124FAE6294954
:106A50002846FDF743F800283FF401AF44F4807462
:106A6000FDE6002322E71A4B029362E791F4050842
:106A700098F40508A0F40508A6F40508AFF4050885
:106A8000D3EF050828700020B8F40508C0F4050805
:106A9000D8F40508E4F405080CF50508A2E4050897
:106AA000EBE40508F9E405080EE5050883FE050892
:106AB000B0A5002097F905081CF5050829F505087B
:106AC00033F5050850E10508E0A400207C7900209A
:106AD00072F405082411050839F5050845F505087F
:106AE00050F505082479002078A2002009F6050851
:106AF0001FF60508B3F40508DFF8BC93DFF8BCA364
:106B000099F800209AF80030DFF8B4839A4214BF55
:106B100001210021B64A20460CBF01270027FAF7C1
:106B200099F99AF80030B34A013B394658F82330B6
:106B300005462046F8F798FE99F80030AD4A013B2B
:106B40003946AD4F58F823302046F8F745FED7EDCB
:106B5000007AAA4AF5EE407AF1EE10FA0CBF012154
:106B600000212046F8F738FEA5492B463A46204634
:106B7000FBF7AAFDA34BA44AA4492046FBF7D6FF86
:106B80002EB1A34B93F90230002B00F00F81A148E6
:106B9000F8F73CFEA048F8F733FE00239C4A9F49D3
:106BA0009F4FA04D2046FCF7F7F89F4B9F4A01935B
:106BB00000923A6829682046FCF73AFF40F2022228
:106BC0009B4B01930092BA68A9682046FCF730FFFE
:106BD000002E40F0ED809748F8F718FE3246964FA9
:106BE0009648DFF8E0C20125002117F8013B10F8B4
:106BF000018B03F1480EEE440EF8208C1CF801EBDB
:106C00000EF14809E94409F8108C002D00F0D280FB
:106C1000A3EB0E056B426B41013108291D46E4D1FF
:106C200083F00101002720468DF83070FAF712F941
:106C3000834A8DF840700EAB29462046F8F714FEC3
:106C40007F4A0AAB29462046F8F7C6FD7D4B7E4AAF
:106C50007E492046FBF76CF97D4B7E4A7E492046F3
:106C6000FBF7FCFB7D4B7E4A7E492046FBF79CFEF2
:106C70007D4B7E4A7E492046FCF788FB7D4B7E4A51
:106C80007E492046FCF764FA002E40F095807C484F
:106C9000F8F7BCFD02967B4E7B4FDFF82C82002577
:106CA00039460222304638F043FE002814BF012145
:106CB0000021029A96F800A020460CBF4FF001096F
:106CC0004FF00009FAF7C6F8BAF1020F029076D138
:106CD0007B784FF0190A40F2EE221AFB032301934E
:106CE0003B786A4A18F80330009349462B46204601
:106CF000F8F7BAFD737840F2EE221AFB03230193F2
:106D00003378624A18F80330009349462B462046F0
:106D1000F8F762FD0135122D06F1020607F10207B0
:106D2000BED100215A4B22465846FAF7C3F8210734
:106D300040F1CC800025E9B2224658460135FCF7E7
:106D4000AFFF042DF7D1534E534D33782B70049B76
:106D500033B95248F8F75AFD51495846FAF77AFEC6
:106D6000FF232B700025E9B2224658460135FCF777
:106D7000BBFF042DF7D14B4C73782370049B002B81
:106D800032D14948F8F742FD45495846FAF792FE94
:106D90004648F8F73BFD4648F8F712FDFF232370FD
:106DA000002013B0BDE8F04FFAF761B8194BF5E6D3
:106DB000204A14E72B462FE7314B02936BE73B78D1
:106DC0003C4A18F80330009349462B462046F8F712
:106DD0004BFD3378374A18F80330009349462B4669
:106DE0002046F8F7F9FC95E7FF2323701CE600BF67
:106DF00080F4050857F505080C89002060F50508A2
:106E0000E0A2002038ED05089C8900202C9A002083
:106E1000FC8900207AF405086FF50508B899002070
:106E2000607A0020F4A400207CF50508FFFF7F00B5
:106E300083F5050886F40508A0A3002050870508FF
:106E400082E805088AF50508C07900201C9E00200C
:106E50008EF50508E0870020A49A002097F5050824
:106E60008C890020909A00209FF50508447C002022
:106E7000A49C0020A8F505086C8A0020ECA3002043
:106E80008AF40508D49B002088870020A2E8050822
:106E900091F40508D8A3002068040020ACF505088B
:106EA00083FE050869040020CFF50508F6F50508FE
:106EB00017F50508B2E80508E8A40020E8780020E6
:106EC00098110508F0780020608905080F4D2246CA
:106ED00029785846FCF7E4FE697822465846FCF7C4
:106EE00003FFA1E5A20706D5084B224619785846AC
:106EF000FCF7D6FE54E763077FF552AF034B2246FB
:106F000059785846FCF7F0FE4AE700BFD8A30020A6
:106F1000002267E4012265E4EFF31182902383F3FA
:106F200012888378B0F800C0002143EA4C039BB27A
:106F30008170D2B282F31188064A180A127880EA68
:106F40001310584002B1C0431B019BB200F00F0068
:106F500018437047C81800202E4A82B093790190D8
:106F6000002B3CD092F82430DFED2B6AD1792B48EE
:106F700007EE903AF8EEE77A294B027886EEA77A88
:106F8000A1F10201B1FA81F103F61C00490983F86D
:106F9000201880ED007A02B3B3F82E18DFED216AD5
:106FA0009DED017A07EE901AF8EE677AB8EE477A0F
:106FB00067EEA67AF7EE006A67EE877A03F5036359
:106FC00077EEA66A002187EEA67A03EBC20219606B
:106FD000083303ED017A9A42F9D102B07047124B9F
:106FE0001B681B01F9D592F82430DFED0B6A0C49C0
:106FF00007EE903AF8EEE77AD37986EEA77A981EF4
:10700000434201F61C02434181F8203882ED007AA8
:10701000E3E700BF343B002055555540341E0020A7
:10702000B0A5002027D4D2368079002070B41A4C45
:107030001A4B90F85850A4FB02425209A3FB02439A
:10704000DB0803EB8303A2EB4303DCB2A542026837
:1070500020D000EB830C4668DCF83050751BDCF860
:10706000086045600025CCF80850CCF830509B00F3
:10707000921B80F858400344013202609A68013242
:107080009A6029B94268013242601A6B01321A6370
:1070900070BC70479B00EEE71F85EB51CDCCCCCC8C
:1070A00038B5094D2B7963B100242B685B6B204602
:1070B0000BB1984708B9002038BD2B7901349C42A8
:1070C000F3D3012038BD00BFB48700200C4B93F8E8
:1070D000392012B90B4B987970470A4A906800B969
:1070E00070470949096840F6B83C091A614504DD52
:1070F0000021907983F8391070470020F0E700BF35
:10710000EC050020B4870020642A00202DE9F84F08
:10711000DFF80C821F46531ED8F8005091460646F1
:10712000142B00F2AE80DFE803F05656565656ACEC
:107130000B0B0B0BAC0B0B0BACACACACAC0B0B00E4
:107140004FF47A7B4FF00A0A012F4AD0002F40D12A
:107150006E4A6F4B14781878631C03F00303834264
:1071600037D06C4D137004EB440305EBC3034FF4AD
:107170007A7283F80CA09A604FEA4408B1B11823E0
:1071800003FB04530C3309E0FF2E07F101070CBF8A
:107190004A460022B94203F8012F07D0BE42F3D17C
:1071A00001374A46B94203F8012FF7D1FFF778FFBC
:1071B000002800F09E80584A08EB0403DB00D26BE5
:1071C000E9180120E85402F51C530F33B3FBF2F326
:1071D0004B60BDE8F88F012FDFF848B14FF0010A8E
:1071E000B4D14E4A537C012B03D0022B00F089808E
:1071F000002798F80400E0B1454B1C78454B182255
:107200000C2112FB04121A44002309E0FF2E03F1A3
:1072100001030CBF49460021834202F8011F08D038
:10722000D9B28E42F2D101334946834202F8011F9E
:10723000F6D142F22830F4F74FF94FF47A70F4F7B0
:107240004BF90FB9EB6998472B6A03B1984798F847
:107250000430DBB1002420460AE0FF2E0FD0204688
:107260009847013498F80430E4B29C4220460DD28D
:10727000EB6B9847A642AB6A4FF00001EDD149464F
:10728000EDE74FF47A7B4FF0010A5DE7AB6903B19C
:107290009847EB6A98475FB90AF1FF3A1AF0FF0A7C
:1072A00012D04FF47A70F4F717F9EB699847CBE7EF
:1072B000EB690AF1FF3A98471AF0FF0A04D04FF43D
:1072C0007A70F4F709F9BFE75846F4F705F998F82A
:1072D0000420002A3FF47DAF0D4B0E481C780D2191
:1072E000182313FB041318440021BDE8F84F38F0AD
:1072F000CFB908EB0403DB00EA18E8545060BDE89E
:10730000F88F9778083F18BF012772E70C2B0020F1
:107310000D2B0020102B0020EC050020343B00201A
:10732000B4870020A08601002DE9F041134C247899
:107330000CB9BDE8F08180460F4616461D46CBB11C
:10734000012BF6D10E4B987980F001000028F0D087
:107350002F2EEED80B4B0C4A1B781278013303F01A
:1073600003039342E5D02B46324639464046BDE8FA
:10737000F041CBE6FFF7AAFEE8E700BFB0870020A8
:10738000B48700200C2B00200D2B002010B5437B70
:1073900082680446581C6073D154627B237B9342FD
:1073A00000D910BD002AFCD02368D4E90101984718
:1073B0000023637310BD00BF427B42B110B5036868
:1073C0000446D0E9010198470023637310BD70475C
:1073D0002DE9F04F06683578012D83B009D0022DD4
:1073E00003D1346A002C00F09180002003B0BDE886
:1073F000F08F96F90460741CF7D0032EF5DC8C4FE7
:107400009C46642303FB067396469A69002AECD0D7
:1074100090F8049093F85900202840F08A8093F85F
:107420005800012800F0858083F85850814D2C6861
:1074300004E02B681B1B192B00F29F80936913F447
:10744000004AF6D14FF0640B0BFB06FB0BF118085A
:10745000BB44222300944FEA49098BF85930B844C1
:1074600040238BF85A300A46CBF85CA0CBF83CE0BE
:10747000CBF84CA0ABF842C00A234946404630F056
:107480007DFD002840F0BC80BBF842309BB2FF2B52
:1074900040F2B980DBF81810674A4B681340674A1E
:1074A00043EA09031A43FF23ABF840304A604FF028
:1074B000640A0AFB067A03E02B681B1B0A2B2BD8F5
:1074C0008A6912F00402F7D0DAF83C304A6A1A707E
:1074D000BAF84230DAF83C20013B9BB2AAF84230BD
:1074E0000132BAF84030CAF83C20BAF84220013BD9
:1074F0009BB292B2AAF8403002B103B3BAF842305C
:107500009BB2002B66D0DAF81810D9E741F0800161
:107510002CF006FC012069E7642303FB067320209E
:10752000D96D83F858200143D96583F8590083F851
:107530005A20434A138801339BB2138055E7DAF887
:10754000181003E02B681B1B0A2B35D88A6912F030
:107550008002F7D0BAF842309BB2FF2B1CD94B689F
:10756000384A134043EA090343F0FF7343F480337E
:10757000FF22AAF840204B60C0E7642303FB067398
:107580002020DA6D00210243DA6583F8581083F871
:10759000590083F85A10CCE7BAF8423029484A68B3
:1075A0009BB2AAF84030DBB249EA034302401343DE
:1075B00043F000734B60A1E7642303FB06772021AF
:1075C000FB6D87F858200B43FB6587F8591087F847
:1075D0005A20AEE72146404630F07CFC03460028A6
:1075E000A7D1DAF81820184C2020D061516821402A
:1075F00051608AF859008AF858308AF85A3089E779
:107600008BF858A095E7BBF84230DBF818100A4811
:107610004A689BB2ABF84030DBB249EA0343024010
:10762000134343F0024343F410534B603FE700BF62
:107630003C31002050430020009800FC0024FF81D2
:107640008E7F0020009C00FC00E800FE10B503685F
:1076500004469B689847FF230122A373627310BD01
:10766000036810B504461B689847236801219B688E
:1076700020469847E37B0133E37310BD2DE9F041C9
:10768000069F044638460D461646984636F076FB69
:107690002844A072E672387850B1069729462568CA
:1076A0002046AC6943463246A446BDE8F0416047F7
:1076B000BDE8F08103689B6A184700BF03685B6DF3
:1076C00003B11847704700BF0368DB6C03B118476C
:1076D000704700BF0B46002110B5C17342749A6C0D
:1076E00003600446017302B19047236801219B683F
:1076F000204698472368FF21A173DB6C0122627347
:107700001BB12046BDE81040184710BD10B40E4B09
:107710000E4C1B7801228240134054F8200071B1B6
:10772000003B18BF012338B18288016883F0010350
:107730001B0102FA03F38B615DF8044B7047B3FA47
:1077400083F35B09EFE700BF782A00206C2A002052
:1077500010B50A4C23681B6B9847094B094A997866
:1077600040F2DC500023A360A4F80530032998BF41
:107770001046BDE81040F3F7AFBE00BFB48700204D
:10778000343B0020FCA6070010B5044C23681B699D
:1077900098470023A371A36010BD00BFB4870020E9
:1077A00010B5074C63791BB12368DB68984700B9B3
:1077B00010BD044B01221B68A271A36010BD00BF65
:1077C000B4870020642A0020F8B5114D00242E1D36
:1077D000522715F8010BF0F795FF01340022202104
:1077E000E4B218B18771C471F0F7CEFA16F8010B44
:1077F000F0F788FF4FF0530C0022402120B180F8B1
:1078000006C0C471F0F7C0FA042CE2D1F8BD00BF85
:1078100020AE0020C3B25E2B9DBF034B03EB800361
:10782000D3F87003014870470840050858B40508AC
:1078300003681B68184700BF03682DE9F0415F6AC1
:107840001FB13B46BDE8F041184704460D461646B9
:1078500000E023689B68204698478642F9D8002EAE
:1078600008DD2E44236815F8011B1B682046984745
:10787000AE42F7D1BDE8F08103685B68184700BFEE
:1078800003689B68184700BF0368DB68184700BFA0
:1078900003689B6A03B11847704700BF0368DB6A3F
:1078A00003B11847704700BF03689B6A70B5044670
:1078B0000D46164603B19847324629462046FFF743
:1078C000BBFF2368DB6A1BB12046BDE87040184748
:1078D00070BD00BF70B504460E46154623682046AD
:1078E0009B689847A842F9D32A4631462046BDE80E
:1078F0007040D9E72DE9F047B64C94F8B1378EB017
:1079000013B10EB0BDE8F087B34B1B685F05F8D527
:10791000D4F8EC39B14AC31A9342054600F32C81DE
:1079200094F8F039012B00F0FD80F3F7FBF894F8A0
:10793000408A00F57A70B8F1010F069000F09B8044
:1079400094F84D3A1BB194F8503A980723D094F824
:10795000523B73B194F8533B002B40F02D81D4F887
:10796000542B94F8596B9E4BB3FBF6F313449D4292
:107970006AD294F86E3B4BB194F86F3B002BC0D0A9
:1079800028460EB0BDE8F04725F066BC94F8703B81
:10799000002BF5D0B5E794F8582A42B1D4F85C0A28
:1079A00010B19049FFF780FF002384F8583A94F80B
:1079B000A07A002F40F0828194F80C3B002B40F01D
:1079C000288194F8A329002A40F0B381864BD4F88B
:1079D000100B196894F8143B2BB1844ED4F8183B63
:1079E000B34200F07183D4F8082B94F8401B7C4B11
:1079F000B3FBF1F313449D42A9D394F8583AC4F869
:107A0000085B002BA3D194F8416BA31993F8447B36
:107A1000F90700F17985BA0700F1EB847B0700F1E3
